:020000040800F2
:1000000000000110F9F90708692A0008B59E0208E6
:1000100099FA070899FA070899FA070800000000FA
:100020000000000000000000000000003D47000844
:10003000414700080000000045470008F10601089C
:1000400099FA070899FA070899FA070899FA070828
:1000500099FA070899FA0708D5C60008D9C6000812
:1000600099FA0708DDC60008E1C600083531000826
:10007000493100085D310008713100088531000800
:1000800099310008AD31000899FA070899FA070874
:1000900099FA070899FA070899FA0708E5C60008C7
:1000A000E12F00080930000831300008CD2F00088A
:1000B000593000086D3000088130000899FA0708AF
:1000C00099FA070899FA070899FA070899FA0708A8
:1000D00099FA0708ED2B0008F92B000899FA070890
:1000E000E9C6000899FA070849470008BD3000082A
:1000F000E53000080D310008A9300008C1310008C2
:1001000099FA0708C93500089530000899FA0708D8
:10011000052C000899FA070899FA070899FA0708C0
:10012000D5310008E9310008FD310008113200081E
:100130002532000899FA070899FA070899FA07087A
:1001400099FA070899FA070899FA070895470008E5
:10015000393200084D32000861320008112C0008C5
:1001600099FA070899FA070899FA070899FA070807
:1001700099FA070899FA070899FA070899FA0708F7
:0801800099FA070899FA070833
:10019000D0E907239A423CBFC1685218D01A704771
:1001A000D0E9092300699A4238BF1218D31A0138DE
:1001B000C01A7047D0E90902101AB0FA80F040095D
:1001C000704700BF0246036A4069D168C05C0133D2
:1001D0008B4228BF00231362704700BF436A8269C5
:1001E000D154436A0169426B01338B4228BF00231B
:1001F0004362D36843F08003D3607047436B188831
:1002000010F0100002D01A889B880120704700BFB0
:10021000436B99891A88890610B504460AD592B2AB
:10022000900607D5E26A002A2AD09888216B80B20E
:100230009047636B99891A88090692B210D5100607
:100240000ED5D4E909128A4215D0A1692069895CCA
:100250000132C9B29980B2FBF0F100FB1122A26217
:10026000998A1A88C90592B204D5D20744BF4FF6BD
:10027000F7721A8010BDDA6822F08002DA60EFE7C8
:100280009B88E2696169DBB28B54E269E168636B68
:100290000132B2FBF1F001FB1022E261CAE700BFBC
:1002A000036942681F2B10B40AD95468A3F1200CCB
:1002B000202101FA0CF1214207D15DF8044B70476F
:1002C0001468202199402142F7D081690024C86830
:1002D0000C7480684C68016821F00101016020689D
:1002E00094F805C00C4C818934F81C4089B221EA8D
:1002F00004011F2B818107D9A3F1200120238B400A
:100300005DF8044BD3607047202101FA03F35DF8D8
:10031000044B9360704700BFC86B08084A1C10B4B8
:1003200018BF4FF0450C494C08BF4FF0800C4FF4FC
:10033000003300E00BB3626B12EA0C0F03F1FF33E2
:10034000F8D0002924DD626B54071DD403291FD087
:100350003E4B5A6BD2071FD402291BD01A69D2B266
:1003600082421DD101295B691CD0062912D113F4E8
:10037000604F43D1364A13600CE0002904DD636B03
:100380005B0701D40329E3D103205DF8044B7047D8
:10039000002BF9D00020F8E701205DF8044B7047EE
:1003A0001020F2E72B4A1A40002AF3D0002B31DB51
:1003B0005C002DD4980031D4D9002DD41A0131D449
:1003C0005C012DD4D80137D419021DD45A02E7D4C8
:1003D0009C022DD4D80229D4190317D45A0323D44C
:1003E0009C0331D4D8032DD4190429D45A0425D41C
:1003F0009C041FD41807CDD51A20C6E7990405D44C
:100400005A04CDD41B04C5D50F20BEE71320BCE78A
:100410000920BAE71C20B8E70B20B6E70A20B4E7AA
:100420000D20B2E70C20B0E71420AEE71220ACE7B5
:100430001120AAE71920A8E70E20A6E71820A4E7B4
:100440001720A2E71620A0E715209EE7002C014008
:100450001020002008E0FFFDF8B5154DEB6A93B1C0
:10046000696B0129044614D0124BDA6A22F00802A3
:10047000DA6240F2FF5100229963EA62236823F0B6
:1004800001032360F8BD0B4AD36B43F48073D3633D
:10049000F8BD084E40F2FF570023B763B36040F247
:1004A0004C43F3600C20FFF739FFB763DCE700BF74
:1004B00010200020002C0140B14BD3E9011270B58F
:1004C0008C0F83F83840C1F3836483F83940C1F35B
:1004D000016483F83A40100EC1F3074483F83B40AF
:1004E0000001C1F30724C9B283F83C4083F83D10F2
:1004F000D887D98F93F89050C2F3035089B2014343
:10050000C2F30344D987C2F3C03083F84040C2F33A
:100510004031C2F3803483F84100012D83F842401A
:100520004FF0000083F84310C2F3003183F8441009
:10053000C2F3072CD96883F8450040F2D680022D1B
:1005400000F0B0802A204FEA4C0C0CF07E0C83F8AF
:10055000514083F852C093F85240C1F3C012144383
:100560001A6983F8524001F07F01D40F83F85310C9
:1005700083F85440910DC2F3417483F8554001F063
:100580000C01C2F3826483F8564083F8571093F845
:100590005710C2F381542143C2F3405583F85710DA
:1005A00083F85850002583F85950C2F3004583F86A
:1005B0005A50C2F3C03583F85B50C2F3803583F8DC
:1005C0005C50C2F3403583F85D505C69C2F300357E
:1005D00083F85E50C2F3812583F85F50C4F307416E
:1005E000C2F30125C2F3460283F860504FF0010CBC
:1005F00083F861200902220E83F862C083F8642028
:10060000A3F86610B3F86610C4F3072289B2114349
:100610002406A3F8661099699C669A6E0C0E42EA4D
:1006200004429A669C6E0A0A02F47F4222439A664A
:100630009D6EDA69C1F307242C43C9B29C6683F826
:100640006C10110E83F86D10110C090619671C6FE0
:10065000110201F47F0121431967196F120292B24E
:100660000A431A67196F1A6A41EA1261196793F807
:100670007410C2F30354214383F87410110A01F477
:100680007061A3F87610B3F87610C2F3072489B22C
:100690002143C2F34602A3F8761083F8782083F84A
:1006A00079C070BD120402F47C129A649A6C0C0E2C
:1006B00042EA04229A649C6CC1F3074222439A6482
:1006C0009A6C013240F10004A40244EA925492026E
:1006D000C3F880204FF40072C3F88440C1F3072CA4
:1006E000C3F88820C1F380342DE74FEA8C2C0CF43A
:1006F00040649C649C6C920002F47F7222439A6472
:100700009D6CC1F3C26445EA91759D6483F84C40C9
:10071000C1F3026483F84D40CA0BC1F3425483F81D
:100720004E4002F00602C1F3824483F84F4083F842
:10073000502093F85020C1F3C034224383F8502056
:100740009D6C93F8504093F840600234012202FA05
:1007500006F6A2404FEAE27EA2FB062406FB0E4408
:1007600005F1010EA2FB0E2E05FB04447444C3E9FF
:100770002024C1F3072CC3F88860C1F38034E2E67B
:100780001020002038B50D4B0D4C1A6840F2FF5573
:1007900040F24D43A5630121A2600D20E360FFF705
:1007A000BDFDA56340B96069C0F34320A0F104001A
:1007B000B0FA80F0400938BD002038BD102000207C
:1007C000002C01402F4B1A68910102D59A6D5207F7
:1007D0004BD42C4B1A68500202D5DA6E11063CD469
:1007E000284B1A68D20102D59A6D90072DD4254B5B
:1007F0001A68510102D59A6D120717D4214B1A6855
:10080000120112D59A6DD0060FD59A6D510334D4CA
:100810009A6DD20503D49A6D22F010029A65194B95
:1008200019484FF000629A6016E670479A6D5003BF
:1008300007D49A6DD10503D49A6D22F008029A6507
:10084000104B4FF080629A60D8E79A6D4FF080713C
:1008500022F002029A659960C9E7DA6E4FF48001CE
:1008600022F08002DA669960BAE79A6D4FF0007163
:1008700022F004029A659960ABE74FF000629A603B
:10088000704700BF0064024058640240384B5A6809
:10089000110303D5D3F8A02052075BD4344B5A6818
:1008A000D00303D5D3F8B420110649D4304B5A688D
:1008B000520303D5D3F8A020900737D42C4B5A68A5
:1008C000D10203D5D3F8A02012071CD4284B5A68B4
:1008D000920217D5D3F8A020D00613D5D3F8A020C4
:1008E000510341D4D3F8A020D20505D4D3F8A020D9
:1008F00022F01002C3F8A0201D4B1E484FF4001236
:10090000DA60A9E57047D3F8A02050030AD4D3F8E1
:10091000A020D10505D4D3F8A02022F00802C3F806
:10092000A020134B4FF48012DA60CFE7D3F8A02059
:100930004FF4802122F00202C3F8A020D960BDE765
:10094000D3F8B4204FF4803122F08002C3F8B420F1
:10095000D960ABE7D3F8A0204FF4002122F00402C5
:10096000C3F8A020D96099E74FF40012DA6070470D
:1009700000640240A064024082B00922274B8DF837
:100980000720DA68D00319D4DA68D10640D4DA68CF
:10099000D20541D4DA6812F0E00F3BD1DB6813F0E6
:1009A000020F0CBF092308238DF807309DF807308C
:1009B000012B0AD09DF8070002B0704701238DF883
:1009C00007309DF80730012BF4D1144A12E0D368A8
:1009D000DB0519D4D36813F0E00F17D1D36813F0F7
:1009E000020F0CBF092308238DF807309DF807304C
:1009F000012BDFD1D168C8034FF00103F4D4D368D1
:100A0000D906E4D50623EFE70223EDE70723EBE75A
:100A10000623D4E70723D2E70223D0E7003C0240B5
:100A2000704700BF704700BF704700BF012070478C
:100A3000034BD3E92503C01AC0F30A00704700BF77
:100A400010200020064AD2E925139942FDD0D11882
:100A50000133C3F30A0391F89C00C2F89830704741
:100A600010200020064BD3F89C0800B97047D3F83B
:100A70009C08A0F10500B0FA80F04009704700BF63
:100A800010200020012380F849307047044BD3E93F
:100A90002503C01AC0F30A00C0F50060704700BF0C
:100AA0001020002010B5D0F8E83504461B6998479F
:100AB000032384F81231002010BD00BF08B50422C2
:100AC00090F81211D0F8E83580F8131180F812214F
:100AD000DB689847002008BD08B5D0F8E435DB692D
:100AE00003B19847002008BD08B5D0F8E4351B6A6B
:100AF0009847002008BD00BF08B5D0F8E4355B6A10
:100B00009847002008BD00BF70B5037805460E4623
:100B10001446DBB101307EF0EBF8431CDBB201334D
:100B20005B00DAB223800323327073702C7864B1D7
:100B30002846022300215A1CD2B2F454B15410F8B2
:100B4000014F0233DBB2002CF5D170BD02221346F7
:100B5000E8E700BF10B5074C2068FF2808D0064919
:100B6000D1F8A02801F6A40100F082F8FF23236049
:100B7000002010BD00000020102000204323014869
:100B80000B80704704000020122301480B8070473F
:100B900048000020042301480B8070475C000020BF
:100BA00010B5044C04480A462146FFF7ADFF204625
:100BB00010BD00BFBC280020A415090810B5044CC6
:100BC00004480A462146FFF79FFF204610BD00BF9C
:100BD000BC280020B815090810B5044C04480A4682
:100BE0002146FFF791FF204610BD00BFBC28002022
:100BF000C015090810B5044C04480A462146FFF701
:100C000083FF204610BD00BFBC280020CC1509087A
:100C100010B5044C04480A462146FFF775FF2046EC
:100C200010BD00BFBC280020D8150908704700BFC0
:100C3000704700BF704700BF704700BF704700BFDC
:100C4000704700BF704700BF044B00200522C3F867
:100C50009C28C3F8AC09C3F8B009704710200020E5
:100C6000024B0020C3F89C08704700BF10200020F2
:100C7000212838B50C4625D0222816D0202812D19C
:100C800089B1072A0FD1174DD5F8B03913B10968CA
:100C9000002098472168A288A379C5F8B419A5F85F
:100CA000B82985F8BA39002038BD0029FBD0022ABE
:100CB000F9D10C4BD3F8AC39002BF4D009880020C3
:100CC0009847F0E70029EED0072AECD1054BD3F87E
:100CD000B419B3F8B82993F8BA392160A280A37186
:100CE000E1E700BF1020002010B4114CD4E92532F8
:100CF0009A1AC2F30A020A44B2F5006F14D879B105
:100D000001444A1E013810F801CFE118904203F166
:100D1000010381F89CC0C3F30A03F4D1C4F89430F2
:100D200000205DF8044B704702205DF8044B7047CB
:100D300010200020034B93F8E009003818BF012071
:100D4000704700BF1020002070B5124D124C29686A
:100D500040F2FF5640F24D430022A6630D20A160F1
:100D6000C5F8DC290121E360FFF7D8FAA66320B9B2
:100D70006369C3F34323042B08D0D5F8143AC5F8AC
:100D8000D039092385F8E039002070BD85F8E039B5
:100D9000022070BD10200020002C014070B50E4DC7
:100DA00095F8E039042B04460E460BD0082B07D1EA
:100DB000D5F8D83983420CD0FFF7C6FF022801D0FE
:100DC000012070BD082385F8E039C5F8DC69C5F855
:100DD000D849022070BD00BF10200020034B93F8BB
:100DE000E009032894BF0020012070471020002054
:100DF00000487047F429002030B4184B00209C7B39
:100E000014B11D688D4206D00130082803F110038B
:100E1000F5D130BC7047D2B1114B03EB40218A426F
:100E200011D0104B93F8B42112B9012283F8B421E8
:100E30000D4B01225A7000F5817003EB0013012263
:100E40009A7130BC7047022CEBD1183BF3E7064B8C
:100E500000F5817003EB00139A71DAE7F05C002073
:100E6000F04C0020D85C0020D84C002030B41D4C41
:100E7000002384F8A03004F1180004E00133082BAB
:100E800000F110001ED005688D42F7D190F80EC019
:100E9000BCF1030FF2D1BAB1134901EB43208242F6
:100EA00009D094F8B42112B9012284F8B4210F4971
:100EB00001224A7000E0183903F5817301EB031138
:100EC00001238B7130BC70470849D4F89C2003F58E
:100ED000817301EB0313013204219971C4F89C2042
:100EE000F0E700BFD85C0020F04C0020D84C002078
:100EF000A8B183681BB10E4B07229A7070470C4A49
:100F00001178D36003294FF0040014BF4FF48071AF
:100F10008021C2E901111361137590707047044A72
:100F200002F580510123537081F8B431704700BF3E
:100F3000D84C002010B5812104467DF083FB20466B
:100F400001217DF07FFB204682217DF07BFBFFF7B6
:100F500087FE002010BD00BF034610B4D9691A698E
:100F6000002040F20114A3F844410860D1699C6D4F
:100F700021F002014FF0010CD161A3F89CC3206065
:100F8000D369044923F4003381F8180A5DF8044B4F
:100F9000D361704710200020202301480B80704748
:100FA00060000020122301480B8070478000002061
:100FB000042301480B807047940000200A4608B5BE
:100FC000054920B90548FFF79FFD034808BD0448BF
:100FD000FFF79AFD004808BD2C2A0020E8150908F3
:100FE0000016090810B5044C04480A462146FFF7CC
:100FF0008BFD204610BD00BF2C2A002018160908C2
:101000001C48D0F8E837D0F8EC2710B59B184FF003
:101010001A040C8001D1184810BD174AD0F8EA070D
:1010200002F1100411464FF0000E4FEA137CB3F1A9
:10103000204F34BF0CF1300C0CF1370C81F802C09A
:1010400081F803E002318C424FEA0313EDD102F143
:1010500008040021030FB0F1204F34BF3033373381
:101060009374D174023294424FEA0010F2D10248D4
:1010700010BD00BF00F0FF1F9800002010B5044C09
:1010800004480A462146FFF73FFD204610BD00BF39
:101090002C2A00202C16090810B5044C04480A46D6
:1010A0002146FFF731FD204610BD00BF2C2A00204D
:1010B00038160908A14A536823F4FD4323F07F033F
:1010C0002DE9F04143F0760353605368032123F484
:1010D0008073536082B011600FF056FB04460D46DA
:1010E0000FF052FB001B61EB0501B0F57A7F71F147
:1010F0000001F5D30FF048FB04460D460FF044FB0A
:10110000001B61EB0501B0F57A7F71F10001F5D3A9
:101110008A4C6368002040F2FF5543F480734FF41B
:10112000806263604FF0FF31A563A060E260FFF76B
:10113000F5F8A563074618B1012002B0BDE8F081BB
:101140004FF4D5724FF48963A5630721A26008208C
:10115000E360FFF7E3F8A56328B9794B012283F830
:1011600090204FF08047754C40F2FF55002240F22E
:101170007743A5630121A2603720E360FFF7CEF833
:10118000A5630028D8D147F000470646804647F4BB
:10119000801701E09642CFD040F27743A56301214A
:1011A000C4F808803720E360FFF7B8F8034640F240
:1011B000694203212920A563002BBDD1A563A76047
:1011C000E260FFF7ABF801364FF6FF72A563002827
:1011D000B2D16369002BDDDA4FF6FF729642ABD0D5
:1011E0005D0000F1B38023689807A5D0544D95F8B1
:1011F0009060042E40F0B280FFF75EF900289BD18A
:101200004E4C2B6840F2FF57A763A36040F2474360
:10121000E36001210720FFF781F8A763636823F4E7
:10122000FD4323F07F036360002885D1022E83D81D
:10123000636913F000737FF47FAF009308264FF4C7
:101240008A63A7630121A6601020E360FFF766F8B8
:10125000A76300287FF470AF2B68A763A36040F2F8
:101260007743E36001213720FFF758F8A763002890
:101270007FF462AF334A6262A662E26A42F03302EE
:10128000E26240F27342A7630121A060E260332072
:10129000FFF744F8A76300287FF44EAF6B4640F297
:1012A0002A4206E0616B890244BFD4F8801043F8FB
:1012B000041B616B1142F5D0636B1B073FF53CAF1C
:1012C000636B9F073FF538AF636B9E063FF534AF06
:1012D000636B98023FF530AF009B1BBA59037FF553
:1012E0002BAF2A6840F2774340F2FF55A5630121F6
:1012F000A2603720E360FFF711F8A56300287FF4B0
:101300001BAF022240F24643A5630121A2600620E2
:10131000E360FFF703F8A56300287FF40DAF63686F
:101320001A0509D4054A084953680B4043F4006381
:10133000536053681B05F7D50020FEE6002C0140E2
:101340001020002000E1F5050081FFFF274D022657
:1013500085F8906023689C073FF4EEAE244C40F281
:10136000FF570023A7630221A36040F2C243E3605A
:101370000846FEF7D3FFA76300287FF4DDAE63695C
:101380006B61A369AB61E369EB61236A2B62022E97
:101390001BD9062E19D0164C2B6840F2FF57A763B5
:1013A000A36040F2C943E36002210920FEF7B6FFC3
:1013B000A76300287FF4C0AE63696B60A369AB606C
:1013C000E369EB60236A2B6116E7094C40F2FF5793
:1013D0000023A763A36040F24343E3600621032098
:1013E000FEF79CFFA7630028D5D0A5E610200020BB
:1013F000002C014010B5104CD4F80C3A43B11968D8
:101400009A880B691A4203D1002384F8E03910BD91
:10141000FFF750FE0028F7D194F8D4390133DBB23E
:10142000072B84F8D439EFD8D4F8143AC4F8D0395B
:10143000012384F8E03910BD1020002070B5A14CC4
:10144000D4F8100A002800F0138194F8E0596B1EBC
:10145000082B0ED8DFE803F0C6057F0D61CA340DF6
:101460001500FFF78FF9002840F0058194F8E05946
:101470006B1EDBB2022B40F2D380042D47D101203A
:1014800070BD914D226840F2FF5640F24D43AE636D
:101490000121AA600D20EB60FEF740FFAE6328B982
:1014A0006B69C3F34323042B00F0C780D4F8D03911
:1014B000D4F8142AFA339342D8D2FFF79BFFC4E73B
:1014C000814D226840F2FF5640F24D43AE63012148
:1014D000AA600D20EB60FEF721FFAE630028E5D186
:1014E0006B69C3F34323042BE0D1D4F8DC3984F8CF
:1014F000D409012B40F2DF80D4F8D8290825013B1C
:101500000132C4F8DC39C4F8D82984F8E059A5F1CF
:101510000800B0FA80F0400970BDE66A002E40F085
:101520009080FFF72FF9002800F09380D4F8C85975
:1015300084F8D469042384F8E039002D9FD0D4F8CE
:10154000CC39D4F8BC29D4F8C0193046A84794F84F
:10155000E0596B1E8DE7FEF7AFFF002860D194F8CD
:101560006420B4F86630A4F8E839A16EA36EC4F81C
:10157000DC09090E04201B0C84F8EA2984F8E00930
:10158000A26E84F8EB1984F8EC39A16E94F86C0023
:1015900094F86D3084F8EE19120A1B0984F8ED29CD
:1015A00084F8EF0994F86D2084F8F439216FB4F8C9
:1015B0007600B4F87630C4F8F01902F00F02C3F3E5
:1015C0000B1384F8F52943EA1023B4F8762003F0CE
:1015D0000F0303F5FA6302F00F02A4F8F63984F85A
:1015E000F82932E7022384F8E0392EE7236B002B39
:1015F0008DD1D4F8C869D4F8143AC4F8D039072585
:1016000084F8E059002E82D0D4F8CC39D4F8BC2923
:10161000D4F8C0190120B04794F8E0596B1E28E7B0
:10162000D4F8143AD4F8D0299B1AC82B7FF66FAFA0
:10163000FFF7E0FE94F8E0591FE7042384F8E0394F
:101640001DE7D4F8D039D4F8142A64339342BFF498
:101650005EAFFFF7CFFED4F8C859002D3FF4F5AECA
:101660000022D4F8CC39D4F8C0191046A847ECE6CB
:1016700084F8E00970BDFEF71FFF00287FF4F6AE86
:1016800094F89030002BA3F10203B3FA83F308BF60
:1016900001255B0984F8D65984F8D739FEF70CFF89
:1016A00000287FF40AAFD4F88020C4F8E42903238B
:1016B00084F8E039C9E6C0D1FFF746FB94F8E05959
:1016C0006B1ED6E610200020002C01402DE9F041D1
:1016D0001F4E80460B4696F81B2B002AFBD19BB36E
:1016E00043445F1E08F1FF38D6F81C3BD6F8202B88
:1016F0000133C3F30A039A4216D10FF045F80446AA
:101700000D460FF041F8001B61EB0501B0F57A7F43
:1017100071F10001F5D3D6F81C3BD6F8202B01332C
:10172000C3F30A039342E8D0D6F81C2BD6F81C3B2F
:1017300018F8011F32440133C3F30A03B84582F895
:10174000241BC6F81C3BCFD10020BDE8F08100BFB0
:101750001020002010B50A4CD4F89C3803B910BDF5
:10176000D4F89C38052BFAD1002A0846D4F8143A4C
:101770001146F4DDFFF7AAFFD4F8143A10BD00BFFC
:101780001020002090F84820531C0244DBB280F85F
:10179000483082F8341090F8492052B1132B0CD9FC
:1017A000002280F8482010B50B4CD4F89C282AB9A8
:1017B00010BD80F84820002BF5D17047D4F89C2844
:1017C000052AF5D119463430D4F8143AFFF77EFFD4
:1017D000D4F8143A10BD00BF1020002090F8481033
:1017E0000023A0F8483001B9704710B5084CD4F870
:1017F0009C381BB1D4F89C38052B00D010BD343078
:10180000D4F8143AFFF762FFD4F8143A10BD00BFC1
:10181000102000202DE9F047534E1F4606EB8003B1
:101820009C68002C00F09B8004F13E03A36104F54A
:101830009F73E3614FF48073C4E90433283623684F
:1018400066600546E16094F83D00A36391460BF0A5
:1018500017F8804694F8440294F83CA0261D00280E
:1018600051D194F8450250BBD4F840326BBB3A07D3
:1018700031D419F0020F49D119F0010F5AD1D4F81F
:10188000483294F9471294F847221B010029DBB231
:101890000DDB3649881880F800335009012302F027
:1018A0001F02934041F820303046BDE8F0873049B0
:1018B00002F00F02114430460B76BDE8F08775F058
:1018C000BBFED4F84032002BD1D02A4A116B0B4317
:1018D00013633A07CDD50135EDB2B8F1000F05D04D
:1018E00040F2067388F80850A8F80630FB0694F812
:1018F00046222FD417F0200F0CBF32211221404670
:101900000AF082FFBBE775F097FEAAE76B1CDBB21B
:10191000B8F1000F05D088F8083040F20653A8F857
:10192000063094F84622404602210AF06DFF19F075
:10193000010FA4D050460AF0A3FF0135EDB218B153
:1019400040F20663C380057294F8462202210AF031
:101950005BFF94E7022140460AF056FF8FE72646D8
:101960003046BDE8F08700BFC86B080800E100E022
:10197000FCEC00E0003802402DE9F047038A84893E
:10198000A4B21C4082B047D0814688464FF0004543
:1019900001F14C0701F13406B4FA84F325FA03F29D
:1019A000D24391B2A9F8101014401B3BB8F1000FBC
:1019B0005FD0042B2ED8DFE803F052483D320300FD
:1019C000D8F80C30D9F82CA033B19B6823B11FFA9A
:1019D0008AF108F104009847D8F8243033B19B68A5
:1019E00023B11FFA8AF108F11C009847D8F83C305F
:1019F00033B19B6823B11FFA8AF108F1340098478C
:101A0000D8F8543033B19B6823B11FFA8AF108F13A
:101A10004C009847002CBFD102B0BDE8F087D8F841
:101A20000C30D9F834105B6808F104009847002C9A
:101A3000B2D1F1E7D8F82430D9F838105B6808F152
:101A40001C009847002CA7D1E6E7D8F83C30D9F81D
:101A50003C105B6830469847002C9DD1DCE7D8F8F5
:101A60005430D9F840105B6838469847002C93D121
:101A7000D2E7042B07D8DFE803F01903140F0A009C
:101A8000D9F83C300193019B002C85D1C4E7D9F8EB
:101A90002C300193019BF7E7D9F834300193019B77
:101AA000F2E7D9F838300193019BEDE7D9F84030DF
:101AB0000193019BE8E700BFF8B5264C94F81B2B77
:101AC000012A034603D0022A09D00020F8BD224E85
:101AD000D6F82C528DB984F81B5B0020F8BD002588
:101AE00040F20112C0E95455C0E95655A0F844210E
:101AF00000F5A2717CF0A2FEEDE7402D20D9402731
:101B0000D4F8201B154AC3F858710A44C3E954227B
:101B100040F20112A3F844210022C3F85C2103F52E
:101B2000A27118467CF08AFED4F8203B3B44ED1BA2
:101B3000C3F30A03C4F8203BC6F82C520020F8BDBA
:101B4000AAB2402A01D02F46DAE7022284F81B2BE2
:101B5000D5E700BF1020002008310020342B0020E2
:101B600001EB810138B500EBC1010F4DB1F88C13C9
:101B700004462846FFF7B8F8E378C4F8A8530120D4
:101B800083424FF000024FF04001C4E9EC12A4F888
:101B90009C0304F56771204608BFC4F8AC537CF081
:101BA0004DFE002038BD00BF38330020F8B52A4C68
:101BB000D4F870320F2B04D05A1CC4F870220020C5
:101BC000F8BD264D95F81B3B0022C4F87022002B6F
:101BD000F5D1D5F8202BD5F81C3B9A42EFD0D5F89B
:101BE000202BD5F81C3B9A422DD8D5F81C6BD5F884
:101BF000203BF61A402E2BD8B3B2402B13BF3746EA
:101C0000402702230123D5F8202B85F81B3B144BDA
:101C1000C0F858711344C0E9543340F20113A0F8DE
:101C200044310023C0F85C3100F5A2717CF006FE5F
:101C3000D5F8203B3B44F61BC3F30A03C5F8203B11
:101C4000C4F82C62BBE7D5F8206BC6F50066D1E777
:101C500001234027D7E700BF0831002010200020D3
:101C6000342B002010B5324B93F8802293F894C2A5
:101C7000D3F87C32044613B152EA0C0231D001236E
:101C8000E06984F8463140F20112A4F84421026868
:101C90002849002AA8BFC2F380739B0301EA1241BE
:101CA00043F020030B4363F31F42BCF1020F0260B9
:101CB00000D010BDE278204BC4F8A8331F200021CB
:101CC000C4E9EC01012A4FF00101A4F89C1308BFFC
:101CD000C4F8AC3304F567712046BDE810407CF0D1
:101CE000ADBD01217CF074FC0122E06984F846213D
:101CF00040F20113A4F84431016800290A460CDBC4
:101D0000C1F380730B4C9B0343F0200304EA1141A1
:101D10000B4363F31F42026010BD064B03EA1143FD
:101D200043F4804343F0200363F31F42026010BD7D
:101D300008310020DFBFFFFF7C3300202DE9F04198
:101D4000B0F8CC15D0F8CE35B0F8D255B0F8D08573
:101D5000C0F84051012284B080F8112101F01F0227
:101D6000012A044600F2CC56ADF80810C1F3072E44
:101D7000CDF80A30ADF80E504FEA134C51D0022A7C
:101D80007746C9B29BB210D0002A55D1BEF1090FD7
:101D90004BD8DFE81EF08900AD004A00C8004A00B9
:101DA0005C01DF004A001301330101F060012029CA
:101DB0005FFA8CF272D0012F00F0B881032F00F08F
:101DC000A181AFBB90F81231022B00F0E381032B0D
:101DD0002BD11CF0800F40F0E98102EB820200EB76
:101DE000C20393F87623003A18BF0122C24D0223A2
:101DF0004FF48071C4E94E3384F81131C4F83031A6
:101E0000A4F81C1105F529730021C4F83411C4E9A4
:101E10004A3304F58E712046C5F8A4227CF0ACFC50
:101E200006E090F81231032B0ED020467CF098FB90
:101E3000002004B0BDE8F08101F080017CF0C8FB17
:101E4000002004B0BDE8F0815FFA8CFCBCF1010F0A
:101E5000EBD8D0F8E43502A99B689847BDF80E305E
:101E6000002BE5D1C4E94A33C4E94C3304214FF4D3
:101E7000807284F81111A4F81C2104F58E7120469B
:101E80007CF07AFC636D9D4A1A61E278012ACFD119
:101E90005E614FF0802219681A60C9E7D0F8E43516
:101EA00002A99B689847C3E790F81231023B012BC7
:101EB000BBD8914BD0F818210021C3F89C1212B165
:101EC0000222C3F89C228E4A02234FF48070002124
:101ED000C4E94C31A4F81C01C4E94E33C4E94A22D8
:101EE00084F8113104F58E7120467CF045FC9FE7A3
:101EF00090F81221023A012A97D8012B98D1D0F8F4
:101F0000E43500259B68C0F8185102A998470422BF
:101F10004FF48073C4E94A55C4E94C5584F8112143
:101F2000A4F81C31A9E7012B00F03B81022B7FF4C0
:101F30007FAF5FFA8CF3002B7FF47AAF03694FEA2F
:101F40001C22023A5B68032A00F2BD81DFE802F03E
:101F5000B6CED2D01E0A022EADF8065000F08A810D
:101F6000032E00F04E81012E7FF45FAFD0F8EC35E8
:101F700080781B680DF106019847BDF80630002BEC
:101F80003FF456AFBDF80E20002A3FF451AF934204
:101F900028BF13464FF480720221A4F81C210022AE
:101FA000C4E94A0084F81111C4E94E33C4E94C3243
:101FB00004F58E7120467CF0DFFB39E7012D7FF4BC
:101FC00034AF90F81231022B00F00881032B7FF41C
:101FD0002CAF4FF4807200F588730221A0F81C2109
:101FE000002280F81111C0E94E55C0E94A33C0E91A
:101FF0004C5200F58E717CF0BFFB19E7DDB23E4F0D
:10200000012D87F895523FF610AF90F81231022B50
:1020100000F0D880032B7FF408AF002D00F035814D
:1020200090F81011012910D0D0F8E4355B6898477A
:1020300097F89512D4F8E43584F810111B682046FF
:102040009847D4F8E8359B68984700230AE758EA90
:1020500005027FF4EAAE90F8121103293FF4E5AED1
:1020600003F07F0580F814510069114663F30A11EB
:10207000036819430423016084F811314FF480731D
:10208000C4E94A22C4E94C22A4F81C3104F58E713B
:1020900020467CF071FB636D184A1A61E278012AD0
:1020A00006D0002D00F0FC80022384F81231BFE638
:1020B0005E614FF0802219681A60F2E702210E4833
:1020C00061F306130022C0F8A0320423C4E94A22B7
:1020D000C4E94C2284F8113101224FF4807304F5D5
:1020E0008E7184F81621A4F81C31C8E60321E6E7B6
:1020F0000521E4E70421E2E7083100201800086028
:10210000A433002090F81211022943D003297FF450
:102110008CAE23B9510602D011467CF059FAD4F89E
:10212000E4359B6802A9204698478EE790F8121183
:1021300002292FD003297FF478AE002B7FF478AEEC
:1021400012F07F0181D01CF0800F40F0AD8002EBD7
:10215000820100EBC10181F8763381F875332823C1
:1021600081F8742303FB020300EB820193F87723C9
:10217000496D0B68023A012A23F400138CBFC3F3A4
:102180000072012262F31C73D4F8E4250B6093689B
:1021900002A9C8E753063FF44BAE11467CF018FA8B
:1021A00046E6D0F8E425C0F81831F0E702F07F02E7
:1021B00002EB820200EBC20393F81E21003A18BF23
:1021C000012213E6002D3FF4A2AE01210322D0F834
:1021D000E43580F8101180F812212FE73B4A80F88F
:1021E00011314FF480710023A0F81C11C0E94E5545
:1021F000C0E94A22C0E94C5300F58E717CF0BCFA6C
:1022000016E6DBB2052B3FF610AEDFE803F02B231A
:102210001B130B03D0F8EC3580789B690DF1060198
:102220009847AAE6D0F8EC3580785B690DF1060195
:102230009847A2E6D0F8EC3580781B690DF10601CD
:1022400098479AE6D0F8EC358078DB680DF1060106
:10225000984792E6D0F8EC3580789B680DF106013E
:1022600098478AE6D0F8EC3580785B680DF1060176
:10227000984782E6D0F8E43580789B6A0DF1060134
:1022800098474670C4F8F00577E60222D0F8E435A6
:1022900080F8122180F810515B682946984736E68D
:1022A000012384F81231C3E5282202FB010080F8E3
:1022B0001C1104EB810180F81E3180F81DE190F8BB
:1022C0001F21896955E70121F9E600BFA0330020ED
:1022D00010B5044629B990F81121032A0DD0002029
:1022E00010BDD0F8E4359B69002BF8D090F812218E
:1022F000032AF4D19847002010BDD0F890230B4654
:10230000D0F87C138A4219D9521AC0F8902394F855
:1023100003C0D0F880038A4228BF0A46BCF1010FEF
:1023200092B234D0C4E9E22304F55D71C4F88003AD
:10233000A4F8743320467CF01FFAD0E7D0F8E435D7
:102340001B691BB190F81221032A1ED000234FF401
:1023500080720421C4E94A33C4E94C3384F8111172
:10236000A4F81C2104F58E7120467CF005FA636DFB
:102370000D4A1A61E278012AB1D104F2CC545C61B1
:102380004FF0802219681A60A9E79847DEE70844F1
:10239000C4E9E22304F55D71C4F88003A4F8743342
:1023A000C4F88403C6E700BF1800086038B50446C7
:1023B00049B990F81131022B11D094F81631012B44
:1023C00039D0002038BDD0F8E4355B69002BF8D057
:1023D00090F81221032AF4D19847002038BDD0F894
:1023E0003831D0F8242193422FD990F803C09B1A9A
:1023F000BCF1010F0D46C0F83831D0F828116ED06D
:102400009BB2C0F830314FF48073C0E94A11C0F874
:10241000345100F58E71A0F81C317CF0ADF9C4E99F
:10242000E255C4F8805304F55D71A4F87453204656
:102430007CF0A2F9C1E73F4B2269D3F8A0125160AA
:10244000002384F81631002038BDD0F83C31B3FBAE
:10245000F2F502FB15350DBB9A421FD8D0F840218A
:1024600093421BD24FF48073A0F81C3100F58E719B
:10247000C0E94A55C0E94C557CF07EF9E378C4F8D0
:102480004051012BC4E9E255C4F88053A4F87453B9
:1024900008BFC4F8845304F55D71C8E7D4F8E43587
:1024A000DB681BB194F81221032A15D0E2780023CF
:1024B0000521012A84F81111C4E9E233C4F88033FC
:1024C000A4F8743304F55D7124D020467CF054F9EF
:1024D000636D194A1A6170E720469847E6E79BB298
:1024E0001144C0F830314FF48073C0E94A11C0F88C
:1024F000345100F58E71A0F81C317CF03DF9C4E92F
:10250000E255C4F8805304F55D71A4F87453C4F81F
:1025100084538CE7C4F8843320467CF02DF9636D36
:102520000548186104F2CC525A614FF080211A68B4
:10253000196042E7083100201800086070B50B7878
:1025400013F060020D46044624D0202A04D0204611
:102550007CF006F8022070BDCA8848781AB31B06C2
:1025600040D5324E3146FEF783FBEB884FF4807244
:102570000221A4F81C21002284F81111C4E94E3371
:10258000C4E94A66C4E94C3204F58E7120467CF0F9
:10259000F3F806E04B780A2B10D00B2B08D0062B53
:1025A000D5D0002070BD02221144FEF761FBF8E790
:1025B0008B78C3BB1E4AC2F8A832F2E7022180F82A
:1025C00011114FF48071A0F81C111A490123C0E9C0
:1025D0004A11C0E94E33C0E94C3200F58E717CF0EF
:1025E000CBF8DEE71449154B0860E078C3F8A02863
:1025F000002103F6A40301284FF00305C4F88C134F
:10260000A4F87413C4E9E42284F81151C4F88823AF
:10261000C4F8803304F55D7108BFC4F884332046E4
:102620007CF0AAF8BDE77BF09BFFBAE7B428002056
:1026300008310020B03300200000002010200020CE
:10264000002310B51946044640227CF02BF8802167
:102650002046002340227CF025F8D4F8E835A07805
:10266000012284F812215B689847002010BD00BF4A
:1026700010B502230446402281217CF013F8204645
:102680000223402201217CF00DF82046032308227A
:1026900082217CF007F8104B0222A3F84C20FEF7B1
:1026A000D3FAE2780D4BC4F8A8334021C4F8B01334
:1026B000012A4FF000004FF00101C4F8B403A4F860
:1026C0009C13204604F5677108BFC4F8AC337CF056
:1026D000B5F8002010BD00BF0000002038330020F6
:1026E00030B5812183B004467BF0ACFF0121204648
:1026F0007BF0A8FF2A4900250223402281F8185ABE
:10270000204681217BF0CEFF01210223402220467A
:102710007BF0C8FF234BD3F8AC2283F894521268A5
:10272000284690470095009AE1681F4B42F010023E
:102730000092009A0A610A690092013B02D0009A55
:10274000D006F8D400230193019B43F020030193AA
:10275000019A154B012060F38A120192019A0A61D5
:102760000A690192013B02D0019A9206F8D4E278FC
:102770000E4BC4F8A8331F200021C4E9EC01012A44
:102780004FF00101A4F89C13204604F5677108BFBF
:10279000C4F8AC337CF052F8002003B030BD00BF69
:1027A0001020002008310020410D03007C33002060
:1027B0002DE9F843444F8046894615461C4697F854
:1027C000E01904290CD0082907D1D7F8D839434596
:1027D00006D0FEF7B9FA0228F1D00120BDE8F8834F
:1027E000012387F8C4393B6397F89030C7F8CC4988
:1027F0000622022B354CC7F8C089C7F8C859C7F85C
:10280000BC9987F8E02918BF4FEA48280A2640F209
:10281000FF554FF48B63A5630121C4F8088018208D
:10282000E360FDF77BFD03464FF0000C40F277427A
:1028300001213720A5631BB3A563C4F808C0E2607B
:10284000FDF76CFD731EA563D0B113F0FF06E0D158
:1028500097F8D5393E63022B26D8013387F8D5394E
:102860000DF092FF04460D460DF08EFF001B61EB4C
:102870000501B0F57A7F71F10001F5D30120ADE7D4
:102880000121484674F050FE104B114959624FF433
:1028900000729A62DA6A002042F09102DA6287F8E6
:1028A000D509B862BDE8F88387F8D569FEF7A2FDBF
:1028B000D7F8C84934B1D7F8CC39D7F8C01932465F
:1028C0000120A0470320EDE710200020002C01404C
:1028D00000E1F5052DE9F04F4B4E994696F8E039A9
:1028E00083B0042B80460191924609D0082B03D077
:1028F000002003B0BDE8F08FFEF726FA0228F7D1DA
:1029000096F890300122022BF2627BD04FEA482BDE
:102910003E4C0198002174F007FE4FF400723C4BCE
:102920006362A262E36A40F2FF5743F09303E362FB
:10293000A763A2604FF48A62E26001211020FDF7D4
:10294000EDFC0A25A76340F25142A7630121C4F8B8
:1029500008B01120E260FDF7E1FC02464FF0000EE6
:1029600040F2774301213720A7639AB3A763C4F8E5
:1029700008E0E360FDF7D2FC013DA76350B315F01A
:10298000FF05E0D196F8D539F562022BB06211D877
:10299000013386F8D5390DF0F7FE04460D460DF0EB
:1029A000F3FE001B61EB0501B0F57A7F71F10001C8
:1029B000F5D39DE786F8D559FEF71CFDD6F8C84932
:1029C000002C95D0D6F8CC39D6F8C0192A4628461E
:1029D000A0478DE7019BC6F8BC39052386F8E0398E
:1029E0000023B362D6F8142AC6F8C0890120C6F8BD
:1029F000C8A9C6F8CC99C6F8D02986F8D53903B04D
:102A0000BDE8F08FC34683E710200020002C014072
:102A100000E1F5051049114BD1F8882042F470020D
:102A200010B4C1F888201A680D4C002042F0010251
:102A30001A6098601A6822F0847222F480321A6058
:102A40005C601A68074C22F480221A60D8608C609F
:102A50005DF8044B704700BF00ED00E00038024015
:102A60001030002400000008704700BF2DE9F84333
:102A700045697DB90768C7F30D0804460E46B8F1ED
:102A8000000F0AD0D6F80080FDF776FF09283BD06A
:102A90006FF001052846BDE8F883514B9F422AD3C9
:102AA00003F580439F4224D303F580439F427FD3A5
:102AB0004C4B9F427FD903F580339F427ED903F56B
:102AC00000339F427DD903F500339F427CD903F543
:102AD00000339F4269D903F500339F4277D903F54C
:102AE00080239F4276D9B7F1016F76D305200DF090
:102AF000A7FE4FF00808FDF73FFF092821D04FF04F
:102B0000FF352846BDE8F883374E336923F4407318
:102B10003361336943F400733361336943F0010374
:102B20003361C7F80080FDF727FF3369092823F0D8
:102B300001033361ACD12368043323602846BDE828
:102B4000F883DFF8A490D9F8103023F44073C9F863
:102B50001030D9F8103043F40073C9F81030D9F8A8
:102B6000103023F0F803C9F81030D9F8103043EAD8
:102B7000080343F00203C9F81030D9F8103043F4C9
:102B80008033C9F81030FDF7F7FED9F8103023F084
:102B90000203C9F81030D9F81030092823F0F803DF
:102BA000C9F810303FF46EAFA9E74FF03808A2E73C
:102BB0004FF010089FE74FF018089CE74FF02008EF
:102BC00099E74FF0280896E74FF0300893E74FF069
:102BD000400890E74FF048088DE74FF058088AE723
:102BE00000400008FFFF0008003C02400148FDF7DC
:102BF0000FBB00BFB80000200148FDF709BB00BFB4
:102C0000040300200148FDF703BB00BF500500206E
:102C10000148FDF7FDBA00BF9C0700202DE9F041F7
:102C20000268214D0746002455F834309A4209D0F5
:102C300001340E2CF8D11D4A0021052005F070FC4E
:102C4000002013E01A4B03EB8408D8F8B0627EB181
:102C5000797901EB410306EBC30300221820C3E995
:102C6000032200FB01609F601A750430BDE8F0810B
:102C700007216C2005F0DAFC0146C8F8B00268B103
:102C800031466C2282F072FED8F8B06205EBC405C2
:102C9000C6E90056F6617663F664D9E7054A052071
:102CA00005F03EFCCCE700BF246C08084816090874
:102CB0000831002070160908704700BF38B5D0E908
:102CC000004007EE902A0068324A334B2468D3F85C
:102CD000E4392468013990428DB210D002F5806247
:102CE00090420CD002F57052904208D002F58062FA
:102CF000904204D002F58062904218BF5B0807EE54
:102D0000103AF8EE677AB8EE477ADFED246A87EE7C
:102D1000270A30EE260A7DF08BFD1E492388421ECD
:102D20008C4292B29BB21AD01D498C4217D0B4F19A
:102D3000804F1FD0A1F580318C421BD001F58061FE
:102D40008C4217D001F580618C4213D015498C421A
:102D500019D123800123E5622285A38238BD23F4A3
:102D60005C739BB223800023E562228523860123C6
:102D7000A38238BD23F45C739BB223800123E562F8
:102D80002285A38238BD08498C42E2D023F44073E7
:102D90009BB2DEE700000140000000200AD7233C80
:102DA00000040140001000400014004070B542686B
:102DB000937903F0020E13F004033AD175469C4652
:102DC0009E464FF4807001235479032C30D8DFE8FD
:102DD00004F08E6202361468704E228C22F48072E7
:102DE0001204120C2284228C22F4007212042B434F
:102DF000120CA58842EA0322A38B23F073031B0461
:102E00001B0CB442ADB243F0600300F09B8006F5AA
:102E10008066B44200F09680A580A383E16322849B
:102E2000A38B23F008031B041B0C43F00803A383AC
:102E300070BD002005464FF0040C0346C4E712683D
:102E4000564E148C24F480542404240C1484148CC2
:102E500024F4005424042B43240C958844EA0334BE
:102E6000938B23F4E6431B041B0CB242ADB243F434
:102E7000C04375D006F58066B24271D095809383C9
:102E800011641484938B23F400631B041B0C43F420
:102E90000063938370BD1468404E228C22F01002B0
:102EA0001204120C2284228C22F0200212042B43E2
:102EB000120CA58842EA0312238B23F4E6431B0479
:102EC0001B0CB442ADB243F4C04359D006F5806642
:102ED000B44255D0A5802383A1632284238B23F49D
:102EE00000631B041B0C43F40063238370BD126852
:102EF000148C24F001042404240C1484148C96886B
:102F000024F0020424042B43240C1C43138B234D74
:102F100023F073031B041B0CAA42B6B243F06003F8
:102F200023D005F58065AA421FD096801383516394
:102F30001484138B23F008031B041B0C43F00803B9
:102F4000138370BD22F4006242EA0E2222F48062F2
:102F500092B225F4405542EA0C2245EA00155BE79F
:102F600025F4804545EA801588E726F44076064337
:102F70004FF6F370204040EA0E0040EA0C04D4E71C
:102F800022F0800242EA0E1222F0400292B225F4B0
:102F9000406542EA0C1245EA80059BE700000140CB
:102FA00042685379032B0FD8DFE803F00B080502C2
:102FB00010684030704710683C30704710683830F7
:102FC000704710683430704700207047024B034848
:102FD000D3F8B012FEF7D0BC083100200000014049
:102FE00010B5064C0648D4F8B012FEF7C5FCD4F86C
:102FF000D0120448BDE81040FEF7BEBC08310020E6
:10300000000001400040014010B5064C0648D4F8CD
:10301000B012FEF7B1FCD4F8D4120448BDE8104059
:10302000FEF7AABC08310020000001400044014026
:1030300010B5064C0648D4F8B012FEF79DFCD4F843
:10304000D8120448BDE81040FEF796BC08310020B5
:103050000000014000480140034B4FF08040D3F88E
:10306000B412FEF789BC00BF08310020024B0348B0
:10307000D3F8B812FEF780BC0831002000040040ED
:10308000024B0348D3F8BC12FEF776BC083100208F
:1030900000080040024B0348D3F8C012FEF76CBC96
:1030A00008310020000C0040024B0348D3F8CC123A
:1030B000FEF762BC083100200004014010B5064C48
:1030C0000648D4F8CC12FEF757FCD4F8DC120448BA
:1030D000BDE81040FEF750BC08310020000401405C
:1030E0000018004010B5064C0648D4F8CC12FEF784
:1030F00043FCD4F8E0120448BDE81040FEF73CBCA5
:103100000831002000040140001C004010B5064CAE
:103110000648D4F8CC12FEF72FFCD4F8E412044889
:10312000BDE81040FEF728BC083100200004014033
:10313000002000400348D0F8F43913B100F6E8103D
:1031400018477047000000200348D0F8143A13B124
:1031500000F6082018477047000000200348D0F808
:10316000343A13B100F628201847704700000020B9
:103170000348D0F8543A13B100F648201847704776
:10318000000000200348D0F8743A13B100F668201C
:1031900018477047000000200348D0F8943A13B154
:1031A00000F6882018477047000000200348D0F838
:1031B000B43A13B100F6A820184770470000002069
:1031C0000348D0F8D43A13B100F6C8201847704726
:1031D000000000200348D0F8F43A13B100F6E820CC
:1031E00018477047000000200348D0F8143B13B183
:1031F00000F6083018477047000000200348D0F858
:10320000343B13B100F62830184770470000002007
:103210000348D0F8543B13B100F6483018477047C4
:10322000000000200348D0F8743B13B100F668306A
:1032300018477047000000200348D0F8943B13B1B2
:1032400000F6883018477047000000200348D0F887
:10325000B43B13B100F6A8301847704700000020B7
:103260000348D0F8D43B13B100F6C8301847704774
:103270000000002030B44568144CA542144D2C6B5E
:103280000CBF44F4001444F480042C6390F914C07F
:10329000C1601201BCF1000F8361D2B20FDB0D4996
:1032A00001EB0C034FEA5C1083F800230CF01F0CB9
:1032B000012303FA0CF330BC41F820307047064B71
:1032C0000CF00F0C63441A7630BC7047006002406B
:1032D0000038024000E100E0FCEC00E02DE9F0479E
:1032E000AB48002242F2043C510143588CEA0303EC
:1032F00013F47C540AD00132102AF5D1A54D0023D5
:10330000C5F8103A85F8E039BDE8F0870144A14DD1
:103310000B7FC5F8101A002BF1D18F689E4B9F428E
:1033200002D048339F42EAD19C4A536A43F4006377
:1033300053620DF029FA064688460DF025FA801BE7
:1033400061EB0801B0F57A7F71F10001F5D3934A82
:10335000536A23F4006353620DF016FA064688465A
:103360000DF012FA801B61EB0801B0F57A7F71F164
:103370000001F5D3DFF82492DFF84882D9F8443011
:1033800043F40063C9F84430D9F8303043F4800383
:10339000C9F83030D9F8303043F00C03C9F8303078
:1033A0004FF00D0A00260C220E2108F59960A8F8AE
:1033B000CEA488F8D06409F027FA0C220E2108F276
:1033C000D440A8F8DAA488F8DC6409F01DFA0C22CD
:1033D0000E2108F59C60A8F8E6A488F8E86409F0D6
:1033E00013FA0C220E2108F2EC40A8F8F2A488F897
:1033F000F46409F009FA0C220E2108F59F60A8F880
:10340000FEA488F8006509F0FFF90C220E2108F5EA
:10341000A560A8F82EA588F8306509F0F5F9604B8D
:10342000C8F83475302283F831234FF400325A60E3
:10343000D9F8303043F48003C9F83030564B9F42FE
:103440005BD0584A5849C2F8A060C2F8A8104FF49F
:103450007411D1605549C2F8A0100721C2F8B41008
:103460004B4A534F33461046114605E00133102BAB
:1034700001F1200100F089808E68BE42F6D14D49ED
:1034800001EB43115B01D1F8EC694B498E426DD0E1
:10349000424E316B41F48001316303440D21998325
:1034A000434993688B4225D00134102C02F120024D
:1034B000F7D10020414900230122FFF7DBFED5F8B8
:1034C0000C3A4BB119689A880B691A4204D100234F
:1034D00085F8E039BDE8F087FDF7ECFD0028F6D16E
:1034E000D5F8142AC5F8D029012385F8E039A5F8C4
:1034F000D40909E700EB4410DCE72A492A488E6525
:10350000234A0866334629484FF074668E60886502
:103510000720C8661046114604E00133102B01F164
:10352000200132D08E68BE42F7D1224901EB43110F
:103530005B01D1F8EC6920498E4220D0174E316BE7
:1035400041F48001316303440D219983124993684A
:103550008B4211D00134102C02F12002F7D100204F
:10356000174900230122FFF785FEA8E70B4E316BB8
:1035700041F40011316390E700EB4410F0E7074E8F
:10358000316B41F400113163DDE700235B68FFDE3E
:10359000E809002010200020586402400038024052
:1035A00000E100E000640240802C01406054A30868
:1035B000A064024000000020006002408D08000866
:1035C000C50700080831002070B52D4C636BD90584
:1035D0001ED54FF4807340F2FF56A363A663E36BDE
:1035E000284D23F4414323F03A03E3636B6B9A07BE
:1035F0001FD4012200236A62AB62214A40F2FF53CA
:103600009363D36B23F4414323F03A03D36370BD38
:10361000636B980703D51B4B02229A62EDE7636B3D
:10362000190721D4636B9A0622D5164B06229A629B
:10363000E3E7154BD3F83425136823F00103136037
:10364000E36A002223F00803E3622A636B6BDB0763
:10365000CFD540F24C43A6630121A2600C20E36069
:10366000FCF75CFEA663C4E7064B04229A62C4E73B
:10367000636BDB06C1D5034B05229A62BDE700BF31
:10368000002C01401020002008310020026836493B
:10369000002310B422F0010221248842026003605A
:1036A00043608360C3600361446138D02F4B98420C
:1036B0002ED02F4B98423CD02E4B984240D02E4BD0
:1036C000984232D02D4B984241D02D4B984246D053
:1036D0002C4B984217D02C4B98423CD02B4B984205
:1036E00016D02B4B984224D02A4B984228D02A4BF4
:1036F00098421AD0294B984229D0294B98422ED073
:10370000284B984208D14FF03D5243F8AC2C03E0CF
:103710004FF4746243F8202C5DF8044B7047224B41
:103720005DF8044B3D229A607047204A43F8642CB0
:10373000F2E74FF474125DF8044B43F8382C7047ED
:103740004FF074625DF8044B43F8502C7047184AF0
:1037500043F87C2CE0E73D2243F8082CDCE7154ACF
:1037600043F8942CD8E700BF106002402860024064
:103770004060024058600240706002408860024031
:10378000A0600240B8600240106402402864024019
:103790004064024058640240706402408864024001
:1037A000A0640240B8640240006002403D00002076
:1037B000400F002000003D20214A936803F00C03D5
:1037C000042B10B43AD0082B1FD01E4B1C4C0360A6
:1037D000A1681D4AC1F30311114491F8CC10CB40EC
:1037E0004360A168C1F38221114491F8CC1023FAFF
:1037F00001F18160A1685DF8044BC1F342310A44D4
:1038000092F8CC20D340C36070475368516813F4DA
:10381000800F536814BF0D4A0A4AC3F3881301F09E
:103820003F01B2FBF1F202FB03F3054A5268C2F317
:10383000014201325200B3FBF2F3C7E7034BC5E785
:10384000003802400024F400C86B080800127A0017
:1038500070B5446B8668A38923F400531B041B0CCA
:10386000A381857990F805C02B0303F40051C5F3BB
:1038700080000CF001032A029B001CF0020F4FEAAB
:10388000003002F4806218BF43F0080302431A4379
:10389000238A9BB223F440530B432382A38923F44E
:1038A000B05323F00C031B041B0C1343A381A38A06
:1038B00023F440731B041B0C84B0A3826846FFF7FB
:1038C0007BFF234B9C4205D003F580639C4201D0D3
:1038D000029B00E0039BA2891E49120403EB8303B1
:1038E0004CBF7600B60003EB8303B3FBF6F3A1FBFA
:1038F0000302A08952096426000406FB12334FEA32
:1039000002121CD41B013233A1FB0313C3F3431374
:1039100013439BB223812A07A38A0AD59BB243F0A3
:103920000803A382A3899BB243F40053A38104B08C
:1039300070BD23F008031B041B0CA382F2E7DB001D
:103940003233A1FB0313C3F342131343E1E700BF78
:10395000001001401F85EB512DE9F8431D462E4B09
:103960009DF820609DF824909842884617463BD0E9
:103970002A4B984240D02A4B984245D0294B984236
:1039800021D14B46324629460520FDF743FF044628
:103990000023C4E90B87C4E90733C4E9093366711E
:1039A000A56084F806902046FFF752FFF107626B8E
:1039B00012D4B3070BD493899BB243F40053938181
:1039C0002046BDE8F88300242046BDE8F883D3688C
:1039D00043F08003D360EEE74FF6DF731380D368C4
:1039E00043F02003D360E4E74B46324629460020EB
:1039F000FDF710FF0446CBE74B463246294601202F
:103A0000FDF708FF0446C3E74B463246294603202C
:103A1000FDF700FF0446BBE70010014000440040F2
:103A2000004C004000140140816011E741710FE734
:103A300081710DE72DE9F043704F07EBC00985B0A8
:103A400005464FEAC00899F8EC0B08F019FF064646
:103A500099F8ED0B08F014FF044699F8EE0B73F09B
:103A6000EBFD6B1CDBB21EB140F60C123372F28020
:103A70001CB1237240F60C23E380304604223A2125
:103A800008F0C2FE042220463A2108F0BDFE07EBF2
:103A900008025B4BD2F8E84B9C4200F08E80594BF9
:103AA0009C4200F09580584B9C4200F09C8047441B
:103AB00097F8EF3B022B32D0032B7CD05349544F65
:103AC000012B08BF0F46A6886846FFF775FE26F053
:103AD0003F06029B4F4AB3FBF7F13604A2FB0323D8
:103AE000360C46EA9346A680228822F00102120490
:103AF000120C22808AB2C1F30B019B0C09B942F06F
:103B000001024FF4967101FB03F34349A1FB031338
:103B10009B0901339BB242F4004223841FE0A68834
:103B20006846FFF749FE26F03F06029A394B3604F5
:103B3000A3FB0213360C46EA9346A680218821F0A7
:103B400001010904090C218034499209A1FB0212E8
:103B500092099B0C0133042A238438BF0422A283D8
:103B600023882F4A9BB243F001032380238823F448
:103B7000816323F002031B041B0C4FF4804143F4C8
:103B8000806323802181238823F080031B041B0C86
:103B9000238023889BB202EB451243F0010323806C
:103BA0000121002382F8385582F8391582F83A3518
:103BB00005B0BDE8F0831B4F85E703F5F2331A6AC1
:103BC00042F400121A621A6A22F400121A626EE7B4
:103BD00003F5F0331A6A42F480021A621A6A22F478
:103BE00080021A6263E703F5EE331A6A42F40002B8
:103BF0001A621A6A22F400021A6258E700000020D2
:103C00000054004000580040005C0040009F240029
:103C1000804F120083DE1B43D34D6210632D3E059F
:103C200008310020C02709002DE9F047924E90F995
:103C300000108046807806EBC1050138CC0090B0BA
:103C4000D5F8E81B14282DD8DFE810F04C0120012E
:103C5000150055005F009E00A600C301B6017A0062
:103C600084003C020402D701C000D0002F003700BE
:103C7000A30195015401888A0C8B81B27F4841EAE7
:103C80000441884300F02081D8E90201101A42F271
:103C9000107263EB0101904271F1000102D3152310
:103CA00088F8023010B0BDE8F08798F81300088259
:103CB000C8E90223122088F80200888A0C8B80B29F
:103CC00040EA04406E4C844300F0B28000200E9025
:103CD0000F9001200F910E900E99002900F017828D
:103CE0000F9914310F910F9909684905CCD5142308
:103CF00088F80230D6E798F8110000F0FE0008823C
:103D0000C8E90223052088F80200888A0C8B80B25B
:103D100040EA04405B4C844300F0A1800020009006
:103D200001900120019100900099002900F0FB8191
:103D3000019914310191019909684F05D7D4A3E77E
:103D400098F8110040F001000882C8E902230B2016
:103D500088F80200888A0C8B80B240EA04404A4C02
:103D600084436DD0002004900590012005910490BB
:103D70000499002900F0D181059914310591059924
:103D800009684D05B3D47FE798F813000882C8E9A5
:103D90000223072088F80200888A0C8B80B240EA50
:103DA0000440374C84435ED00020029003900120F1
:103DB000039102900299002900F0C1810399143106
:103DC0000391039909684E0591D45DE7088820F4B2
:103DD00080600004000C088098F8110000F0FE00DC
:103DE0000882C8E90223102088F80200888A0C8B18
:103DF00080B240EA0440234C844312D000200C904F
:103E00000D9001200D910C900C99002900F09181EA
:103E10000D9914310D910D99096848053FF567AF6B
:103E200032E798F81330FF2B06D198F810301BB109
:103E3000132388F8023035E7112388F8023031E780
:103E4000D8F81400012800F08F81022800F0438286
:103E5000098B0E21C8E9022388F8021022E7062305
:103E600088F802301EE7D8F81400002800F06D81B1
:103E7000082388F8023015E7000000200100030045
:103E8000840007008200070002000300088820F475
:103E900000600004000C0880088880B240F4806054
:103EA0000880088880B240F480700880032088F879
:103EB0000200888A0C8B81B2A94841EA04418843F8
:103EC000C8E902237FF4EEAE98F81230002B40F0E0
:103ED000CE8198F81330FF2B00F03F82042388F83E
:103EE0000230DFE6098889053FF5CEAE002388F869
:103EF0000230D7E6344494F8EC0B08F0C1FC0646D7
:103F000094F8ED0B08F0BCFC964AB2F898350133F2
:103F10009BB28246A2F8983516B13368B2881A83EC
:103F2000BAF1000F04D0DAF80030BAF804201A838E
:103F30001121304608F044FC1121504608F040FCA5
:103F40004FF0090965272EB13368B28819690A4212
:103F500040F02381013F00F01D810CF015FC044668
:103F60000D460CF011FC001B61EB0501052871F1F9
:103F70000001F6D3E7E7088880B240F400700880BB
:103F80004FF6FF3088820121C8E9022388F8021029
:103F900088E6D8F81400002800F06D81D8F81840A1
:103FA00014F8016B0E8201381225C8E90504C8E92E
:103FB000022388F8025075E6888A0C8B81B2684823
:103FC00041EA044188437FF45FAE0A2388F8023057
:103FD00068E6088880B240F480700880092088F87C
:103FE0000200888A0C8B81B25D4841EA0441884313
:103FF000C8E902237FF456AEE7E7002401250A94BE
:104000000B940B910A950A98002800F047810B98B1
:1040100014300B900B98006846077FF535AED8F842
:104020001400032800F06D81022800F24381088803
:1040300020F480600004000C0880088880B240F4FE
:1040400000700880098A88F81C40C8E9022388F8B3
:10405000025027E600200124089009900991089455
:104060000898002800F014810998143009900998E4
:10407000006847077FF508AEEFF31185102080F345
:104080001288088880B240F400700880D8F81800C0
:104090000E8A471CC8F81870EDB2067085F31188B7
:1040A0000D8AD8F818106FF001004E1CC8F818607F
:1040B0000D70C8E90223C8F8140088F81C4088F87D
:1040C0000240EFE50020069007900120079106903E
:1040D000069C002C00F0E880079C14340794079C91
:1040E000246864067FF5D0AD0C8AD8F818104D1CF2
:1040F000C8F818500C70D8F8141088F81C00013952
:10410000C8E90223C8F8141088F80200CAE50F991C
:1041100018310F910F990968B6E505991831059185
:1041200005990968B0E5019918310191019909686B
:10413000AAE50D9918310D910D990968A4E5039927
:1041400018310391039909689EE5088880B240F40C
:10415000007008800121C8E9022388F80210A1E557
:104160000100030008310020088820F4806000046A
:10417000000C0880EFF31184102080F31288088B64
:10418000088880B240F40070E4B2088084F311889B
:104190000C215FE616B13368B2885A830CF0F4FA4A
:1041A00004460D460CF0F0FA001B61EB05010528F2
:1041B00071F10001F6D316B13368B2881A830CF09E
:1041C000E3FA04460D460CF0DFFA001B61EB050133
:1041D000052871F10001F6D3B9F101097FF4B2AEFF
:1041E00016B13368B2885A830CF0CEFA04460D46F5
:1041F0000CF0CAFA001B61EB0501052871F1000102
:10420000F6D3BAF1000F04D0DAF80030BAF804207F
:104210005A830CF0B9FA04460D460CF0B5FA001BAF
:1042200061EB0501052871F10001F6D316B1336881
:10423000B2881A830CF0A8FA04460D460CF0A4FAD2
:10424000001B61EB0501052871F10001F6D3BAF1FD
:10425000000F04D0DAF80030BAF804201A8398F975
:104260000000441C3FF442AEFFF7E4FB3EE60F23A0
:1042700088F8023016E5088880B240F400700880A3
:104280000121C8E9022388F81C1088F8021009E50A
:1042900009991831099109990968F5E40B991831C0
:1042A0000B910B990968EFE4079918310791079969
:1042B0000968E9E4D8F81800098A441CC8F81840CD
:1042C0000170D8F81410C8F808200139C8F8141083
:1042D000C8F80C30E6E4088880B240F4006008803A
:1042E000EFF31184102080F31288088B088820F4E3
:1042F00080600004000CE4B2088084F311880D2172
:10430000A8E5088820F480600004000C0880EFF322
:104310001184102080F31288D8F818000D8A461CEA
:10432000C8F818600570088880B240F40070E4B2E4
:10433000088084F31188D8F81800098A441CC8F84A
:1043400018400170D8F814100C200239C8E9022373
:10435000C8F8141088F80200A4E498F81030002B74
:104360003FF4BCAD31E600BF38B5184D9DF814E000
:1043700005EB40144FEA401C94F8390500B938BDEC
:10438000490084F84B25C4F84C3584F849150023BE
:10439000049984F848E5022205F5A76584F84A35B2
:1043A000C4F8501584F8543584F83A2565440CF067
:1043B000EBF902460B462846FFF736FC94F83A35EF
:1043C000002BF4D194F8540538BD00BF083100200B
:1043D00038B5184D9DF814E005EB40144FEA401C29
:1043E00094F8390500B938BD84F84B25C4F84C352C
:1043F00001220023490005F5A76584F84A2584F8C1
:104400005435049A84F848E5022384F84915C4F821
:10441000502584F83A3565440CF0B6F902460B464F
:104420002846FFF701FC94F83A35002BF4D194F8B4
:10443000540538BD08310020F0B589B00023904AFA
:1044400002930393136843F48033136003E0029BE9
:10445000B3F5A04F09D0136803F400330393029B14
:1044600001330293039B002BF1D0854B1B6813F49F
:10447000003318BF01230393039B012B01D000BF1E
:10448000FDE77F4B7F491A6C7F4842F080521A64E7
:104490000A6842F440420A609A689A609A6842F454
:1044A00000429A609A6842F4A0529A6058601A6872
:1044B00042F080721A601A689001FCD5734A40F28B
:1044C00005711160996821F003019960996841F0C4
:1044D0000201A2F580629960936803F00C03082B37
:1044E000FAD1936803F00C03042B00F0C680082B6C
:1044F00000F0AB80664A624B66499868664D674E2D
:10450000674FC0F303100144002491F8DC10CA4047
:104510006449E9606449586FA960596BC6F8E42999
:1045200021F080015963596F604A614841F0807100
:104530005967196B0A431A635A6B5A639A6B9A63E9
:104540001A6C5C490A431A64596C5B4A0A435A6400
:1045500048F2FF7123462246CDE900447AF022FA60
:104560005648234622464FF6FF71CDE900447AF0C3
:1045700019FA5348234622464FF6FF71CDE900440D
:104580007AF010FA4F48234622464FF6FF71CDE9E4
:1045900000447AF007FA4C48234622464FF6FF7152
:1045A000CDE900447AF0FEF94848234622464FF60A
:1045B000FF71CDE900447AF0F5F9454823462246DB
:1045C0004FF6FF71CDE900447AF0ECF941482346FB
:1045D00022464FF6FF71CDE900447AF0E3F9234615
:1045E00022464FF6FF713C48CDE900447AF0DAF9F3
:1045F00004A8FFF7E1F8D5F8FC200499D6F8E439CF
:10460000364842F08072C5F8FC20354AC2F8B00F37
:104610005460106840F0010010604FF47A72B3FBF0
:10462000F2F3013BB3F1807F2E4AB1FBF2F2C7F8FF
:104630009C2508D24FF0E022F0215361072385F832
:1046400023109461136109B0F0BD5168536852683A
:104650004902C2F388124CBF23490D4903F03F03BE
:10466000B1FBF3F303FB02F2054B5B68C3F30143B9
:1046700001335B00B2FBF3F23DE71B4A3BE700BFAF
:10468000003802400070004008544007003C0240DF
:104690000024F400C86B080800ED00E000000020D2
:1046A000083100200003FA0500000008FF916700B0
:1046B00000000240FFC9FE1033570700000402400B
:1046C00000080240000C02400010024000140240AA
:1046D00000180240001C02400020024055CEACC52C
:1046E000001000E040420F0000127A0082B0064B3A
:1046F000002201920193019B03EB80030193019B34
:10470000196002B0704700BF5028004010B51C204F
:1047100008F0B6F81121044608F052F84CB12368AD
:10472000A2885A83C8200CF05DF82368A2881A83F7
:1047300010BDBDE81040C8200CF054B8704700BF51
:10474000704700BF704700BF10B5104C94F8AA35F1
:1047500023B90F4B4FF480225A6110BD4FF0E02275
:10476000D2F8103D23F00603C2F8103DFEF752F9CF
:10477000D4F8B0359B68DB07EBD5D4F8AC261368CA
:1047800023F0030161F307031360E2E7083100201F
:10479000003C01402DE9F04FA34CD4F8AC355A69E8
:1047A000D5078BB002D50BB0BDE8F08F5A699B6975
:1047B00012EA0301F7D0C1F307430803019300F1A4
:1047C000E180019B5D073FD48807CEB203D5D4F8C2
:1047D000AC3502225A610029C0F24A820A05C1F3AF
:1047E000072500F19981370708D5904B9048D3F8F9
:1047F0000C3C9847D4F8AC3508225A61F60600F113
:104800000F82E80600F1BE81A80600F11781019B26
:10481000DA0609D5854B8648D3F81C3C9847D4F86E
:10482000AC354FF480125A61019B9B06BBD57F4B80
:104830007F48D3F8203C9847D4F8AC354FF40012A9
:104840005A610BB0BDE8F08FD4F8B0359E69DB69D2
:104850001E40B6B2002EB7D0754D4FF0000B05F1DB
:1048600018080F46F00740F18280D4F8B015D8F848
:10487000002008694B6B23FA0BF3DB01DBB2034327
:104880009068034013F00109D8B200F00F824B6B1F
:10489000012000FA0BF023EA00034B63012393602D
:1048A000624B6348D3F8043C5FFA8BF1984794F865
:1048B000A335012B00F07E8219F0800F57D0D5E987
:1048C0004CC1D5F82431D8F800E0ACEB010293429A
:1048D000DEF8180028BF134680B20333B0EB930F05
:1048E00045D9D4F8B03594F8A395CDE9026BBA4612
:1048F00067469C46B94237D2D5F82431781A984297
:1049000028BF184600F1030BD5F828314FEA9B0B5E
:10491000B9F1000F10D182B203329210D8F8B8600A
:104920000AD04946013153F8047B37608A42F9D1F5
:10493000D5E94C71D5F82831014403448F42C5F8BC
:104940002831C5F83411DEF818300AD195F81C0169
:10495000012202FA00F0DCF8342022EA0002CCF84E
:1049600034209BB29B45C5D3DDE9026B57467608E0
:104970000BF1010B05F1280508F104087FF472AF73
:10498000394621E7D4F8B0359D69DB691D402D0C0F
:104990003FF417AF04F5B468DFF890B0029104F269
:1049A000F45600274FF00109C24608E06D0807F1F0
:1049B000010706F1040608F1280800F09181EA07D2
:1049C000F4D53068D4F8B015836849690B40D9B282
:1049D000DB0740F1708194F8A335C0F80890012BF3
:1049E00007D10169D8F87C33C1F312015B1AC8F80A
:1049F0008C33DBF8003CF9B25046984794F8A33565
:104A0000012BD3D1002FD1D194F8B136052BCDD1C4
:104A1000D4F8F435074919610749596119684FF00D
:104A200080211960C2E700BF08310020000000208B
:104A3000A836002018000860743C0020D4F8B05557
:104A4000D4F8B825AB68C3F34103022B136814BF35
:104A50000021032161F30A0313606B6843F4807340
:104A600006A86B60FEF7A8FED4F8AC25079ED368B5
:104A700023F47053D360A86810F0060FC0F341010F
:104A800000F03C819F49A0483144814240F2AE8110
:104A90009E48A6F57401A1F51051814240F2AA8109
:104AA0009B499C4831448142C0F0A8819A48A6F1B4
:104AB0008C71A1F54341814240F2A4819749984805
:104AC00031448142C0F0A2819649974831448142E5
:104AD000C0F0A0819548A6F1B771A1F55851814267
:104AE000C0F0A0819249934831448142C0F0968140
:104AF000914892493044884234BF06200520402521
:104B0000012160F38D23D3604FF4005384F8A21584
:104B1000A4F8A45553617AE600238DF8133094F875
:104B2000B2368DF81330864B8648D3F8143C98473C
:104B3000D4F8B035D4F8AC25986894F8AA354FF479
:104B400000615161002B3FF44EAEC3077FF54BAEC1
:104B500094F8B536012B7FF446AE9DF81330032B45
:104B60007FF441AED4F8AC3677491A6842F00102BE
:104B70001A601A6842F003021A600B6943F00603D8
:104B80000B6130E6D4F8B065D4F8AC157368002733
:104B900023F0010373600597059B43F02003059301
:104BA000059B67F38A130593059B0B61674BBC4616
:104BB0000A690592013B02D0059A9206F8D494F84E
:104BC000A12552B1624B03EB820EFF2253F8040F72
:104BD0008260D86B73458260F8D10B2363F30707BB
:104BE00063F3070C4FF0FF33B3614FF00113F36130
:104BF0007761C6F810C03368564823F4FE6333600B
:104C000094F8A325D4F8F435012A18616FD04FF435
:104C100080534B614A4B4B48D3F8103C9847F3E51F
:104C2000D4F8AC359A6922F010029A611A6AC2F37C
:104C30004340022802F00F0100F09080062812D1B4
:104C400001EB810104EBC101D4F87066D1F82C09A5
:104C5000C2F30A1210443268C4F86C2B3268C4F8EC
:104C6000702BC1F82C099A6942F010029A61C8E5CC
:104C700094F8AA353BB1D4F8AC26136823F00300AE
:104C800060F307031360D4F8B0252D4B2D48D3F8FB
:104C9000185C5368029123F001035360A847D4F8CD
:104CA000AC3502994FF000425A6197E5010707D5EC
:104CB000082393605BE68A0707D50223836075E6C5
:104CC000C3060FD51023936051E60B077FF56EAE38
:104CD000DBF8083C5046984733680821996065E640
:104CE00002996EE5410679D5402393603FE61A4A62
:104CF0005A611A684FF080221A6088E74FF40075F5
:104D00000920FEE6401E1BFF3F420F00DFC81000D7
:104D10002013FBFE20D61300FF69180000D3CEFE3F
:104D200040771B00C05BB3FEC091210040AC270060
:104D3000C01D6AFE40E13300803C36FEE09C41002D
:104D400000000020A836002000ED00E0410D030027
:104D5000BC36002018000860743C002047F6F07054
:104D6000104280D0C2F30A1201EB810004EBC000B4
:104D700002F1030C5FEAAC0CD0F82069D4F870E6BD
:104D80004FEA810818BF002006D00130DEF800701D
:104D900046F8047B8445F8D1414404EBC101D1F8C5
:104DA00020091044C1F82009D1F82C091044C1F899
:104DB0002C0958E7BBF1000F7FF47EAD94F8B136B3
:104DC000042B7FF479ADD4F8F435184A1A61184AE7
:104DD0005A611A684FF080221A606DE5830758BF48
:104DE00081467FF569AD02239360C0E5012140252E
:104DF0000E2086E6012140250D2082E60121402576
:104E00000C207EE6012140250B207AE60121402579
:104E10000A2076E601214025092072E6012140257D
:104E200007206EE60121402508206AE61800086088
:104E3000743C002002784368022A11D00C490269B0
:104E4000D1F8180210B41840D1F81042D1F80C1261
:104E5000931E400A04FB030008445DF8044B7047AE
:104E6000034AD2E9802102EB410202EB5320704752
:104E7000D85C00202DE9F04F12F0020A884E83B072
:104E80009B4601D000286FD0D6F80852002D58D18B
:104E90004FF0FF3C834C844FCDF804C0E046E6461B
:104EA000002300922268A57B904200F09E80002D96
:104EB00040D003F58179012D07EB09190AD199F842
:104EC0000750EA0706D415F07E0F03D1ED0900F074
:104ED00090809E460133082B04F11004E2D1BCF10E
:104EE000000F009A04DABEF1000FC0F29280F4467F
:104EF0006D4CD6F8983004EB0C1741F2180E0133C4
:104F000047F80E0041F21C0E0CF5817547F80E3083
:104F10002F01C6F89830E35104EB051300275F60BA
:104F200004EB05139B79042B7AD8DFE803F02940C2
:104F3000194043009C460133082B04F11004B1D101
:104F4000CDE7D6E9833404FB05339842A0D396F825
:104F5000B43113B9012386F8B431534B01225A708E
:104F6000002003B0BDE8F08F96F8B431A6F5805468
:104F7000002B59D001230220637003B0BDE8F08FED
:104F800012F0010776D104EB0513D01093F807E077
:104F9000BBF1030F60F3C71E83F807E068D94FF633
:104FA000FF735B4528BF5B4604EB05108380BAF1B5
:104FB000000F49D1500705D504EB0510C37943F024
:104FC0000103C371D30608D504EB0515EB79C3F3D0
:104FD0004502013262F34603EB71344B012003EBCF
:104FE0004C230B6003B0BDE8F08F009A05BB9C46D4
:104FF0007EE7A568019A954238BF984603F1010300
:1050000038BF2A46082B019204F110047FF44AAFFE
:1050100065E7B8F1000FA8BFC446BFF669AF9FE7C8
:1050200096F8B431002BA5D1012386F8B431A1E75D
:10503000D6F898701C4C03F581759C462B010137FE
:10504000E750C6F898706BE7D6F89830D6F89C0011
:1050500001330130C6F89830C6F89C0004EB0C1000
:1050600041F21C06835104EB051304209871A1E75B
:105070003B4699E70E4BD3F8943B002B3FF470AFBF
:105080000A495E680B4A01EB4C210023B047002817
:105090003FF466AF04EB05150223AB7160E700BF78
:1050A000D85C0020F05C0020D84C0020F04C0020A0
:1050B00008310020F90D000870B5104E3378022B2E
:1050C0000F4B0BBF020AC0F3D412C4B200F07F042E
:1050D000D3F8000282B010440D460023032201A938
:1050E000FFF7C8FE012807D13378019A022B0CBFC5
:1050F00022F8145042F8245002B070BDD84C002061
:10510000D85C00202DE9F04FDFF820910D4699F88A
:1051100000102B68032985B0164640D0022966D1BD
:105120004FEA132A5FFA83F84FF4807B421E012A6C
:1051300024D801249E421CD901288CBF00220122C0
:10514000394F0192D7F878211AB1D7F894119942C2
:1051500050D0D7F8000200235044092203A9FFF7DA
:1051600089FE012824D0022815D020B12B689E4248
:10517000E8D82E60032005B0BDE8F08FB8F1000F2D
:1051800014D0294B93F8B42112B9012283F8B42129
:10519000012389F80130022005B0BDE8F08F4FF0FF
:1051A000800BC3F3D41A03F07F08BFE75C46C1E766
:1051B00099F80010022916D00329ECD1039B53F86B
:1051C000282022F07042019BD5F800C0B2FA82F28A
:1051D00052099A4220D0A0440CEB0403D8452B601E
:1051E0001DD20229EAD1039B33F81820EBE74FF4D4
:1051F000807BD6E7D7F81012013A02EB4122490230
:10520000B2FBF1F21344B3FBF4F204FB12320AB125
:1052100023449B1A2B60AAE76645ACD8A9E70AF19C
:10522000010A4FF00008A2E7D85C0020D84C00200B
:105230002DE9F04FDFF850910B6899F800C0174640
:1052400009F58052BCF1020FD2F8005283B08B46B0
:10525000824640F08180DEB2A6EB030805EB132501
:10526000B8444FF480729044BB4208F1FF38B8FB59
:10527000F2F843D2A844BCF1030F06EB0704A4EBF9
:10528000030414BF4FF4807280229442A8EB0503FC
:1052900028BF1446B6BB944234BF0B220A2201A990
:1052A0002846FFF7E7FD012829D199F800C0DBF86F
:1052B0000000BCF1020F00F1010325D0A64210D27C
:1052C000019906F18042013A01EB8202043901EBB7
:1052D000840142F8043F8A4203F10103F9D1DBF86B
:1052E0000000A31B0344BAF1010FCBF8003023D018
:1052F0009F4205F101054FF00006BCD8012003B024
:10530000BDE8F08F0B22CAE7A642EAD2019906F166
:105310000042013A01EB4202023901EB440122F85A
:10532000023F8A4203F10103F9D1A31B0344BAF1FE
:10533000010FCBF80030DBD1BB42D9D1BCF1020F59
:10534000019B18D004F18044013C4FF0FF3243F838
:105350002420DBF80030CBE703F07F06C3F3D41240
:10536000BCF1030FA6EB03081544B84414BF4FF477
:105370008072802277E704F10044013C4FF6FF720F
:1053800023F814200120BAE7D84C002030B5044699
:10539000C06983B010B9012003B030BD0D460023B1
:1053A000032201A9FFF766FD0128F5D1B4F92020F9
:1053B000002A19DB019B012D4FEA421103EB421237
:1053C00003D0022D1BD1E5205854A368D361237864
:1053D000032B04D10023137753779377D377636A32
:1053E00053831B0C9382D6E7064A92F8B41109B98D
:1053F00082F8B401044B01225A700220CCE7E36822
:10540000E4E700BFD85C0020D84C00202DE9F04331
:10541000814683B00E4699F83C30042B00F2898017
:10542000DFE803F02F03704F3F00434DDFF810819A
:105430004FF6F77705F5805418E0BA4260D871F05E
:10544000A1FE01284FF0000138D1D9F83000FFF754
:1054500033FE012832D1019AD4F81412C9F8302051
:10546000531E8B4228BF0B46C4F814322A78D9F851
:105470003030032A01A918469AB2DED14345DED95D
:105480003EE0710001F0FE014846FFF77FFF012872
:1054900043D1D9F83430002B18BF022089F83C00E2
:1054A000B9E799F82830042B04BF002389F8283085
:1054B000D9F838300BB148469847012003B0BDE811
:1054C000F0831E48D9F82C20D0F89431C0F89421EC
:1054D0009B1AD0F8102202FB03F3D0F8782102EBDC
:1054E0004322C0F87821D0F87C2102EB4322C0F897
:1054F0007C21002100F5B870FFF748FF01280CD18E
:105500000420CBE7D9F8342009F130010020FFF75F
:105510008FFE012801D10320C0E70228CED199F8DF
:105520002830042B04BF002389F8283003B0BDE8DD
:10553000F0830220F3E700BFD84C0020D85C0020A5
:10554000F7FFFF0F38B5044694F83430052B58D8D0
:10555000DFE803F0372B2319100394F82830082BC9
:1055600004BF002384F82830274B012283F8B5219B
:10557000022038BD94F82830082B04BF002384F89B
:105580002830012038BD00212046FFF7FFFE01280A
:1055900037D1042084F83400D6E7D4E90B01FFF7B3
:1055A0008BFD01282DD10320F4E7206B4FF0FF3154
:1055B000FFF782FD012824D1E36A002BF3D00220FB
:1055C000E8E7114DD5F8082204F13001012002323C
:1055D000FFF798FD012805D00238C0B2012810D885
:1055E0000520D7E7E368D5F81012226BC5F814221E
:1055F00003EB4123C4E90332E36A002BCAD16262A0
:10560000C8E7002038BD00BFD85C002070B5044654
:1056100094F83830032B4BD8DFE803F01F170B0248
:1056200000212046FFF7B2FE431EDBB2012B40D91A
:1056300070BD626B04F130010120FFF7F9FD012814
:10564000F2D1032384F83830E2E71F480021FFF746
:105650009DFE0128E8D10223F4E71C4AE56802F523
:1056600080531278D3F81012D3F89401032A14BF90
:105670004FF48072802202FB01F105EB4125C4E961
:105680000350D3F87851A5EB4125C3F87851D3F8EE
:105690007C51861AA5EB41210244C3F89421C3F83A
:1056A0007C11E36AC4E90C025BB960620123C9E7BB
:1056B000022094F82830062B04BF002384F82830F9
:1056C00070BD2663F2E700BF485E0020D84C002082
:1056D0002DE9F0434368C3F308020A44B2F5007FA2
:1056E00083B005460C4605D223446B60012003B00D
:1056F000BDE8F08390F91A20501C0AD0464902F503
:10570000817201EB0212D17921F00101D171FF22E6
:10571000AA7695F91B20511C16D03F4E02F58172D6
:1057200006EB021106EB0212C979D079C1F34501EB
:10573000012986BF01F1FF3101F03F010021FF2661
:1057400061F34600D071EE762A78022ACCD0324E30
:1057500006F58058D8F81022B4EB422F4FEA4229C0
:105760002BDCD8F818721F407A42A24225DCE219DD
:105770004A45286913D32A7E120729D5D8F89421DF
:10578000411C8A421BD300D100214B44DB1BA4EBFC
:105790000909686109EB070429616B600846002864
:1057A000A4D03278032A31D080B24FF6F7729042FB
:1057B0009CD81A4614446C6098E7002097E798F844
:1057C000B42102BB012388F8B43173706B68DCE745
:1057D00001A971F0D7FC0128EFD16B6829782869FD
:1057E0006861A4EB09049944A9EB070301986B6075
:1057F00002293C4428611A46D1D1D8F82012B3EBD3
:10580000412FD7D372E701227270BEE7034A90425C
:105810003FF66CAFCDE700BFD84C0020F7FFFF0F7D
:105820002DE9F047044682B094F83830032B00F29B
:10583000AB80DFE803F09A170C02236C002084F899
:10584000280003B19847022002B0BDE8F087236C1E
:10585000002284F828200BB120469847012002B08E
:10586000BDE8F08723786668484F022B1CBF474B82
:10587000D3F81832204618BF1E40FFF7DBFAC6F3F4
:105880004F26361A0546B6B2A7F5805811E0D7F86C
:1058900010325A1E914557D2FFF71AFF40B997F8B8
:1058A000B43113B9012387F8B431012388F80130EA
:1058B000013506EB050C022201A9002328461FFA38
:1058C0008CF9FFF7D7FA01284FF400724FF000016E
:1058D000BAD1019880F04AF8E3694FF4007120468C
:1058E000002BD4D06368002BD1D1019B4FF0203224
:1058F0004FF02E0C4FF0100EC3F80120C3F8052016
:10590000A3F8092083F800C042F62E6AD4F824C018
:10591000A3F820A083F80BE0C3F82220C3F82620C8
:1059200083F82A20E26BA3F81AC05A872CFA0EFCDF
:1059300022FA0EF283F82BE09A86A3F814C0D7F867
:1059400010325A1E9145A7D3C3EBC353590201F538
:1059500000712046FFF7BCFE28B997F8B4317BB13F
:105960000B4B01225A70022007E02046FFF7EAFDA8
:10597000012802D0022807D1032084F8380053E719
:10598000012387F8B431EBE700205DE7D85C002005
:10599000D84C00202DE9F041B1F904300F2B82B032
:1059A0000E460446174632D02046FFF743FA94F9D4
:1059B0001B80B8F1FF3F3BD05C4B41F2180203EB78
:1059C00008118A58904211D1183303EB4825B38847
:1059D00001331BB205EB4315B38020463D60FFF752
:1059E00029FA3060012002B0BDE8F08103F5805251
:1059F00092F8B41100295CD001225A702378022B4E
:105A00004CD02269002A60D100233B60EAE74FF4C2
:105A10000071FFF75DFE002847D04FF6FF73B3809B
:105A20002046FFF707FA94F91B80B8F1FF3FC3D176
:105A30002378022B41D02269002AE5D03B4B1B780A
:105A4000032B69D093B24FF6F7718B4294BF0023BA
:105A50000123002BD6D138B9354B93F8B421002A55
:105A60004DD0324B01225A700023112201A9FFF7B9
:105A700001FA012810D1019D2E4BEB1A48BF03F209
:105A8000FF13B3F5805F4FEA63222DD24FFA82F8FD
:105A900084F81B80002D9AD12378B0E7244A6368EC
:105AA000D2F82022B3EB422FAED2002002B0BDE8E4
:105AB000F081012182F8B4119EE71D4BD3F820221A
:105AC0006368B3EB422FC6D39EE7184B1B78032BBA
:105AD00019D093B24FF6F772934294BF002301237B
:105AE000002B91D10020E1E7114B93F8B42112B9BA
:105AF000012283F8B4210D4B01225A70C8E701221C
:105B000083F8B421ADE70C4B9A4294BF00230123E4
:105B1000002B7FF479AFE5E7074B9A4294BF00234F
:105B20000123002B7FF46EAF95E700BFD84C002017
:105B3000D85C0020F04C0020F7FFFF0F2DE9F04368
:105B4000044689B094F83030042B11D8DFE803F014
:105B5000501361035A00237E9A0640F1FA80E069EF
:105B60000023112204A9FFF785F9012800F0F18034
:105B700009B0BDE8F083C64D03AE04F11C07324600
:105B800039462846FFF706FF012800F0FD8002286D
:105B9000EED1C04901F5805595F9D2315A1C0AD091
:105BA00003F5817301EB0313DA7922F00102DA7154
:105BB000FF2385F8D23195F9D3315F1C16D003F558
:105BC000817301EB031201EB0313D279D979C2F38C
:105BD0004502012A86BF02F1FF3202F03F02002295
:105BE00062F34601FF22D97185F8D321042306E030
:105BF000A74871F0E3FD4FF6FF720123228484F879
:105C000030309FE70020E36A207009B0BDE8F04320
:105C10001847A14D95F8E031002BA9D104F11C07DC
:105C200003AE05F5DC78324639464046FFF7B2FE52
:105C3000012840F01A81039B002B00F0F4801A78B1
:105C4000E52A01D0002AEED19449591A48BF01F241
:105C5000FF11B1F5805F4FEA612280F050818D49DC
:105C600012018F480244907B04280CD0D5F898008C
:105C70000130C5F89800506004209073D5F89C203E
:105C80000132C5F89C2095F9D221561C0AD002F5A4
:105C9000817201EB0212FF2085F8D201D07920F049
:105CA0000100D07195F9D321501C18D002F58170F4
:105CB00001EB001201EB0011D279C2F34502012A77
:105CC0004FF0FF0088BF02F1FF3285F8D301C87999
:105CD0008CBF02F03F02002262F34600C8711846F2
:105CE000202200217FF042FED4F83120D4F8351074
:105CF00041600260B4F8392094F83B10817202814F
:105D0000627EC272019005A802F0B4FF019B0028D8
:105D100000F0DE809DF816009DF817209DF8191000
:105D200042EA4012BDF81400A0F2BC7042EA4022E0
:105D30009DF81A00490141EA50019DF8180041EA16
:105D4000C02192B288B2D9811A821A83D8820323E1
:105D500055E7204671F032FD2369002B00F08A8060
:105D6000237E03F0F70213F00403227640F09A80BA
:105D7000122A00F0B080E36A0022204684F828202E
:105D800009B0BDE8F0431847DDF80C80B8F1000F0A
:105D900000F0C18098F80030002B00F0BC8098F82B
:105DA0000B9019F0080F7FF4EAAE0B2204F13101D9
:105DB00040467EF035FC00287FF4E1AE637E89EA40
:105DC0000303D90640F1E680324901F5805595F983
:105DD000D2315A1C0AD003F5817301EB0313FF2261
:105DE00085F8D221DA7960F30002DA7195F9D321CE
:105DF000571C3FF4FBAE02F5817201EB021301EB7D
:105E00000212DB79D179C3F34503012B86BF03F17D
:105E1000FF3303F03F03002363F34601FF23D171F7
:105E200085F8D331E2E695F8B831022B4FF009023C
:105E30003FF4DCAE95F8E031002B7FF4D7AEC5E936
:105E40007D3385F8F03185F8EC31D5F8CC31C5F8E3
:105E5000E4310F48D5F8143285F8E021C5F8E8316F
:105E6000FFF7DEFC01283FF4DEAE02287FF480AEAF
:105E70000423C4E6237E1B077FF57DAF064B93F812
:105E80009821002A7FF474AE072283F8982172E7E4
:105E9000905E0020D84C0020D85C0020F04C002000
:105EA000F05C0020A568E66A002384F828302946C3
:105EB0002046FFF70DFC002866D194F82830002B0F
:105EC0007FF456AE0223C4E90B6584F828304FE610
:105ED00044F2817238E7626AE16AA163042084F8BF
:105EE00028002046C4E90B22C4E9023384F83C3080
:105EF0006363636209B0BDE8F04371F05FBC95F87D
:105F0000B42112B9012285F8B421454901224A7011
:105F10006FF00F02A5E6424901F5805595F9D2319F
:105F20005F1C0AD003F5817301EB0313DA7922F0C9
:105F30000102DA71FF2385F8D23195F9D3315E1C65
:105F400016D003F5817301EB031201EB0313D27931
:105F5000D979C2F34502012A86BF02F1FF3202F06D
:105F60003F02002262F34601FF22D97185F8D32156
:105F7000237ED8067FF53AAE2A4871F01FFC4FF613
:105F8000FF72022322843AE6002E3FF4F1AD204650
:105F900033463AE6B8F81420B8F81A30224D43EAEE
:105FA00002436362D5F81022D8F81C30A360520275
:105FB000B3FBF2F102FB113109B113445B1AE36048
:105FC00084F8199095F9D23115495E1C0AD003F571
:105FD000817301EB0313DA7922F00102DA71FF23F6
:105FE00085F8D23195F9D321501C3FF4B0AE02F5BB
:105FF000817201EB021301EB0212DB79D179C3F359
:106000004503012B86BF03F1FF3303F03F03002359
:1060100063F34601FF23D17185F8D33197E600BFC2
:10602000D84C0020905E0020D85C002070B503782A
:10603000017E023B012B044602D911F0060F68D104
:106040008D0643D494F91A30581C0AD0374A03F508
:10605000817302EB0313FF20DA7922F00102DA7177
:10606000A07694F91B305A1C16D0304803F5817283
:1060700000EB021300EB0210DB79C279C3F3450396
:10608000012B86BF03F1FF3303F03F03002363F3CB
:106090004602FF23C271E3760B070ED5244B93F81B
:1060A0009821072A06D093F8B421002A38D01F4A35
:1060B00001215170002283F89821E26A00232370A5
:1060C00084F8283022B3BDE87040104700231948F7
:1060D000E5691A018258954206D00133082BB1D0E8
:1060E0001A0182589542F8D1104803F5817300EBEC
:1060F0000312D279C2F34502012A15D9013A02F0FE
:106100003F0200EB0313D87962F34600D87199E798
:1061100070BD0121FFF73AF90128F9D1217E8FE7FF
:10612000012283F8B421C2E70022EAE7D84C00201C
:10613000D85C0020F05C002038B5184D05F580547F
:10614000014694F8E00120B961B191F8283013B10B
:1061500038BD002038BD04F5DC7044227EF0E4FA3E
:10616000012038BD44220E487FF000FC2B78D4F883
:106170001C12C4F8DC1103224FF6FF70022B18BF6B
:106180001346A4F8D20184F8D021054884F8B83128
:10619000102284F8D12171F011FBE1E7D84C0020E6
:1061A000905E00204FF0FF3C2DE9F041344A354D20
:1061B0006446002304E00133082B02F1100216D0DC
:1061C00010780428F7D103F5817005EB0010C17930
:1061D000CE07F0D4601C52F80A1C01D08C45EAD9D5
:1061E0001C460133082B8C4602F11002E8D1002C2A
:1061F00002DA0120BDE8F081224DDFF8948004F539
:10620000817705EB07139988D8F8943BF9B92601F3
:10621000D8F8943BDFF87C802E4441F2180208EB5A
:106220004421B058EBB1DC68174A0023A047C0B145
:1062300002280AD108F6E87805EB0715D8F89C3053
:106240000122013BC8F89C30AA710020D2E705EB7F
:10625000041041F218022601805813B19B68984738
:10626000D6E70A4BD3F89C2005EB07150320013A2B
:106270000121C3F89C20A87183F8A010E5E700BFB6
:10628000FE5C0020D84C00206D0E0008D85C002079
:1062900008310020F04C00202DE9F04390F8283020
:1062A000013B83B00446082B0BD8DFE803F0393DEF
:1062B0001F24052A0A2F34000121FFF7A7F801281F
:1062C00002D003B0BDE8F0832378216C002284F86B
:1062D0002820002BF5D0D4E9010383424FF00302BC
:1062E00038BF0346A36084F82820E162204603B04B
:1062F000BDE8F0439AE6002103B0BDE8F043FFF7A4
:1063000085B803B0BDE8F043FFF780B903B0BDE83E
:10631000F043FFF717B903B0BDE8F043FFF780BAC9
:1063200003B0BDE8F04309E4534F4368D7F818526F
:10633000026BD7F8101290F800C01D4005EB020E5A
:10634000BEEB412F4FEA4126184645D3A7F58059A9
:106350004FF6F778BCF1020F14D0216908460029E6
:106360005ED16068A368E26A834238BF03460021B9
:10637000A36084F82810002AA3D0204603B0BDE80B
:10638000F04310476068D7F82012B0EB412F68D275
:106390002069217E090735D5D7F8941100F1010E47
:1063A00071452BD297F8B41100294BD1012387F8FE
:1063B000B43189F8013094F800C06368226B921BF5
:1063C0002A4433445B1B9642C4E904E063602263C1
:1063D00018464FF00005BDD9BCF1020F41D021692C
:1063E0000029BFD0254B1B78032B40D089B24FF634
:1063F000F7739942B6D810446060B3E7DFD14FF02D
:10640000000EDCE701A970F0BDFE01287FF459AF52
:106410002069DDF804E094F800C06368226BCEE7E1
:1064200099F800E0BEF1030F12D01FFA81FEC645B5
:1064300094BF4FF0000E4FF0010EBEF1000FA8D038
:106440006068CDE7012189F8011094F800C0B6E733
:10645000DFF82CE0714594BF4FF0000E4FF0010EB5
:10646000EBE7D7F82032B0EB432FC4D37AE7044BE5
:1064700099423FF677AFBEE7D85C0020D84C0020A9
:10648000F7FFFF0F70B5194D194BC5F8983B194B25
:1064900085F8A41B002683F8186A05F69833C0E92E
:1064A00054330D23C0F8583140F201130446C0F8AC
:1064B0005C6100F5A271A0F8443178F0BFF91F23A8
:1064C000C4E9EC36E378012205F51D759342C4F862
:1064D000A853A4F89C2308BFC4F8AC5304F5677113
:1064E0002046BDE8704078F0A9B900BF083100200F
:1064F0005553425310200020F0B50B7813F0600282
:1065000083B004462BD0202A30D14A78FE2A39D0D5
:10651000FF2A2DD14A88002A3BD1CA88002A38D1C7
:106520001F0636D46148624B80F8182AC4F8B42399
:10653000E278012183F89412A4F89C1303F51D73EB
:106540001F21012AC4F8B013C4F8A83304F56771F9
:1065500008BFC4F8AC33204678F070F906E04B78F9
:106560000A2B1AD00B2B08D0012B2AD0002002E0D6
:1065700077F0F6FF022003B0F0BD4D4B4A8883F858
:10658000A92BF3E74F8827B9CD88012D01D11B0630
:1065900042D4204677F0E4FFECE7022180F81111A5
:1065A0004FF48071A0F81C1142490123C0E94A113F
:1065B000C0E94E33C0E94C3200F58E7178F0DCF85A
:1065C000D4E78B88C0681E06DDB244D40192019ADC
:1065D000394B42F010020192019A02610269019264
:1065E000013B02D0019AD206F8D4314E294620460A
:1065F00078F028F8294696F8945202234022204643
:1066000078F050F8022DB1D18121204677F0E0FFDB
:10661000002386F89432A9E7254ED6F8AC329B6960
:106620009847C0B286F8A80B0028B2D0022306F61D
:10663000A83684F811314FF48073C4E94E55C4E98B
:106640004A66C4E94C57A4F81C3104F58E71204603
:1066500078F092F88AE70092009A174B42F02002F5
:106660000092009A65F38A120092009A0261026910
:106670000092013B02D0009A9106F8D40C4E2946B4
:10668000204677F0DFFF294696F8945202234022F5
:10669000204678F007F8022DB6D0012D3FF466AF02
:1066A00001212046FFF7EEFE60E700BF102000202A
:1066B00008310020B13C0020410D030010B50D4B06
:1066C00093F8183A022B07D0033B012B02D8002184
:1066D000FFF7D8FE002010BD074B93F88112044647
:1066E00070F0CCF90028F5DA01212046FFF7CAFE48
:1066F000F0E700BF1020002008310020F8B53F4C23
:1067000094F8186A05467EB1012E01D00020F8BD2C
:106710003B4B93F8811270F0B1F90028F6DA31465C
:106720002846FFF7AFFEF1E7354FB0F8B433D7F89E
:106730007C22C7F8A02B1F2BD7F87822C7F89C2BF8
:1067400008D1304BD7F874229A4203D197F88112BE
:10675000012919D997F8AA3B5A1CD2B207EBC303F7
:10676000042A18BF1646052283F8AC2B4FF40052BA
:106770002846C3F8B02B022387F8AA6B87F8943217
:10678000FBF770FA0020F8BD97F88232013B0F2B1F
:10679000E0D870F073F9002827DB94F8183A013B31
:1067A000022BB3D9B7F8CC3B1BB3042284F8182AC8
:1067B000154AC5F85C61C5E95422D7F87C2287F8F0
:1067C000A46B934228BF1346D7F8A02BC5F85831C5
:1067D00040F20111A5F84411D21A05F5A27128461C
:1067E000C7F8A02B78F02AF890E72846FBF73AFA8A
:1067F0008CE719462846FFF745FE87E71020002062
:106800000831002055534243D83C002038B5084B8E
:106810001B6853B1DB6914460D4698474FF400736B
:1068200002682A600020236038BD1B68FFDE00BFBD
:106830009C3C002008B5054B1B6823B11B69984799
:10684000013840B208BD4FF0FF3008BD9C3C00202D
:106850000020704700207047704700BF704700BF9E
:10686000D0ED007AD0ED036A30EE677AE6EE877AF3
:10687000B0EE670AC0ED007A704700BF90ED017A74
:10688000B5EE407AF1EE10FAF0EE407A09D19FEDC4
:106890000D7A60EE870AF7EE006A86EEA07A80ED48
:1068A000017A31EE077A90ED000A80ED021AC1EE0E
:1068B000076A77EEC07AC0ED036AA6EEA70A80EDFC
:1068C000000A7047DB0FC940D0ED056AD0ED017AB0
:1068D00090ED066AD0ED025A90ED035AC0ED066ABB
:1068E000B0EE407A26EEA70AD0ED007A80ED057A68
:1068F000A7EE870AD0ED077AA5EE860A90ED086A22
:10690000D0ED045AC0ED087AA5EE670AA5EEC60AD6
:1069100080ED070A704700BFF0EE406AD0ED007AC4
:1069200090ED050A90ED037A90ED016AD0ED025AE0
:10693000A7EEA60AD0ED047A27EE407A67EEC07A79
:10694000A6EE267AE5EEA67A90ED066AC0ED067A06
:1069500036EE076A80ED056A704700BF03685A1C6F
:1069600002601970704700BF2DE9F04FD0E9003187
:10697000856889B04A1C00EB81045918F1EE407A11
:106980000591002D92FBF3F103FB1122426000F10F
:10699000800A84ED200AC4ED407A00F5807240F34D
:1069A0008780691C012603F1FF3B06914FF0020925
:1069B0000795B6460599A1EB090090FBF3F103FB9F
:1069C0001100411C91FBF3F403FB14110AEB800846
:1069D00002EB800CF14501EB0E00D8ED006A90FB54
:1069E000F3F49CED006AA3EB090603FB140055DDEC
:1069F000CDE90198CDE903C637460D46044641E08E
:106A0000AB420AEB840902EB840804F1010441DD86
:106A10000AEB850C02EB85060135DCED007AD8ED3A
:106A2000005A96ED007AF4EEE67AF1EE10FA0FDDF8
:106A300099ED005AF4EEC57AF1EE10FA08DDB4EEE5
:106A4000E65AF1EE10FA58BFF0EE456ACCED006A56
:106A5000B4EEC67AF1EE10FA0DDDB4EEE57AF1EEA1
:106A600010FA08DDF4EEC65AF1EE10FA58BFB0EE97
:106A7000656A86ED006A01375F4530DAB0EE476A35
:106A8000F0EE676AA342BBDCAB429046D1464FF0C2
:106A90000104BDDC1646D4460125BEE706990EF179
:106AA000010E714509F102090BF1FF3B82D1079DEF
:106AB0000599491B91FBF3F003FB10130AEB8301CB
:106AC00002EB830391ED000A93ED007A30EE470A62
:106AD000F6EE007A20EE270A09B0BDE8F08FDDE976
:106AE0000198DDE903C698ED006ADCED006A41E03B
:106AF0008B420AEB800C02EB800700F1010041DDC4
:106B00000AEB810502EB81040131D5ED007AD7ED66
:106B1000005A94ED007AF4EEC67AF1EE10FA0FD531
:106B20009CED005AF4EEC57AF1EE10FA08D5B4EEF9
:106B3000C65AF1EE10FAD8BFB0EE456A85ED006A8C
:106B4000B4EEE67AF1EE10FA0DD5B4EEE57AF1EE98
:106B500010FA08D5F4EEE65AF1EE10FAD8BFF0EECE
:106B6000656AC4ED006A01365E4597DAF0EE476A61
:106B7000B0EE676A8342BBDC8B421746D4464FF0C7
:106B80000100BDDC144655460121BEE703685A1CCE
:106B900002601970704700BF024B186803681B68D9
:106BA000184700BF005F0020007970470079C0F3EC
:106BB0004010704700794009704700BF90F83C20B2
:106BC000034602F0FF0012B1002283F83C20704718
:106BD0004FF48053838170474FF400638381704783
:106BE0004FF40063838170474FF4006383817047E3
:106BF0004FF40063838170474FF4006383817047D3
:106C00004FF4006383817047074B10B403F1100108
:106C1000002453F8042B824208BF43F8044C8B42F3
:106C2000F7D15DF8044B7047045F002070B5374C16
:106C3000608CA38AB4F92C50B4F92660B4F91AC058
:106C40001B1A208C00FB03F3B4F92A0005EBE33593
:106C5000C00290FBF5F000EBE330A0F57A6EB4F9DA
:106C6000243020630EFB0EF52D1305FB06F605FB05
:106C700003F3B4F91C500EFB0CFC0EFB05F51B14C2
:106C800003EB65334FEAEC2CB4F918500CEBE62C0F
:106C90000CEB850C0233B4F93450A66BE48B9B10DB
:106CA00003F500430CFA05FC04FB03F30CF1020CA2
:106CB0004CF25034A6EBAC0C2C4104FB0CF4002C31
:106CC0004FEAD333ABBF6400B4FBF3F3B4FBF3F38D
:106CD0005B0089B11C120E4D04FB04F440F6DE3655
:106CE00006FB04F403FB05F5241404EB254404F629
:106CF000CF6403EB24130B602AB100EB800040004B
:106D0000083000111060012070BD00BF005F00203E
:106D100043E3FFFF01207047012070472DE9F04F4A
:106D2000734DE86BB5F84030B5F94CE0B5F948C0A3
:106D3000B5F84680B5F94E6085B0C3EB20140092DB
:106D400004FB04F4B5F94420CDF80CE0241302FB55
:106D500004F45B00B5F942200296C3EBE00302FBAA
:106D600003F3A41304EBE324EB6D0193A4F5FA30D1
:106D7000B5F94A30AC6580FB00EA4FEAE37B03FBE0
:106D80000AF98CFB00C20EFB0B99A3FB0E3BCB4414
:106D900012031B0A42EA1C5243EA0B634FEA0C3C03
:106DA00013EB0C0342EB2B22A3FB083C02F5004241
:106DB00008FB02CC4FEAEC734FEA6C0953EA6C0C07
:106DC0000F46B5F9501000F09180029E019A86FBA3
:106DD0000008C2F5801C01FB0AFA4A464FEA4848FF
:106DE0004FEAE17948EAD0380EFB09A94004A1FB3B
:106DF0000E1E4118F14449EB080900200CF0004830
:106E0000039E411848EA5C084FEACC7CBCEB010CBD
:106E100009EBC60968EB09081CEB0C0E48EB0801EE
:106E20001EEB0C0E48EB010188014FEA8E1940EA77
:106E30009E601EEB090E41EB0001890041EA9E7144
:106E40004FEA8E0E1EEB0C0E48EB01014FEA8E004E
:106E5000890010EB0C0041EA9E7148EB010178F0CB
:106E600061FDB5F956304FEA61384FEA503E4EEABF
:106E7000C14EDA1703FB08F984460EFB0299B5F9F7
:106E80005400B5F95220A3FB0E35A94403FB08F5C5
:106E90000EFB0955A3FB0E3E75445B0E43EAC5137A
:106EA00013EB0C0341EB65654FEAE07E00FB01F15B
:106EB0000EFB0C11A0FB0C0C6144C00C40EA4130ED
:106EC0001B1845EBE1451B0A43EA056303EB02137C
:106ED0000FB11B0A3B60009B23B104EB8404803498
:106EE00024121C60012005B0BDE8F08F0023EFE7FD
:106EF000005F002031B10A4BD3ED1F7AFDEEE77A37
:106F0000C1ED007A52B1064B9FED067AD3ED207A9F
:106F100067EE877AFDEEE77AC2ED007A01207047CE
:106F2000005F00200000C8422DE9F04F614DB5F828
:106F30009230D5F88400B5F890E0B5F88E40B5F8F9
:106F4000946085B01B02C01A67EB0707B5F88C3058
:106F50000191AEFB001C0EFB07CCC9091B0441EAE2
:106F60004C61C9189346A4FB003EB5F88A2004FB87
:106F700007EE4FEA13234FEAC23243EA0E634FEAA9
:106F8000EC1C4CF1000C9B18A6FB002406FB0744EC
:106F90004FEAD25242EA44224FEA2E2E4EF1000E20
:106FA000E41512F5FA6944F10006B9F5FA6F029694
:106FB00076F1000632DAA2FB02A802FB04F6039483
:106FC00008EB46044FEA84084FEA8A0616EB0A06E5
:106FD00048EA9A7844EB08084FEA560A4AEAC87A1F
:106FE000B608B1EB0A0A46EA8876334C6CEB680CBB
:106FF0009E1B3346029E6EEBA80EA1454FF0FF3458
:10700000A641514627DB00FB07F7A0FB000202EB7D
:107010004702C00F40EA4200B9EB0009019C8CB165
:10702000D5F89800A0FB033200FB0E225B0D43EA6B
:10703000C2235B1A4FEA625262EB0C02DB0B43EA9B
:1070400042432360BBF1000F01D0CBF80090012038
:1070500005B0BDE8F08F40F6AC56039C921944F1A0
:10706000000402FB04F4A2FB026202EB44024FEABA
:10707000C208F400341B48EA567862EB080864182A
:107080004CEB080C2146B41942EB0208A41942EB60
:1070900008084FEA880848EA9478A400A41B68EB23
:1070A0000208620842EAC8729A1A6EEB680E13462A
:1070B000A9E700BF005F002024FAFFFF012070470E
:1070C00010B40F4B0F4C1B68D4F89C001B1AFA2B02
:1070D0000BD811B1D4F8A4300B6012B1D4F8A83099
:1070E000136001205DF8044B7047074A13680020C5
:1070F00023F0040384F8A00013605DF8044B70478C
:10710000242A0020005F002000000010064B00220F
:107110000021C3F8AC20C3F8B020C3F8B420C3F8F2
:10712000B8100120704700BF005F0020104B114ACB
:107130001B68D2F8B8105B1AFA2B16D8D2ED2B6A5E
:1071400092ED2C7AD2ED2D7AFDEEE66ABDEEC77A8D
:1071500016EE903AFDEEE77AC38617EE103A0387F3
:1071600017EE903A4387012070470020704700BF18
:10717000242A0020005F002030B50F4A83B092F827
:10718000BC500191B5B9D2F8C0509DB12B681A68B6
:1071900082B19B6873B104462846984750B12B686A
:1071A000019922461C6828460B46214603B0BDE8DB
:1071B0003040084703B030BD005F00200B4B70B576
:1071C000D3F8C4608EB133681A6872B19B6863B13A
:1071D000054630460C46984738B133682A46196848
:1071E00030462346BDE87040084770BD005F002070
:1071F0002DE9F041DFF888801F4FD8F8D8203B6890
:10720000B8F8DC10118343B39B69984728B3002674
:107210003B6813B11B69984790B9B6F57A7F21D0C6
:1072200009F0B2FA013604460D4609F0ADFA001B2A
:1072300061EB0501B0F57A7F71F10001F5D3E7E765
:10724000D8F8D830B8F8DC205A83B6F57A7F4FF0FA
:10725000FF3018BF0020BDE8F081084B3B601B6881
:107260009847D4E7D8F8D830B8F8DC205A834FF0E4
:10727000FF30BDE8F08100BF9C3C0020300C0020B6
:10728000F03300202DE9F84FDFF8BCA0DAF89C00BD
:107290009046BAF8A0204283002B45D09B46294F48
:1072A0008946C34441F289363A6852B10023546892
:1072B00049461A464046A047A0B93B680BB11B6936
:1072C0009847013E34D009F05FFA04460D4609F0B4
:1072D0005BFA001B61EB0501B0F57A7F71F10001EB
:1072E000F5D3E1E741F289363B6813B11B69984752
:1072F00080B9013E1CD009F047FA04460D4609F05A
:1073000043FA001B61EB0501B0F57A7F71F10001D2
:10731000F5D3E9E708F10108D84509F50079C1D1AD
:10732000DAF89C00BAF8A02002830020BDE8F88FAC
:10733000DAF89C30BAF8A0201A834FF0FF30BDE88D
:10734000F88F00BF9C3C0020F03300202DE9F84F5F
:10735000DFF8C0A0DAF89C009046BAF8A02042837B
:10736000002B48D09B462A4E8946C3443268FAB166
:1073700041F289370023D46849461A464046A0475F
:107380003368B0B10BB11B699847013F37D009F0A2
:10739000FBF904460D4609F0F7F9001B61EB050106
:1073A000B0F57A7F71F10001F5D33268002AE1D19E
:1073B000002341F2893713B11B69984788B9013F0F
:1073C0001DD009F0E1F904460D4609F0DDF9001B76
:1073D00061EB0501B0F57A7F71F10001F5D33368F7
:1073E000E9E708F10108D84509F50079BED1DAF8D6
:1073F0009C00BAF8A02002830020BDE8F88FDAF8DC
:107400009C30BAF8A0201A834FF0FF30BDE8F88F07
:107410009C3C0020F033002038B51446002944D0AD
:10742000344BDFED355AD3ED327AB3F9E42093EDE6
:10743000350AB8EEE77A05EE102AC7EE256AB3F9E9
:10744000E0200D46D3ED337A06EE102AF8EEE77A07
:10745000B3F9E220C7EEA54A05EE902AB3F9DE2083
:1074600007EE102AF8EEE55AB3F9DC20B8EEC77A39
:1074700007EE902AA6EEA57AB8EEC55AB8EEC66A0F
:10748000F8EEE77AA6EE856AE6EE877A93ED367A2D
:10749000B8EEC77AB8EEC00AA6EE867AA6EE870ADC
:1074A000A4EEA70A79F0C4F928600CB3114B9FED44
:1074B000126AD3ED337AB3F9D220B3F9D030F8EEB3
:1074C000E76A07EE102A86EE860A07EE903AB8EED3
:1074D000C77AF8EEE77A20EE070AB6EE006AA7EE62
:1074E000860ADFED066A20EE260A79F0A1F920600F
:1074F000012038BD005F00200000F04A0000C842B3
:107500002DE9F0410446D0E90030134483421DD8F0
:107510000D4601EB0208B2B104F10C07002601E0B0
:10752000A84510D023695A1C2261234415F8011B79
:107530001973042AF4D139462046FBF797FAA84577
:10754000C4E90460EED16069BDE8F0814FF0FF301E
:10755000FAE700BF034690F910002DE9F041244CF2
:1075600000EB800016469A6804EB80009207D0F882
:10757000208009D5404677F0BFFA3146404677F083
:10758000BBFA0120BDE8F0815D69084615B12B68A2
:10759000AA885A83174B184F1C68184B7A684FEA11
:1075A000C40CA3FB0C3C4FEA9C1C7B689B1A9C45BB
:1075B000FBD20146404677F09FFA3146404677F0CD
:1075C0009BFA0E4B78680C494FF4FA7204FB02F2F6
:1075D000A3FB023292094B681B1A9A42FBD2002D80
:1075E000CFD02B68AA881A830120BDE8F08100BFA4
:1075F000300C0020A4360020001000E0D34D6210B3
:1076000000680379012B0AD0022B01D000207047BB
:107610008368DB074FF0F00218D5FF219AE700B529
:10762000826890F910C0417C85B002F0010201929D
:107630000DF10F0200926046FF224FF0F00C8DF822
:107640000FC0FCF7C5FE05B05DF804FB7F2181E7A4
:1076500000680379CA4341EA0211012BCAB208D07B
:10766000022B01D0002070478368DB0716D5D2219A
:1076700070E700B585B090F910C08DF80F208268D2
:10768000417C02F001020DF10F00CDE90002D2228F
:107690006046FCF79DFE05B05DF804FB522159E7FA
:1076A00000680379012B0AD0022B01D0002070471B
:1076B0008368DB074FF0B40218D5FF214AE700B515
:1076C000826890F910C0417C85B002F001020192FD
:1076D0000DF10F0200926046FF224FF0B40C8DF8BE
:1076E0000FC0FCF775FE05B05DF804FB7F2131E7A4
:1076F00000680379012B09D0022B01D000207047CC
:107700008368DB070A4616D5A52123E700B5826802
:1077100090F910C085B002F001028DF80F10417C85
:107720000DF10F00CDE90002A5226046FCF750FEE6
:1077300005B05DF804FB25210CE700BF0068037964
:10774000012B0AD0022B01D0002070478368DB0791
:107750004FF0960218D5FF21FCE600B5826890F93B
:1077600010C0417C85B002F0010201920DF10F02C0
:1077700000926046FF224FF0960C8DF80FC0FCF788
:1077800027FE05B05DF804FB7F21E3E6006803797E
:10779000012B09D0022B01D0002070478368DB0742
:1077A0000A4616D58721D5E600B5826890F910C043
:1077B00085B002F001028DF80F10417C0DF10F0031
:1077C000CDE9000287226046FCF702FE05B05DF8B5
:1077D00004FB0721BEE600BF00680379C901012B45
:1077E000CAB205D0022B01D0002070477821B1E643
:1077F00000B585B090F910C08DF80F208268417CEB
:1078000002F001020DF10F00CDE90002782260467E
:10781000FCF7DEFD05B05DF804FB00BF00680379EE
:10782000012B0AD0022B01D0002070478368DB07B0
:107830004FF0550218D5A5218CE600B5826890F965
:1078400010C0417C85B002F0010201920DF10F02DF
:1078500000926046A5224FF0550C8DF80FC0FCF742
:10786000B7FD05B05DF804FB252173E600680379D8
:10787000012B0AD0022B01D0002070478368DB0760
:107880004FF02E0218D5F42164E600B5826890F915
:1078900010C0417C85B002F0010201920DF10F028F
:1078A00000926046F4224FF02E0C8DF80FC0FCF7CA
:1078B0008FFD05B05DF804FB74214BE6144B0068A6
:1078C0009A8E037992013432012BD2B208D0022B66
:1078D00001D0002070478368DB0716D5F42139E614
:1078E00000B585B090F910C08DF80F208268417CFA
:1078F00002F001020DF10F00CDE90002F422604612
:10790000FCF766FD05B05DF804FB742122E600BFBC
:10791000005F002000B500680379012B85B012D00C
:10792000022B03D0012005B05DF804FB8368DB0760
:107930004FF031024CBFF4217421FFF70BFE012000
:1079400005B05DF804FB826890F910C0417C02F03C
:10795000010201920DF10F0200926046F4224FF0F5
:10796000310C8DF80FC0FCF733FD012005B05DF838
:1079700004FB00BF00680379012B06D0022B01D065
:107980000020704701225821E4E500B5826890F993
:1079900010C0417C85B002F0010201920DF10F028E
:1079A0000092604658228DF80F30FCF711FD05B0AB
:1079B0005DF804FB00680379012B06D0022B01D08F
:1079C0000020704701224821C4E500B5826890F983
:1079D00010C0417C85B002F0010201920DF10F024E
:1079E0000092604648228DF80F30FCF7F1FC05B09C
:1079F0005DF804FB00680379012B06D0022B01D04F
:107A0000002070471A460821A4E500B5826890F965
:107A100010C0417C85B002F0010201920DF10F020D
:107A20000092604608224FF0020C8DF80FC0FCF760
:107A3000CFFC05B05DF804FB00680379012B06D08C
:107A4000022B01D0002070470122082182E500B5F9
:107A5000826890F910C0417C85B002F00102019269
:107A60000DF10F020092604608228DF80F30FCF7EE
:107A7000AFFC05B05DF804FB2DE9F0410C4E356814
:107A800073691D4011D0DFF82C800127B5FA85F409
:107A9000C4F11F0408EB840307FA04F4D3F8E800E8
:107AA00003689847A5437461F0D1BDE8F08100BF39
:107AB000003C0140005F0020074B53F8203021B10B
:107AC0004BB11A689B8853837047002BFCD01A680F
:107AD0009B88138370477047C06C080810B54FEA45
:107AE000511E024400EB8E0C624529D901F01F03A0
:107AF0004FF0FF3450F82E1004FA03F30B4093FAC2
:107B0000A3F3B3FA83F3DBB2202B16D10CF10401FB
:107B10008A4202D817E08A4212D98C460431DCF836
:107B2000003093FAA3F3B3FA83F3DBB2202BF2D045
:107B3000ACEB000C03EBCC0010BD03EB4E1010BD02
:107B40004FF0FF3010BD204610BD00BF03694168F3
:107B500090ED067AF0B4C56A394E876853EA01029F
:107B600004BF316841606A1C30EE077A0133012A94
:107B700080ED067A0361C26240D090ED075AD0EDE5
:107B8000096A346807EE902A70EE455AB8EEE76A43
:107B9000611AC5EE867AB94277EE857A30EE670AC9
:107BA000C0ED087AE5EE806AC0ED077AC0ED0A6A9A
:107BB000C0ED096A01D8F0BC7047012A29DD07EE43
:107BC000905AF8EEE77A86EEA76AB5EEC06AF1EE53
:107BD00010FA1EDBF1EEC67AF4EE677AF1EE10FAD7
:107BE00017D6D0ED056AF4EEE76AF1EE10FA13D578
:107BF000037BEBB10323F0BC03707047326880ED68
:107C0000080A521ABA424FF0000180ED070A416299
:107C1000D1D9DFED0C7AE4E707EE903AF8EE677A17
:107C20000223C7EE276AF0BC0370C0ED066A7047F6
:107C300031684160002203618261C362BBE700BF1B
:107C4000242A002000000000DFED4F4A10B58446D2
:107C500000F1480E0346B1EC017AD3ED067ADA6AF8
:107C600077EE877A0132012AC3ED067ADA6254D0C0
:107C700093ED075A93ED096A07EE902A77EE455A7D
:107C8000F8EEE77AC5EEA76A76EE857AF0EE466AF8
:107C900037EE677AC3ED087AE5EE876AC3ED0A6AC4
:107CA000C3ED077AC3ED096A18337345D3D1374C56
:107CB000416822680369521A816801338A4203616C
:107CC0002AD990ED056A00F1300EDCF82C20DCEDAD
:107CD0000A6A012A02F1FF3126DD07EE901AF8EE5A
:107CE000E77A86EEA77AB5EEC07AF1EE10FA1BDBE2
:107CF000F1EEC77AF4EE677AF1EE10FA14D6E645A3
:107D0000B4EEE76A0CF1180C16D0F1EE10FADCD5DF
:107D1000037B6BB30323037010BDF0EE477AF0EEE4
:107D2000646A83ED087ABBE7DFED177AE645B4EEC7
:107D3000E76A0CF1180CE8D1F1EE10FAE8D407EE7E
:107D4000903AD0ED066A90ED0C7AD0ED125AF8EE2A
:107D5000677A022386EEA76A0370C7EE276A85EE6C
:107D6000A77A80ED066AC0ED0C6A80ED127A10BD2C
:107D700000222168416003618261C362026343643F
:107D80008264C36510BD00BF00000000242A0020EB
:107D9000B0EEC06AF0EEE05AF4EEC65AF1EE10FA18
:107DA000F0EE407A0EDCB5EE400AF1EE10FA4BD060
:107DB000F4EEC65AF1EE10FAF0EE466A50D5B0EE87
:107DC000655A03E0F0EE656AB0EE465A85EE267A13
:107DD0009FED252A9FED253A9FED254ADFED254AA7
:107DE000DFED252ADFED253ADFED256AA7EE023A21
:107DF000E7EE223AA7EE034AB7EE005AE7EE044A4E
:107E0000A7EE235AE7EE246AF4EEC65AB1EE667A7C
:107E100087EE050AF1EE10FA48BF9FED1A7AF5EEEB
:107E2000C00A48BF37EE400AF1EE10FA48BF9FED96
:107E3000167AF5EEC07A48BF37EE400AF1EE10FA36
:107E400048BFB1EE400A7047DFED107A9FED100A8F
:107E5000F5EEC00AF1EE10FA58BFB0EE670A7047AF
:107E6000B0EE465AB2E700BF39094E3DE3B59EBEBB
:107E700088FA16BE45FE7FBF99FB243F69A2163ED5
:107E8000A7DFA8B4DB0FC93FDB0F4940A7DFA83449
:107E9000DA0F494091ED007AD0ED047A90ED054A71
:107EA000D0ED064A90ED075AD0ED085A90ED096AD8
:107EB000D0ED0A6AE7EE077AF7EE003AC0ED047AF1
:107EC00091ED007AD1ED017AA7EE274A90ED0B7A79
:107ED00080ED054A91ED024A91ED003AD0ED0C7A21
:107EE000E3EE044AC0ED064AD1ED004A35EE245ACD
:107EF00080ED075AD1ED014A91ED005AE4EE855A22
:107F0000C0ED085AD1ED015AA5EEA56A80ED096AC7
:107F1000D1ED015A91ED026AE5EE866AC0ED0A6A7A
:107F2000D1ED016A37EE267A80ED0B7AD1ED026A47
:107F300091ED007AE6EE877AC0ED0C7A91ED026A57
:107F4000D1ED016AD0ED0D7A90ED0E7A90ED0F4AE9
:107F5000D0ED104A90ED115AD0ED135AE6EE267A84
:107F600075EEA35AC0ED0D7AD1ED026AD0ED127A0A
:107F700090ED006AA6EEA67AD0ED016A80ED0E7A49
:107F800091ED027A34EE074A90ED027A80ED0F4AC5
:107F900091ED004A74EE844AC0ED104AD1ED014AD9
:107FA00035EE245A80ED115A91ED025AC0ED135A64
:107FB00077EE857AC0ED127AD1ED017AD1ED005AD3
:107FC00091ED025A67EEA77AE5EEA57AE5EE057A1D
:107FD000A5EEA76A80ED006A91ED016AE6EE276AD8
:107FE000C0ED016AD1ED026AA6EEA77A80ED027AB1
:107FF00090ED037A77EE277AC0ED037A704700BFE1
:108000002DE9F04F4FF0000989B0864600F11005C8
:108010000646034600F13008074648462C46CDF890
:108020000CE08B469C46B24600283CD10CF1040C77
:10803000A445FBD1032800F1010151D09C46AA467A
:10804000029398B1DCED047A0192AAEB0903B646DB
:108050007246F3EC016A92ED007AE6EEC77A534578
:108060000EF1100ECCED047AF2D1019ADCED046A27
:1080700015ED047AC6EE877A0CF1100CC4450AF1AE
:10808000100ACCED007ADCD1029B0436143308468A
:1080900008F1040814351034103709F104099C461E
:1080A000B2460028C2D0DCED007A0192D6463946AD
:1080B0007246F1EC016A92ED007AE6EEC77A9942D7
:1080C0000EF1100ECCED007AF2D10CF1040CA445A7
:1080D000019A0AF1040AE6D1032800F10101ADD1A9
:1080E000DDF80CE0002359460493059306930793AB
:1080F0007646774604AD0020F2EC017AE5EC017A91
:10810000B0B104AC3B46B4EC017AF3EC016AE6EEA4
:10811000C77AB34245ED017AF5D1013004280BD07E
:10812000F2EC017A10371436E5EC017A0028E8D138
:10813000103714360120DFE708AD75ED017A1031F4
:108140000EF1400E04287446A1F1040241ED017ABB
:108150001ED07346F3EC016AB1EC017AE6EEC77A01
:10816000A342C2ED007AF5D15EED016A87EEA67AF0
:10817000013882ED007A17D0AEF1140E103C114692
:1081800075ED017A0428A1F1040241ED017AE0D1F4
:108190005EED016A87EEA67A103CAEF1140E032064
:1081A00001ED017A1146EBE709B0BDE8F08F00BFA1
:1081B000DFED297AB4EEE70AF1EE10FA28DD9FED43
:1081C000277A30EE470AB4EEE70AF1EE10FAF8DC4F
:1081D000DFED237AB4EEE70AF1EE10FA2FDD30EE90
:1081E000670A37EEC00A60EE007A9FED1E7A9FEDB7
:1081F0001E6ADFED1E6AA7EE876A9FED1D7AE7EE25
:10820000866A60EE275AA7EEA67AA5EE870A70471F
:10821000DFED187AB4EEE70AF1EE10FAD8D59FED4B
:108220000F7A30EE070AB4EEE70AF1EE10FAF8D44E
:10823000DFED0B7AB4EEE70AF1EE10FACFDC9FED3A
:108240000E7AB4EEC70AF1EE10FA44BF30EE270AF8
:1082500037EE400AC7E700BFDB0F4940DB0FC940DC
:10826000DB0FC93F9A7C2E36FAAF4FB93587083CF1
:10827000A4AA2ABEDB0F49C0DB0FC9BF10B5404C12
:10828000B4FBF2F4A14219D3DFED3E7AF7EE005AC7
:10829000B0EE677AB0EE676AF0EE676A0023C0ED71
:1082A000005AC0ED017A80ED027A80ED036AC0EDDC
:1082B000046A836143610362C36110BD07EE902AC3
:1082C000B8EE677ADFED307A27EE277AB7EE006AEC
:1082D000C6EE076A07EE901A9FED2C7AF8EE677AE1
:1082E000B0EE405A67EE877AC7EEA64AFDEEE47A12
:1082F00017EE902A2032402A3FD8B0EE640AFFF7EA
:1083000057FFB0EE404ADFED227A34EEA70AFDEEC9
:10831000C07A17EE902A2032402A29D8FFF748FF6A
:10832000F8EE006A60EE266A012B1CD0B7EE006AF8
:1083300036EE406AF6EE004A66EE244A35EE055AFD
:10834000F7EE007A84EE057A77EE275A37EEC75AB1
:1083500084EEA57AC6EE257A86EEA56AC5EE256A74
:10836000F0EE475A9AE7B0EE666AF7EE004AE5E7A4
:10837000DFED086A9FED030AD6E79FED024AC2E7E8
:1083800020A1070000000000BD378635DB0FC94083
:10839000DB0FC93F00000080DFED077A30EE270ACF
:1083A000FDEEC07A17EE903A2033402B00D8FFE65E
:1083B0009FED020A704700BFDB0FC93F00000000BD
:1083C0002DE9F84FDDF82CB09DF828408946002CA7
:1083D0001BF8011B0CBF4FF020084FF030081C1E8B
:1083E0000546174608463ADB00295CD0002C55D0DC
:1083F0004FF0000A5B4600E064B313F8016B013CE8
:10840000002EF9D1BAF1000F2FD1264644B14D45C7
:108410004146284600D2B847013CF8D10B9B18785A
:108420000146A0B14FF0FF344FF0000A00E09B4638
:108430004D45284600D2B8475B4613F8011B00297A
:10844000F5D10B9BF61A5E44BAF1000F10D13046FD
:10845000BDE8F88FBAF1000F1BD15646E0E7634242
:1084600029B31C464FF0010AC4E70028E0D10646B4
:10847000002C04F1FF3AEADD54464D4541462846BA
:1084800000D2B847013CF8D2013656443046BDE828
:10849000F88F06460028DAD02646C9E72646A246C7
:1084A0004FF0FF34C4E72646002CB0D1CFE76FEA87
:1084B000040A0E46E0E700BF0FB430B583B006AB48
:1084C0000A4C53F8042B0193D4E9D10171F018F848
:1084D0000546206803685B6998470028F9D028465C
:1084E00003B0BDE8304004B0704700BF005F00201B
:1084F0000EB410B583B005AB044653F8042B0749FE
:10850000009301A8019470F0FBFF019B00221A70F8
:1085100003B0BDE8104003B0704700BF8D6B00088A
:108520000CB4F0B53C4CD4F84C33ADF5277D002BA2
:108530006DD094F8543399420BD9D4F858230123C1
:108540008340134205D10DF5277DBDE8F04002B010
:108550007047324B324A1B68A2FB030292094FF468
:108560007A7101FB123306A82E49FFF7C1FF06AB53
:1085700003442D49AC9A01930646ADAB01A8009384
:1085800070F0BEFF019B0A22591C01911A70019BD9
:108590000022591C01911A70D4F84C53ADB12B68CC
:1085A0005B6A1BB128469847D4F84C539DF81810C5
:1085B0000029C8D00DF119042B6828461B6898477C
:1085C00014F8011B0029F7D1BDE7D4F85073002F30
:1085D000B9D0304426AB841CFD2206A9ADF810208A
:1085E00018462246CDF81250ADF816507CF09CF893
:1085F00002220346044402A93846CDE9023436F08B
:10860000D1FC0DF5277DBDE8F04002B07047D4F8ED
:108610005033002B8DD196E7005F0020242A0020E4
:10862000D34D6210981609085D690008184A10B504
:10863000D2F85C43033004EB9003B3F5007F18D805
:1086400002EB8101C2F85C3302F5587202EB84043C
:10865000D1F8602B20F003001044C3F50073C1F87B
:10866000600B0C4A9B0004210020FFF759FF2046B5
:1086700010BD00210846084AFFF752FF074AD2F80A
:10868000B030002443F00073C2F8B030204610BD73
:10869000005F0020A4160908C81609080000001091
:1086A00038B50568EB690446F3B1987800B938BD70
:1086B000B3F90A2007EE902AF8EEE77A0120C4ED1C
:1086C000057AB3F90C2007EE902AF8EEE77AF1EE7E
:1086D000677AC4ED047AB3F90E3007EE903AF8EEFB
:1086E000E77AC4ED067A38BD09211420FFF79EFF12
:1086F0000346E861D9E700BF38B50568EB69044671
:10870000E3B1987800B938BDB3F9042007EE902A98
:10871000F8EEE77A0120C4ED047AB3F9062007EEFB
:10872000902AF8EEE77AC4ED057AB3F9083007EE3F
:10873000903AF8EEE77AC4ED067A38BD09211420A4
:10874000FFF774FF0346E861DBE700BF38B5056853
:10875000EB690446E3B1987800B938BD9A88D2BA7B
:1087600007EE902AF8EEE77A0120C4ED047ADA8861
:10877000D2BA07EE902AF8EEE77AC4ED057A1B89A3
:10878000DBBA07EE903AF8EEE77AC4ED067A38BD28
:1087900009211420FFF74AFF0346E861DBE700BF29
:1087A00038B50468E3690D467BB1987800B938BDE7
:1087B0005B89094ADBBA82FB0312DB17C3EB221386
:1087C00003F26D132B80012038BD09211420FFF71F
:1087D0002DFF0346E061E8E7797878782DE9F041EC
:1087E00003EB4306964602EB460612F9067B86B07B
:1087F0000346754692F80080A3EB0804A3EB070C30
:10880000002CB8BF6442BCF1000FB8BFCCF1000C23
:108810006445B8BF154602F10602B8BF4FFA88F7A3
:10882000B242E7D16A889EF80000B842144614D1DB
:10883000BEF80200A1EB0008A1EB020CB8F1000F9A
:10884000B8BFC8F10008BCF1000FB8BFCCF1000CF4
:10885000E045BEBF7546024604460EF1060E76455B
:10886000E1D16A7904922A79CDE902422878054A51
:10887000CDE9001003210120FFF752FE284606B083
:10888000BDE8F081D81609084B1EDBB2062B9CBF51
:10889000214A02EB430330B598BF9D8B1F4BA3F1D8
:1088A000580488BF4FF48075002808BF1C46A446B2
:1088B00020893CF8082B87B04FFA82FE90B1A5EBD7
:1088C0000E022B1A002AB8BF5242002BB8BF5B42DF
:1088D0009A42C4BF64464FFA80FE3CF8080F002855
:1088E000EDD122880E4B0F4893F8E8CBA37905937E
:1088F000A38804930C4BBCF1000F18BF0346A0786B
:10890000CDE90015CDE902200321084A0120FFF737
:1089100007FE204607B030BDC06C0808B015002027
:10892000005F0020502C0908B41509081417090825
:1089300003685A1C02601878704700BF03681A4623
:10894000591C016012F8021B0260587841EA0020AD
:10895000704700BF10B402681346511C016013F841
:10896000021B0360D31C5478036093781B0443EA12
:108970000423141D0460D0785DF8044B0B4343EAD4
:108980000060704712B370B50446864604E0981B39
:1089900017D114EB0C0C15D01EF8013BA3F14100CC
:1089A000192811F8010BA0F1410598BF2033192DAA
:1089B000A2EB0E0C00F12006E9D91B1A04D1002805
:1089C000E7D170BD604670BD184670BD1046704757
:1089D00010B402888378174C02F0030101EB4101C7
:1089E000013B03EB810304EB4303C1789B8DA2F5AC
:1089F000FA62920840F2B55404FB02334A1E134453
:108A0000017942798479008903EB430301EBC301C7
:108A1000C1EB0111084B02EB8102C2EB02122344AD
:108A200003EB820300214FF47A72C3FB02015DF86D
:108A3000044B7047C06C080880436D38F8B5164683
:108A40001F460446394630464FF47A72002376F0CA
:108A500069FF3C4D3C4B054483FB05602844E91706
:108A6000C1EB601183FB01030B44384EC817C0EB08
:108A7000631086FB003CC317354EC3EBAC0386FB8B
:108A800003764FEAE37ECEEBE61EC1EB0116A5EBC3
:108A9000860CC0EB0015A1EB8501617103EB43016E
:108AA000A0EBC10040F2B55101FB1E33B3F5896F55
:108AB00084F806C020714FEA8E0636DA40F2DA21D9
:108AC0008B4238DCB3F5B77FB4BF4FF0000E4FF0E8
:108AD000010E20490EEB4E0001EBC0017546B1F8C6
:108AE00042004FEA4E071C4907EB0E0C01EBCC0C81
:108AF0000CF1160C0B2101E03CF8020D984211DD3F
:108B00000139F9D11349774401EBC701888D01215F
:108B1000013306F5FA6E1B1A7544A170E3702281C9
:108B20002580F8BD0131C9B2F2E7032540F2965025
:108B3000AE460627D7E7022540F22940AE46042775
:108B4000D1E700BF80BC92C789888888ABAAAA2ACF
:108B500073B06D16C06C0808EC6C080830B52F4C6B
:108B600086460D460FCC8DB0EC46ACE80F000FCC1E
:108B7000ACE80F0094E80F001EF0030F8CE80F0024
:108B80000FD1274B274A03FB0EF3B2EBB30F43D3AE
:108B9000254AB2EB331F34BF01220022C2F11D026D
:108BA00000E01C220EF1FF33002B019240F26D1207
:108BB000194602FB0EF2B8BF0EF1020102EBA10250
:108BC0001A491B4C81FB0301DB17A3EB6110024424
:108BD000C3EBE1131A44253284FB02311144D3174D
:108BE000C3EBA103C3EBC303D31AADF10402EE46FA
:108BF00002EB85015EF8040FC21884FB023C94442A
:108C0000D317C3EBAC03C3EBC3037145A2EB030360
:108C1000F0D1C01A0DB030BD1D22C3E74C6D08085D
:108C2000295C8FC2285C8F020AD7A3001F85EB51F5
:108C3000932449920D4B10B5D3F8F04BD3F8F43B85
:108C400054EA030209D1014640F201130020C1F8A1
:108C5000023088710880088110BD054A1268121917
:108C600043F10003FFF7EAFE012010BD005F002082
:108C7000242A002030B5144DD5F8F01BD5F8F43B6C
:108C800051EA030283B0044609D1002040F20113E7
:108C90002080C4F80230A071208103B030BD0B4A9F
:108CA0001268521843F10003FFF7C8FEB5F8F83B0D
:108CB000ADF8063020460DF1060221466EF0C2F9ED
:108CC000012003B030BD00BF005F0020242A002037
:108CD00088422DE9F0414FF001043DD301FB04F43B
:108CE000B0FBF4FC8C45F9D23CB3002616E0BCF195
:108CF000090F274698462C4623DD002A0CBF4FF06B
:108D0000570E4FF0370EF444B94288F800C003F113
:108D1000010306F1010610D8B0FBF5FCB4FBF1F538
:108D200004FB1C00002EE2D1BCF1000FDFDCA142ED
:108D30000AD90CF1300C03F801CB00221A70BDE8FF
:108D4000F0814FF0300EDEE7B0FBF5FC2C4605FB62
:108D50001C00B5FBF1F5E7E78446C6E72DE9F041D5
:108D6000044694421546084609D2B4FBF2F6154B68
:108D700005FB16441B5D00F8013BBDE8F081B4FB28
:108D8000F2F69642B6FBF2F70CD20E4B05FB1767D4
:108D900005FB1644DA5D00F8012B1B5D00F8013B72
:108DA000BDE8F081BA42B7FBF2F807D9054B05FBE5
:108DB000187813F8082000F8012BE7E74046FFF782
:108DC000CDFFF3E760170908B5EEC00ADFED347A8E
:108DD000F1EE10FACCBF30EE270A30EE670ADFED75
:108DE000317A20EE270A30B5FDEEC07A87B017EE53
:108DF000904A054684EAE470002303A9A0EBE470DE
:108E0000CDE9003302936EF077FC002CB4BF2D2324
:108E1000202303A88DF8003075F06AFF012829D0BF
:108E2000022833D003281DD003A968467DF056FCE4
:108E3000684675F05DFFC41EE4B2224669462846C6
:108E40007BF072FC00232B55284675F051FF2E2332
:108E50002B5401300DEB040128447DF0B4FC28466E
:108E600007B030BD302303A968468DF801307DF08E
:108E700035FCDDE743F23002302303A96846ADF844
:108E800001208DF803307DF029FCD1E743F2300357
:108E900003A96846ADF801307DF020FCC8E700BFAB
:108EA0006F12033A00007A440278202A034600F148
:108EB0000100F9D0092AF7D02D2A29D02B2A03BF87
:108EC0005A78B7EE000A0346B7EE000AA2F1300165
:108ED000C8B20928DFED4C7A10D8F2EE046A07EE2A
:108EE000101AB8EEC77A13F8012FA7EEA67AA2F1EE
:108EF0003001C8B20928F0EE477AF0D92E2A49D0BD
:108F0000197801F0DF01452907D020EE270A7047C4
:108F10005A78BFEE000A0346D8E710B459782D29D5
:108F200062D02B2954D0A1F13002092A03F10103A8
:108F300055D80024002202EB820201EB420213F812
:108F4000011FA1F130000928A2F13002F3D9B2F5D6
:108F50009A7F134628BF4FF49A73072A50D9DFED42
:108F60002B6A1A46B7EE007A083A072A27EE267AC5
:108F7000FAD803F007032BB1F2EE046A013B27EEA7
:108F8000267AFBD16CB3C7EE877A5DF8044B20EEEE
:108F9000270A70475978A1F13002D0B2092803F1AD
:108FA0000103AED8F2EE046AF0EE665A07EE102A1C
:108FB000B8EEC77A13F8011F87EE266AA1F13002D6
:108FC000D0B2092866EEA56A77EE867AEED998E7E0
:108FD0009978A1F13002092A03F10203A9D9B7EE69
:108FE000007A67EE877AD0E79978A1F13002092AF2
:108FF00003F1020388BFB7EE007AC4D8012499E7D1
:10900000B7EE007AB7E700BF0000000020BCBE4CFE
:109010000378202B024600F10100F9D0092BF7D08C
:109020002D2B08BF5378A3F13001CBB206BF024607
:109030004FF0FF3C4FF0010C092B4FF0000000D91E
:10904000704712F8013F00EB800001EB4000A3F1F4
:109050003001CBB2092BF4D90CFB00F0704700BFF4
:1090600070B5344D2B787E2B01D0002070BD0822C6
:109070004FF4FC4341F2210019B200294FEA4303A7
:10908000B6BF80EA41019BB28BB2013AF4D1B5F888
:10909000011069B32848294CA042E6D20638461888
:1090A000A642E2D241F2210C0529DED9864214D033
:1090B000013806F1FF3E10F8012F082183EA022350
:1090C0001AB2002A4FEA4303B6BF8CEA42029BB2AF
:1090D00093B20139F4D17045EDD1318849B1B21D57
:1090E000A242C2D27218A2423046BED21646DBE776
:1090F000134E741E41F22100A44614F8012F0821DA
:1091000083EA02231AB2002A4FEA4303B6BF80EA79
:1091100042029BB293B20139F4D16645ECD1728818
:10912000D01A084A331D5B1BB0FA80F04009A2F840
:10913000FC3B70BD00000E0807000E080000100880
:1091400001000E08005F00202DE9F04F914B924A7C
:109150008BB00020D21ACDE90600CDE90800D11865
:1091600005928E4A0393049110690028C0F2818110
:109170008A4AF320D0600020089089480122884262
:109180008DF8242000F271817E2007928DF818005E
:109190004FF4FC42082041F2210514B2002C4FEAA2
:1091A0004202B6BF85EA440492B2A2B20138F4D1B9
:1091B0007C48ADF802207C4A90427CD2804641F245
:1091C0002105B8F80200B8F80020C0F30B07C2F37D
:1091D0000B04120BBE1D4FF000098DF8082002048D
:1091E000ADF80460ADF806408DF8099000F1C38039
:1091F00006338B4200F2398101AE0DF10A0B344681
:1092000001E0A34513D0079B14F8011B03F12802CA
:109210006A440133042B079302F8101CF1D106A90C
:1092200003A8F9F723FCA345CDE90790EBD1089BF0
:10923000002BC0F21A81BDF8024016F8013B08224B
:1092400084EA032423B2002B4FEA4404B6BF85EA24
:109250004303A4B29CB2013AF4D1B345EDD1D8F89E
:1092600004603A46314603A8FEF74AF90028C0F2E6
:10927000FC80F019864213D0711E013811F8013FAD
:10928000082284EA032423B2002B4FEA4404B6BF29
:1092900085EA4303A4B29CB2013AF4D18142EDD1F4
:1092A000DDE90302ADF8024011463F4A08F1140817
:1092B0009045034685D302334FF000089942ADF83C
:1092C0000480C0F0D28001AD2E460DF106042F4679
:1092D00001E0BC4213D0079B17F8011B03F12802E1
:1092E0006A440133042B02F8101C0793F1D106A93C
:1092F00003A8F9F7BBFBBC42CDE90780EBD1089B83
:10930000002BC0F2B280BDF8023041F2210016F805
:10931000012B83EA0223082219B200294FEA4303F2
:10932000B6BF80EA41019BB28BB2013AF4D1B4429C
:10933000EDD10399ADF80230049B0231994200F25D
:1093400094800DF10206144602E0B54200F08A80D6
:10935000079B16F8011B03F128026A440133042B12
:1093600002F8101C0793F0D106A903A8F9F77EFBB9
:10937000CDE90740E9E7CB460BF1010B06335FFA75
:109380008BFB99428DF809B06FD301AE0DF10A0A3B
:1093900034460DE000000E0800001008003C0240BA
:1093A00001000E0800960908B49B0908A24515D0D3
:1093B000079914F801CB01F128030DEB03000131EB
:1093C0000429079100F810CCF0D106A903A8F9F7F9
:1093D0004DFB0023A24508900793E9D1089A002A83
:1093E00043DBBDF8024016F8012B082184EA022471
:1093F00022B2002A4FEA4404B6BF85EA4202A4B270
:1094000094B20139F4D1B245EDD1D8F8041001EB92
:1094100009063A46314603A8FEF772F8002824DB15
:10942000F019864213D0711E013811F8013F08224D
:1094300084EA032423B2002B4FEA4404B6BF85EA32
:109440004303A4B29CB2013AF4D18142EDD1DDE9EB
:109450000302BBF1030FADF8024003461146B944C5
:109460008AD121E7089B002B09DA00200BB0BDE868
:10947000F08F1548506000F18830506078E607980A
:1094800040B912490A6942F000420A61B3FA83F016
:109490004009EBE7DDE9033203449342E5D806AB2C
:1094A000C0F10402002118447CF060FA06A903A868
:1094B000F9F7DCFA002803460890D6DB9DF8242053
:1094C000002AE3D0DDE700BF23016745003C0240EE
:1094D00008B5FFF739FE40B9FFF736FE28B9FFF7A8
:1094E00033FE10B9052007F0ABF9FFF7B9FD0028EE
:1094F000F8D008BD70B545880B460446C5F30B058A
:109500002A46002118467CF031FA0A4A2169914224
:10951000034606D3084A914206D3BDE87040184678
:1095200008470029F9D170BD2A46BDE870407BF09C
:10953000FBB800BFB49B0908E3A0090810B5037984
:10954000012B84B08E460ED0022B02D0002004B036
:1095500010BD8368DB0758BF01F07F0104B0BDE890
:109560001040FDF7F7BF144682688DF80F4002F0F7
:10957000010201920DF10F020092417C90F910005E
:109580007246FAF725FF04B010BD00BFF8B5782287
:10959000074600210068FFF7D1FF052607F0F4F821
:1095A00004460D4607F0F0F8001B61EB0501B0F52D
:1095B0007A7F71F10001F5D3013EEFD138682022A6
:1095C0000121FFF7BBFF052607F0DEF804460D4634
:1095D00007F0DAF8001B61EB0501B0F57A7F71F155
:1095E0000001F5D3013EEFD1324638680221FFF782
:1095F000A5FF642607F0C8F804460D4607F0C4F836
:10960000001B61EB0501B0F57A7F71F10001F5D324
:10961000013EEFD10120F8BDF8B5072207460A2127
:109620000068FFF78BFF052607F0AEF804460D46ED
:1096300007F0AAF8001B61EB0501B0F57A7F71F124
:109640000001F5D3013EEFD1386824224121FFF714
:1096500075FF052607F098F804460D4607F094F8C4
:10966000001B61EB0501B0F57A7F71F10001F5D3C4
:10967000013EEFD13868C0224221FFF75FFF052687
:1096800007F082F804460D4607F07EF8001B61EBF8
:109690000501B0F57A7F71F10001F5D3013EEFD1FC
:1096A0000120F8BD10B50446002221210068FFF713
:1096B00045FF2068FC222021FFF740FF2068402260
:1096C0002421FFF73BFF20680C222321FFF736FF00
:1096D000206800222221FFF731FF012010BD00BFCA
:1096E000F8B50122074610210068FFF727FF00B9EF
:1096F000F8BD142607F048F804460D4607F044F874
:10970000001B61EB0501B0F57A7F71F10001F5D323
:10971000013EEFD13868A022BDE8F84011210DE7E5
:1097200010B5044600680379012B84B011D0022BD8
:1097300002D0002004B010BD01220B21FDF70AFF6A
:109740000028F6D020681D22092104B0BDE8104091
:10975000F4E6826890F910C0417C8DF80F3002F079
:10976000010201920DF10F02009260460B22FAF7FE
:109770002FFEE5E710B50446C06900B110BD092110
:109780001420FEF753FFE06110BD00BF10B5174C69
:1097900004EB8000406830B300EB400004EB800332
:1097A00093F901CCBCF1FF3F1ED093F8090CD0B166
:1097B00004EB0C0293F8080C92F854EC8C2314215F
:1097C00003FB0CFC00220CEB000304EB4303013908
:1097D000B3F8583C704412FA83F2F4D1044BA3FB63
:1097E0000230C0F30F1010BD002010BD005F00203C
:1097F000CDCCCCCC70B5104B104CA3421AD2054640
:1098000002E00C33A34215D293F805C08C45F8D181
:1098100093F804C0AC4501D0002DF2D1D879904224
:10982000EFD1186890F804E0E645EAD106689E4258
:10983000E7D170BD002070BDE4A00908A0A209080E
:109840000379022B00D0704710B490F910201C4807
:109850001C4C83B002EB82020831694400EB8202A7
:109860000094126A11F8084C17498A4224D0A1F5D5
:1098700078418A4222D001F580618A4218D111884C
:1098800021F04001090403EB8303090C118000EB74
:1098900083001388C16A23F0380331F824101B04B5
:1098A0001B0C0B43138013889BB243F040031380BF
:1098B00003B05DF8044B70470023E0E70123DEE7C7
:1098C000300C00200001020300300140F8B50468AC
:1098D000002107462046FFF7B3FFB6221421204699
:1098E000FFF72CFE642606F04FFF04460D4606F0F7
:1098F0004BFF001B61EB0501B0F57A7F71F10001B0
:10990000F5D3013EEFD1812210213868FFF716FE12
:1099100006F03AFF04460D4606F036FF001B61EBE9
:109920000501B0F57A7F71F10001F5D38022152190
:109930003868FFF703FE06F027FF04460D4606F0E1
:1099400023FF001B61EB0501B0F57A7F71F1000187
:10995000F5D338680321BDE8F84071E7F8B504682D
:10996000002107462046FFF76BFFB6227E212046E6
:10997000FFF7E4FD642606F007FF04460D4606F0F7
:1099800003FF001B61EB0501B0F57A7F71F1000167
:10999000F5D3013EEFD1324638687C21FFF7CEFD8A
:1099A000642606F0F1FE04460D4606F0EDFE001BAF
:1099B00061EB0501B0F57A7F71F10001F5D3013E4D
:1099C000EFD1386804227D21FFF7B8FD642606F048
:1099D000DBFE04460D4606F0D7FE001B61EB0501D9
:1099E000B0F57A7F71F10001F5D3013EEFD18C2201
:1099F00040213868FFF7A2FD06F0C6FE04460D467A
:109A000006F0C2FE001B61EB0501B0F57A7F71F133
:109A10000001F5D3022241213868FFF78FFD06F0DF
:109A2000B3FE04460D4606F0AFFE001B61EB0501D8
:109A3000B0F57A7F71F10001F5D338680221FFF7A4
:109A4000FFFE4FF40063BB81F8BD00BF2DE9F0417C
:109A5000076882B08046B6227E213846FFF76EFD49
:109A6000642606F091FE04460D4606F08DFE001BAE
:109A700061EB0501B0F57A7F71F10001F5D3013E8C
:109A8000EFD102213846FFF7DBFE7B6913B11A687C
:109A90009B88538306F078FE04460D4606F074FE5C
:109AA000001B61EB0501B0F57A7F71F10001F5D380
:109AB0007B6913B11A689B8813830A2606F064FE3B
:109AC00004460D4606F060FE001B61EB0501B0F593
:109AD0007A7F71F10001F5D3013EEFD132467C214E
:109AE0003846FFF72BFD06F04FFE04460D4606F004
:109AF0004BFE001B61EB0501B0F57A7F71F10001AF
:109B0000F5D3002259213846FFF718FD06F03CFE38
:109B100004460D4606F038FE001B61EB0501B0F56A
:109B20007A7F71F10001F5D397F910308D4A03EB7C
:109B3000830302EB8303BA681C6A5E2192078DF8E7
:109B4000071040F1E48001230DF1070200212046B7
:109B500074F082FF4FF4A473834A2046002174F00E
:109B60007BFFBB689B0740F1E5800A2606F00CFEF0
:109B700004460D4606F008FE001B61EB0501B0F53A
:109B80007A7F71F10001F5D3013EEFD10122592115
:109B90003846FFF7D3FC06F0F7FD04460D4606F005
:109BA000F3FD001B61EB0501B0F57A7F71F1000157
:109BB000F5D38C2240213846FFF7C0FC06F0E4FDC7
:109BC00004460D4606F0E0FD001B61EB0501B0F513
:109BD0007A7F71F10001F5D3032241213846FFF766
:109BE000ADFC06F0D1FD04460D4606F0CDFD001B90
:109BF00061EB0501B0F57A7F71F10001F5D35B4CA3
:109C0000D8F8382098F83500B4FBF2F2032391B26B
:109C1000574AFEF7E3FD4388B4FBF3F4C8F840402D
:109C20000279422142F0C0023846FFF787FC06F075
:109C3000ABFD04460D4606F0A7FD001B61EB0501D8
:109C4000B0F57A7F71F10001F5D30822432138463F
:109C5000FFF774FC06F098FD04460D4606F094FDEF
:109C6000001B61EB0501B0F57A7F71F10001F5D3BE
:109C7000042258213846FFF761FC06F085FD0446B2
:109C80000D4606F081FD001B61EB0501B0F57A7F02
:109C900071F10001F5D30A2253213846FFF74EFC3B
:109CA00006F072FD04460D4606F06EFD001B61EBEA
:109CB0000501B0F57A7F71F10001F5D300227C2116
:109CC0003846FFF73BFC06F05FFD04460D4606F004
:109CD0005BFD001B61EB0501B0F57A7F71F10001BE
:109CE000F5D306227D213846FFF728FC06F04CFD0F
:109CF00004460D4606F048FD001B61EB0501B0F57A
:109D00007A7F71F10001F5D302B0BDE8F0817B6983
:109D100013B11A689B885383164B17491A68174B5F
:109D20004868D200A3FB023292094B681B1A9A4280
:109D3000FBD208E70F4B10491A68104B48684FF4E4
:109D4000FA7404FB02F2A3FB023292094B681B1A5D
:109D50009A42FBD27B69002B3FF407AF1A689B88BD
:109D6000138302E7300C00207C6D080840420F008E
:109D7000C46E0808A4360020001000E0D34D621025
:109D80002DE9F041836B07685A4A5B4DB5FBF3F14F
:109D90000446062389B290F83500FEF71FFD002126
:109DA0004388B5FBF3F5804625643846FFF748FD48
:109DB00080226B213846FFF7C1FB642606F0E4FCE5
:109DC00004460D4606F0E0FC001B61EB0501B0F512
:109DD0007A7F71F10001F5D3013EEFD103226821B2
:109DE0003846FFF7ABFB642606F0CEFC04460D4672
:109DF00006F0CAFC001B61EB0501B0F57A7F71F13A
:109E00000001F5D3013EEFD101226B213846FFF767
:109E100095FB0F2606F0B8FC04460D4606F0B4FC90
:109E2000001B61EB0501B0F57A7F71F10001F5D3FC
:109E3000013EEFD118221B213846FFF77FFB0F268A
:109E400006F0A2FC04460D4606F09EFC001B61EBEA
:109E50000501B0F57A7F71F10001F5D3013EEFD134
:109E600018221C213846FFF769FB0F2606F08CFCF0
:109E700004460D4606F088FC001B61EB0501B0F5B9
:109E80007A7F71F10001F5D3013EEFD198F80420FB
:109E90001A213846FFF752FB0F2606F075FC0446E0
:109EA0000D4606F071FC001B61EB0501B0F57A7FF1
:109EB00071F10001F5D3013EEFD198F80520192189
:109EC0003846FFF73BFB642606F05EFC04460D4671
:109ED00006F05AFC001B61EB0501B0F57A7F71F1C9
:109EE0000001F5D3013EEFD138460321BDE8F04132
:109EF000A6E400BFD86E080840420F002DE9F041EB
:109F0000836B0768654A664DB5FBF3F1044606238B
:109F100089B290F83500FEF761FC00214388B5FB5B
:109F2000F3F5804625643846FFF78AFC80226B21D2
:109F30003846FFF703FB642606F026FC04460D4670
:109F400006F022FC001B61EB0501B0F57A7F71F190
:109F50000001F5D3013EEFD1072268213846FFF713
:109F6000EDFA642606F010FC04460D4606F00CFCE3
:109F7000001B61EB0501B0F57A7F71F10001F5D3AB
:109F8000013EEFD132466B213846FFF7D7FA6426FF
:109F900006F0FAFB04460D4606F0F6FB001B61EBEB
:109FA0000501B0F57A7F71F10001F5D3013EEFD1E3
:109FB00001226B213846FFF7C1FA0F2606F0E4FBB9
:109FC00004460D4606F0E0FB001B61EB0501B0F511
:109FD0007A7F71F10001F5D3013EEFD118221B21E8
:109FE0003846FFF7ABFA0F2606F0CEFB04460D46C7
:109FF00006F0CAFB001B61EB0501B0F57A7F71F139
:10A000000001F5D3013EEFD118221C213846FFF79D
:10A0100095FA0F2606F0B8FB04460D4606F0B4FB91
:10A02000001B61EB0501B0F57A7F71F10001F5D3FA
:10A03000013EEFD198F804201A213846FFF77EFA46
:10A040000F2606F0A1FB04460D4606F09DFB001B03
:10A0500061EB0501B0F57A7F71F10001F5D3013EA6
:10A06000EFD198F8052019213846FFF767FA6426E2
:10A0700006F08AFB04460D4606F086FB001B61EBEA
:10A080000501B0F57A7F71F10001F5D3013EEFD102
:10A0900038460321BDE8F041FFF7D2BBD86E08086F
:10A0A00040420F002AE700BFF0B5046883B00746BE
:10A0B00000212046FFF7C4FB0C2225212046FFF794
:10A0C0003DFA0A2226213868FFF738FA0022632178
:10A0D0003868FFF733FA386881222721FFF72EFA14
:10A0E000142606F051FB04460D4606F04DFB001BFE
:10A0F00061EB0501B0F57A7F71F10001F5D3013E06
:10A10000EFD10C2225213868FFF718FA0A22262100
:10A110003868FFF713FA0F2263213868FFF70EFA49
:10A12000386881222721FFF709FA0A2606F02CFB5E
:10A1300004460D4606F028FB001B61EB0501B0F557
:10A140007A7F71F10001F5D3013EEFD1032301AA1B
:10A15000102138466CF030F80A2606F015FB04464C
:10A160000D4606F011FB001B61EB0501B0F57A7F8F
:10A1700071F10001F5D3013EEFD19DF804009DF887
:10A1800005109DF806202C4B803080318032A3F8DA
:10A19000A00FA3F8A21FA3F8A42F25210C22386832
:10A1A000FFF7CCF90A2226213868FFF7C7F93246B3
:10A1B00063213868FFF7C2F9386881222721FFF749
:10A1C000BDF90A2606F0E0FA04460D4606F0DCFA70
:10A1D000001B61EB0501B0F57A7F71F10001F5D349
:10A1E000013EEFD10DF103020123022138466BF04D
:10A1F000E3FF01230DF10302092138466BF0DCFF78
:10A2000038680C222521FFF799F938680A2226219F
:10A21000FFF794F9386812226321FFF78FF9812242
:10A2200038682721FFF78AF938680321FFF708FB10
:10A23000012003B0F0BD00BF005F00202DE9F04118
:10A2400005461F4695F91030244803EB830300EBC5
:10A250008300AB68D0F8208016469A070ED540469A
:10A2600074F04AFC3B4632460021404674F0F4FB51
:10A27000AB689B0718D50120BDE8F0816B6913B16D
:10A280001A689B885383164B164A1B684FEAC30E05
:10A29000154BA2FB0E2E5A684FEA9E1E5C68A4EB7B
:10A2A000020CE645FAD2DAE70D4B0F491A680D4B5E
:10A2B0004FF4FA7000FB02F2A3FB023248689209E5
:10A2C0004B681B1A9A42FBD26B69002BD3D01A68D9
:10A2D0009B8813830120BDE8F08100BF300C002073
:10A2E000A4360020D34D6210001000E030B505798F
:10A2F000012D83B08E460DD0022D02D0002003B078
:10A3000030BD8468E40758BF41F0800103B0BDE868
:10A31000304093E714468268009402F00102417CC9
:10A3200090F9100001927246FAF752F803B030BD6E
:10A330002DE9F04105461F4695F91030244803EBFE
:10A34000830300EB8300AB68D0F8208016469A07A1
:10A350000ED5404674F0D0FB3B46002231464046C5
:10A3600074F07AFBAB689B0718D50120BDE8F0813B
:10A370006B6913B11A689B885383164B164A1B6886
:10A380004FEAC30E154BA2FB0E2E5A684FEA9E1ED3
:10A390005C68A4EB020CE645FAD2DAE70D4B0F49F4
:10A3A0001A680D4B4FF4FA7000FB02F2A3FB023265
:10A3B000486892094B681B1A9A42FBD26B69002BC2
:10A3C000D3D01A689B8813830120BDE8F08100BFB9
:10A3D000300C0020A4360020D34D6210001000E0A5
:10A3E00030B50579012D83B08E460DD0022D02D0F7
:10A3F000002003B030BD8468E40758BF41F08001FD
:10A4000003B0BDE8304093E714468268009402F040
:10A410000102417C90F9100001927246F9F7A4FF05
:10A4200003B030BD2DE9F043836B0768804A814C4F
:10A43000B4FBF3F185B08046062389B290F835006D
:10A44000FEF7CCF900214388B4FBF3F48146C8F849
:10A4500040403846FFF7F4F980226B213846FFF779
:10A460006DF8962606F090F904460D4606F08CF934
:10A47000001B61EB0501B0F57A7F71F10001F5D3A6
:10A48000013EEFD1032268213846FFF757F89626A0
:10A4900006F07AF904460D4606F076F9001B61EBEA
:10A4A0000501B0F57A7F71F10001F5D3013EEFD1DE
:10A4B00003226B213846FFF741F806F065F90446A0
:10A4C0000D4606F061F9001B61EB05010F2871F1E3
:10A4D0000001F6D310226A213846FFF72FF806F064
:10A4E00053F904460D4606F04FF9001B61EB0501D8
:10A4F0000F2871F10001F6D300226C213846FFF7D6
:10A500001DF806F041F904460D4606F03DF9001B22
:10A5100061EB05010F2871F10001F6D399F80520D0
:10A5200019213846FFF70AF806F02EF904460D46C1
:10A5300006F02AF9001B61EB05010F2871F10001FB
:10A54000F6D318221B213846FEF7F8FF06F01CF957
:10A5500004460D4606F018F9001B61EB05010F28B3
:10A5600071F10001F6D318221C213846FEF7E6FFF0
:10A5700006F00AF904460D4606F006F9001B61EBE9
:10A5800005010F2871F10001F6D399F804201A2172
:10A590003846FEF7D3FF06F0F7F805460C4606F0FE
:10A5A000F3F88C4208BF8542F9D003213846FFF703
:10A5B00047F9D8F800000623432102AAFFF710FF4D
:10A5C00028B3BDF80810BDF80A30BDF80C20C9BA90
:10A5D00007EE901ADBBAD2BAF8EEE76A07EE102A55
:10A5E00007EE903AB8EEC77AF8EEE77AC8ED076A58
:10A5F000C8ED087A88ED097AFDEEE77ACDED017AAB
:10A600009DF90430013305D005B0BDE8F083D8EDE5
:10A61000087AF1E7D8ED077AFDEEE77ACDED017A19
:10A620009DF904300133EFD1062006F009F900BF8F
:10A63000D86E080840420F0010B504460068037940
:10A6400082B0022B0CBF4321032106236A46FFF789
:10A65000C7FE68B1BDF80010BDF80220BDF8043097
:10A6600049BA52BA5BBAE1866287238702B010BD4D
:10A67000C4F83600608702B010BD00BF2DE9F04776
:10A68000164F97F8A93F824689466BB9DAF8000061
:10A6900097F8AA3F00244A46492187F8A94FFFF7B7
:10A6A0009FFE0120BDE8F08706F06EF8D7F8B03FB6
:10A6B000C51AC5F5FA55002DE8DD06F065F84FEA34
:10A6C000E57804460E4606F05FF8001B61EB0601D4
:10A6D000A84271EB0801F6D3D8E700BF005F002065
:10A6E0002DE9F041624C0546D4F8B80FC5F83600A4
:10A6F00094F8A83FB4F8BC2F6A87012B82B076D0BB
:10A70000022B0FD0002B69D10122022128466DF0C7
:10A7100021F9012394F8BE6F84F8A83F304602B0B7
:10A72000BDE8F08194F8A93F05F1360804F6B87742
:10A73000002B6ED169462846FFF7A0FF9DF8063032
:10A74000064600284AD01B0748D4B4F8A02FBDF80D
:10A75000003013FB02F3474A93427DDBB3F5000F51
:10A760006FDA002BB8BFFF331B125B421BB2B4F889
:10A77000A22FEB86BDF8023013FB02F33D4A934251
:10A780006EDBB3F5000F6FDA002BB8BFFF3343F376
:10A790000F23B4F8A42F2B87BDF8043013FB02F36A
:10A7A000344A93425ADBB3F5000F5BDA002BB8BF93
:10A7B000FF331B125B421BB2D5F83600C4F8B80F4A
:10A7C0006B87B8F80430BB8000220123304684F840
:10A7D000A82F84F8BE3F02B0BDE8F08100263046C5
:10A7E00084F8A86F84F8BE6F02B0BDE8F08194F8D9
:10A7F000A93F94F8BE6FD3B969462846FFF73EFFDC
:10A800009DF8003008B19A071DD1002384F8A83FB5
:10A8100084E705F0B9FFD4F8B03FC01AB0F5FA5F8D
:10A8200088DA94F8BE6F304602B0BDE8F08105F0DA
:10A83000ABFFD4F8B03FC01AB0F5FA5FFFF66EAFC9
:10A84000DAE70D4B93E70722032128466DF082F8E3
:10A85000022384F8A83F61E7084B88E7074BABE782
:10A86000064B96E7044BA7E747F6FF7391E700BF57
:10A87000005F002001FF7FFF0180FFFF0080FFFFDE
:10A8800010B5044600680179012984B02AD0022954
:10A8900002D0002004B010BD836813F0010F02AA9B
:10A8A0004FF0060308BF8221FFF742FD0028F0D0D9
:10A8B000BDF9083006EE903ABDF90A3007EE103ABD
:10A8C000BDF90C3007EE903AF8EEE66AB8EEC77ABA
:10A8D000F8EEE77AC4ED076A84ED087AC4ED097AE8
:10A8E00004B010BD8368417C90F9100003F00103AF
:10A8F000019302AB009302220623F9F735FDD5E759
:10A9000030B5044600680379012B85B014D0022BC2
:10A910000FD1826802AD12F0010F18BF03212A4641
:10A9200008BF8321FFF704FD18B19DF90930002B02
:10A9300010DB002005B030BD8368417C90F9100029
:10A9400003F0010302AD0193009502230322F9F7FE
:10A950000BFDE9E7206807232A461221FFF740FD97
:10A960000028E6D09DF90A209DF809309DF90C10C9
:10A9700043EA022313EB430248BF03329DF80B3036
:10A98000921043EA012307EE902A13EB4302F8EEFC
:10A99000E77A48BF03329DF90E109DF80D30C4EDE3
:10A9A000047A921007EE902A43EA012313EB430343
:10A9B000F8EEE77A48BF03339B10C4ED057A07EE43
:10A9C000903AF8EEE77AC4ED067AB3E770B5066818
:10A9D000F46982B00546002C3FD03379012B04F195
:10A9E00004022DD0022B26D1B36813F0010F4FF0D3
:10A9F0000C03304614BF19468C21FFF799FCA07058
:10AA0000D8B1B4F9043007EE903AF8EEE77AC5ED24
:10AA1000077AB4F9063007EE903AF8EEE77AC5ED1A
:10AA2000087AB4F9083007EE903AF8EEE77AC5ED07
:10AA3000097A02B070BD0023A370002002B070BD7F
:10AA4000B368717C96F91000009203F00103019342
:10AA50000C231A46F9F788FCD1E709211420FDF7E9
:10AA6000E5FDF06104462E68B7E700BF70B50668E3
:10AA7000F46982B00546002C3FD03379012B04F1F4
:10AA800003022DD0022B26D1B36813F0010F3046FC
:10AA90004FF00D0314BF0C218C21FFF749FCA0706F
:10AAA000D8B1B4F90A3007EE903AF8EEE77AC5ED7E
:10AAB000077AB4F90C3007EE903AF8EEE77AC5ED74
:10AAC000087AB4F90E3007EE903AF8EEE77AC5ED61
:10AAD000097A02B070BD0023A370002002B070BDDF
:10AAE000B368717C96F91000009203F001030193A2
:10AAF0000C220D23F9F738FCD1E709211420FDF7CA
:10AB000095FDF06104462E68B7E700BF10B50068F8
:10AB10000379012B84B00C461AD0022B02D00020FE
:10AB200004B010BD836813F0010F03AA4FF00303B4
:10AB300014BF2221A221FFF7FBFB0028EFD0BDF9B3
:10AB40000D3003EB83031B12E633238004B010BDEA
:10AB50008368417C90F9100003F00103019303AB7B
:10AB6000009322220323F9F7FFFBE6E710B5044622
:10AB700000680379012B84B02DD0022B01D0002076
:10AB800027E0836813F0010F02AA4FF0060314BFF9
:10AB90001F219F21FFF7CCFB0028F0D0BDF8081043
:10ABA000BDF80A20BDF80C30C9BA07EE901AD2BA27
:10ABB000F8EEE76A07EE902ADBBAB8EEE77A07EE1E
:10ABC000903AF8EEE77AC4ED046A84ED057AC4EDB4
:10ABD000067A04B010BD8368417C90F9100003F040
:10ABE0000103019302AB00931F220623F9F7BCFB7C
:10ABF000D2E700BF10B5044600680379012B84B08A
:10AC00002DD0022B01D0002027E0836813F0010F24
:10AC100002AA4FF0060314BF2521A521FFF788FBE8
:10AC20000028F0D0BDF80810BDF80A20BDF80C309F
:10AC3000C9BA07EE901AD2BAF8EEE76A07EE902A80
:10AC4000DBBAB8EEE77A07EE903AF8EEE77AC4EDB1
:10AC5000076A84ED087AC4ED097A04B010BD8368F0
:10AC6000417C90F9100003F00103019302AB0093C3
:10AC700025220623F9F778FBD2E700BF10B500685C
:10AC80000379012B84B00C4625D0022B01D0002083
:10AC90001FE0826812F0010F18BF1D2103AA08BF30
:10ACA0009D21FFF745FB0028F1D0BDF80C309FED4A
:10ACB000116ADFED116ADBBA07EE903AB8EEE77A77
:10ACC000C7EE067A77EEA67AFDEEE77A17EE903AAF
:10ACD000238004B010BD8368417C90F9100003F01C
:10ACE0000103019303AB00931D220223F9F73CFB00
:10ACF000D9E700BFCFF7534100007A4370B506682B
:10AD0000F46982B00546002C3FD03379012B04F161
:10AD100004022DD0022B26D1B36813F0010F304668
:10AD20004FF00E0314BF3B21BB21FFF701FBA070C6
:10AD3000D8B1A389DBBA07EE903AF8EEE77AC5ED11
:10AD4000077AE389DBBA07EE903AF8EEE77AC5EDC9
:10AD5000087A238ADBBA07EE903AF8EEE77AC5ED77
:10AD6000097A02B070BD0023A370002002B070BD4C
:10AD7000B368717C96F91000009203F0010301930F
:10AD80003B220E23F9F7F0FAD1E709211420FDF751
:10AD90004DFC0446F061B8E700B500680379012B6B
:10ADA00085B011D0022B01D000200AE003AAF621C1
:10ADB000FFF7BEFA0028F7D0BDF80C30094A5BBA9D
:10ADC000938205B05DF804FB8368417C90F9100024
:10ADD00003AA03F00103CDE900230223F622F9F7C9
:10ADE000C3FAE7E7005F002000B500680379012B94
:10ADF00085B01ED0022B01D0002017E0032303AA48
:10AE0000F621FFF795FA0028F6D09DF80D309DF851
:10AE10000CC00F499DF80E201B0243EA0C4313435C
:10AE2000B1F93420C2F10802D3408B6305B05DF85C
:10AE300004FB8368417C90F9100003AA03F001032E
:10AE4000CDE900230323F622F9F78EFADBE700BFF2
:10AE5000005F002000B500680379012B85B033D076
:10AE6000022B0AD01F49D1F8C03FD1F8C42FCA63C2
:10AE70000020CB6505B05DF804FB062302AAF7218C
:10AE8000FFF756FA0028EDD09DF809309DF808C06C
:10AE90009DF80C209DF80A109DF80BE01B0143EA79
:10AEA0000C3312019DF80DC043EA111342EA0E3231
:10AEB0000C4942EA1C12C1F8C03FC1F8C42FCA6352
:10AEC000CB6505B05DF804FB8368417C90F9100008
:10AED00002AA03F00103CDE900230623F722F9F7C4
:10AEE00043FACFE7005F002000B500680379012B2B
:10AEF00085B01ED0022B10D09DF80D309DF80C00AF
:10AF00009DF80E10124A1B0243EA00430B43012036
:10AF1000C2F8843005B05DF804FB836813F0010FBC
:10AF200003AA4FF0030314BF00218021FFF700FAAA
:10AF3000E2E78368417C90F9100003AA03F0010363
:10AF4000CDE9002303230022F9F70EFAD4E700BF6E
:10AF5000005F002000B500680379012B85B01ED08A
:10AF6000022B10D09DF80D309DF80C009DF80E10AE
:10AF7000124A1B0243EA00430B430120C2F89830F7
:10AF800005B05DF804FB836813F0010F03AA4FF0CE
:10AF9000030314BF00218021FFF7CAF9E2E78368A9
:10AFA000417C90F9100003AA03F00103CDE90023CE
:10AFB00003230022F9F7D8F9D4E700BF005F00208F
:10AFC00010B500680379012B84B029D0022B01D081
:10AFD000002023E0836813F0010F4FF0030303AA5E
:10AFE00014BF19468321FFF7A3F90028F0D09DF87C
:10AFF0000C309DF90C109DF80D209DF80EC01B041F
:10B00000002943EA0223A8BF00210C4AB8BF4FF031
:10B010007F4143EA0C030B43C2F8CC3004B010BDAF
:10B020008268417C90F9100002F0010203AC032316
:10B03000CDE900421A46F9F797F9D6E7005F0020FC
:10B0400000B500680379012B85B02AD0022B01D00E
:10B05000002023E0836813F0010F03AA4FF00303DD
:10B0600014BF00218021FFF763F90028F0D09DF87C
:10B070000C309DF90C109DF80D209DF80EC01B049E
:10B08000002943EA0223A8BF00210D4AB8BF4FF0B0
:10B090007F4143EA0C030B43C2F8C83005B05DF8AA
:10B0A00004FB8368417C90F9100003AA03F00103BC
:10B0B000CDE9002303230022F9F756F9D5E700BFB5
:10B0C000005F002010B5044600230068C4F8363045
:10B0D00063870379012B84B022D0022B01D000209A
:10B0E0001CE0836813F0010F02AA4FF0060314BF9F
:10B0F00003218321FFF71CF90028F0D0BDF90A30A5
:10B10000BDF80810BDF80C205B4201EB410103EBD8
:10B11000430302EB4202E1862387628704B010BD3D
:10B120008368417C90F9100003F00103019302ABA6
:10B13000009303220623F9F717F9DDE770B50446FB
:10B14000234894F9103003EB830300EB8300A368DA
:10B15000066A15469A070DD5304673F0CDFC0123DB
:10B1600000222946304673F077FCA3689B0716D56A
:10B17000012070BD636913B11A689B885383154B16
:10B18000154A1B6850684FEAC30C144BA3FB0C3CD8
:10B190004FEA9C1C53681B1A9C45FBD2DCE70D4B05
:10B1A0000D491A680D4B4FF4FA7000FB02F2A3FB35
:10B1B0000232486892094B681B1A9A42FBD26369B3
:10B1C000002BD5D01A689B881383012070BD00BF67
:10B1D000300C0020A4360020001000E0D34D621097
:10B1E00010B50379012B82B08E460DD0022B02D010
:10B1F000002002B010BD8368DB0758BF41F080011A
:10B2000002B0BDE8104099E714468268009402F04D
:10B210000102417C90F9100001927246F9F7A4F8FE
:10B2200002B010BD70B505682B79012B84B00446BF
:10B230000E4616D0022B02D0002004B070BDAB68C1
:10B24000E122DB074CBF114661212846FCF782F959
:10B250000028F1D020683246FF2104B0BDE87040DC
:10B26000BEE7AA68697C95F9100002F001020DF1B1
:10B270000F0501920095E1228DF80F20F9F7A8F84B
:10B28000E6E700BF70B505682B79012B84B0044652
:10B290000E4617D0022B02D0002004B070BDAB6860
:10B2A000DB074FF0C3024CBFE12161212846FCF7C8
:10B2B00051F90028F0D020683246FF2104B0BDE8E3
:10B2C00070408DE7AA6895F91000697C02F00102D0
:10B2D00001920DF10F020092C3228DF80F20E1229E
:10B2E000F9F776F8E5E700BF70B505682B79012B13
:10B2F00084B004460E461CD0022B02D0002004B0BD
:10B3000070BDAB68DB074FF0F0024CBFE12161215B
:10B310002846FCF71FF90028F0D02246FF2152F8FA
:10B32000040BFFF75DFF0028E8D02379337004B0E9
:10B3300070BDAA6895F91000697C02F001020192C3
:10B340000DF10F020092F0228DF80F20E122F9F7A3
:10B350003FF8E0E7F0B5046883B0002107462046D7
:10B36000FEF76EFA15227E212046FEF7E7F86426E6
:10B3700005F00AFA04460D4605F006FA001B61EBDB
:10B380000501B0F57A7F71F10001F5D3013EEFD1EF
:10B39000386811227E21FEF7D1F8052605F0F4F970
:10B3A00004460D4605F0F0F9001B61EB0501B0F510
:10B3B0007A7F71F10001F5D3013EEFD138680DF1CC
:10B3C00007020321FFF70CFF9DF8073003F03C0351
:10B3D000142B40F09B800C2240213868FEF7AEF819
:10B3E00005F0D2F904460D4605F0CEF9001B61EBDD
:10B3F0000501B0F57A7F71F10001F5D3BB6B454CC7
:10B40000454AB4FBF3F197F83500092389B2FDF7FB
:10B41000E5F9034642215A88B4FBF2F43C641A79F8
:10B420003868FEF78BF805F0AFF904460D4605F0D5
:10B43000ABF9001B61EB0501B0F57A7F71F10001FA
:10B44000F5D3082241213868FEF778F805F09CF919
:10B4500004460D4605F098F9001B61EB0501B0F5B7
:10B460007A7F71F10001F5D3002243213868FEF79D
:10B4700065F805F089F904460D4605F085F9001BCD
:10B4800061EB0501B0F57A7F71F10001F5D310226F
:10B4900051213868FEF752F805F076F904460D465A
:10B4A00005F072F9001B61EB0501B0F57A7F71F1CF
:10B4B0000001F5D30A2253213868FEF73FF805F062
:10B4C00063F904460D4605F05FF9001B61EB0501C9
:10B4D000B0F57A7F71F10001F5D3802256213868EA
:10B4E000FEF72CF805F050F904460D4605F04CF92E
:10B4F000001B61EB0501B0F57A7F71F10001F5D316
:10B5000038680321FEF79CF903B0F0BD062005F072
:10B5100097F900BF40420F00FC6E08082DE9F04388
:10B52000836B0768A04AA14CB4FBF3F183B080465B
:10B53000052389B290F83500FDF750F900214388C2
:10B54000B4FBF3F48146C8F840403846FEF778F97A
:10B55000002276213846FDF7F1FF0F224E213846B2
:10B56000FDF7ECFF0F2605F00FF904460D4605F038
:10B570000BF9001B61EB0501B0F57A7F71F1000159
:10B58000F5D3013EEFD199F805204F2102F00F02CB
:10B590003846FDF7D3FF0F2605F0F6F804460D46B2
:10B5A00005F0F2F8001B61EB0501B0F57A7F71F14F
:10B5B0000001F5D3013EEFD199F80520502102F0AA
:10B5C0000F023846FDF7BAFF0F2605F0DDF80446F6
:10B5D0000D4605F0D9F8001B61EB0501B0F57A7F47
:10B5E00071F10001F5D3013EEFD1FF22522138461F
:10B5F000FDF7A4FF0F2605F0C7F804460D4605F039
:10B60000C3F8001B61EB0501B0F57A7F71F1000111
:10B61000F5D3013EEFD198F83510072941D0644D9C
:10B6200095F8E80BFDF730F90446012276213846FB
:10B63000FDF784FFA2780C213846FDF77FFF2279C1
:10B640000D213846FDF77AFFA279A388120142EA5C
:10B650001322D2B20E213846FDF770FF4FF48071ED
:10B6600095F8E80BFDF710F90446022276213846DA
:10B67000FDF764FFA2785200032102F0FE02384673
:10B68000FDF75CFF227904213846FDF757FFA279C8
:10B69000A388120142EA13220521D2B23846FDF7EF
:10B6A0004DFF002276213846FDF748FF0322142182
:10B6B0003846FDF743FF0F2605F066F804460D46B1
:10B6C00005F062F8001B61EB0501B0F57A7F71F1BE
:10B6D0000001F5D3013EEFD1324663213846FDF734
:10B6E0002DFF642605F050F804460D4605F04CF891
:10B6F000001B61EB0501B0F57A7F71F10001F5D314
:10B70000013EEFD1082265213846FDF717FF64217D
:10B710000DF107023846FFF763FD9DF8072022F080
:10B72000100242F06002642138468DF80720FDF7D0
:10B7300005FF0F2605F028F804460D4605F024F80D
:10B74000001B61EB0501B0F57A7F71F10001F5D3C3
:10B75000013EEFD10DF106024D213846FFF740FDC5
:10B760009DF8062002F03F0242F040024D2138468B
:10B770008DF80620FDF7E2FE0F2605F005F80446D9
:10B780000D4605F001F8001B61EB0501B0F57A7F6D
:10B7900071F10001F5D3013EEFD103213846FEF7E8
:10B7A0004FF803B0BDE8F083346F080840420F0043
:10B7B000005F0020F0B583B015460DF107021C466E
:10B7C00006460F46FFF70CFD9DF8072005EA020329
:10B7D000A34201D103B0F0BD22EA0502224339465B
:10B7E000304603B0BDE8F040FDF7A8BE10B582B00A
:10B7F00004466A4600680821FFF7F2FC9DF8003015
:10B80000DB0602D4002002B010BD206806236A4681
:10B810000021FEF7E5FD0028F4D09DF801309DF8E9
:10B8200000109DF802209FED4A6A1B0203EB0143C2
:10B830009DF804101C029DF803401A444FEA0121B0
:10B840009DF8053001EB044148BF02F17F420B44F3
:10B8500007EE902A090248BF03F17F43B8EEE77A6A
:10B8600007EE903AF8EEE77AC7EE066A394BB3F97D
:10B870006C20B3F9721093F8C84F112CC7EE863ABA
:10B8800007EE102A93ED1A6AB3F96E20D3ED197AF8
:10B89000F8EEC65A06EE102AB3F9702005EE102A0B
:10B8A000B3F9742004EE901A04EE102AB8EEC77AA9
:10B8B000F8EEE77AB8EEC66AB8EEC55AF8EEE44A92
:10B8C000B3F97610B3F97820B8EEC44A27EE237A9C
:10B8D00026EEA32A23D0A6EE845AA6EEA46AE5EEAD
:10B8E000265AE5EEA67A77EE877AE6EE027AB3F983
:10B8F000622007EE102AB3F96020C3ED1F7A06EE2E
:10B90000902AB8EEC77AF8EEE66A27EE237AB6EE0A
:10B91000006AA6EE867A83ED207A02B010BD03EEAF
:10B92000102AF8EEC32A03EE101AA6EEA24AB8EEC9
:10B93000C33AA4EE265AE6EE834AE5EE265AA4EE72
:10B94000A66AE5EEA67A77EE877AE6EE027ACEE789
:10B9500000007848005F0020F0B5044683B00D4633
:10B960001746061D20680379012B1AD0022B02D03E
:10B97000002003B0F0BD8368DB0732464FF0FF01C3
:10B980005CBF3246FF21FFF7D9FB0028F0D015B18C
:10B990002379DB07E6D4002FEBD023793B7003B08B
:10B9A000F0BD8268417C90F9100002F00102CDE9FF
:10B9B0000062FF22F8F7D8FCE7E700BF30B5044685
:10B9C000051D20680379012B83B017D0022B02D00C
:10B9D000002003B030BD8368DB072A464FF0FF012B
:10B9E0005CBF2A46FF21FFF7A9FB0028F0D023798E
:10B9F000DB07EED520680379012BE7D18268417C13
:10BA000090F9100002F00102CDE90052FF22F8F790
:10BA1000ABFCEAE730B50246044652F8040B037962
:10BA2000012B83B00ED0022B01D0002008E0FF21B3
:10BA3000FFF784FB0028F8D02079C04300F0010014
:10BA400003B030BD8568417C90F91000009205F08C
:10BA500001050195FF22F8F787FCEBE730B5B4222A
:10BA600083B00446FF210068FDF768FD10B900208F
:10BA700003B030BD20680379012B04F1040514D014
:10BA8000022BF4D18368DB072A464FF0FF015CBF2D
:10BA90002A46FF21FFF752FB0028E8D02379DB0775
:10BAA000E6D520680379012BEAD18268417C90F9C0
:10BAB000100002F00102CDE90052FF22F8F754FC19
:10BAC000EAE700BF30B50A4683B00446A521006806
:10BAD000FDF734FD10B9002003B030BD20680379B4
:10BAE000012B04F1040514D0022BF4D18368DB0789
:10BAF0002A464FF0FF015CBF2A46FF21FFF71EFBDD
:10BB00000028E8D02379DB07E6D520680379012BEC
:10BB1000EAD18268417C90F9100002F00102CDE97F
:10BB20000052FF22F8F720FCEAE700BF70B582B0B0
:10BB3000CDE900230446FFF791FF10B9002002B0C1
:10BB400070BD20685522A521FDF7F8FC0028F5D02E
:10BB5000251D20682A46FF21FFF742FB0028EDD073
:10BB60002379DB07F5D40DF1FF350DF1070615F844
:10BB7000011F2046FFF7A6FF0028DFD0B542F6D10F
:10BB8000DDE700BF002A35D0F0B5044683B00E468D
:10BB90008F18051D16F8012B2068A521FDF7CEFC96
:10BBA00090B9002003B0F0BD8268417C90F910008C
:10BBB00002F00102CDE90052FF22F8F7D5FB002880
:10BBC000EFD02379DB0710D520680379012BEBD068
:10BBD000022BE6D18368DB072A464FF0FF015CBFEA
:10BBE0002A46FF21FFF7AAFAE9E7B742D2D101209E
:10BBF00003B0F0BD0120704770B5962282B00446B4
:10BC00000E460068FF21FDF799FC10B9002002B034
:10BC100070BD251D20680379012B1FD0022BF5D1A3
:10BC20008368DB072A464FF0FF015CBF2A46FF21ED
:10BC3000FFF784FA0028E9D02379DB07EAD4E12270
:10BC400020681146FDF77AFC0028DFD020683246D4
:10BC5000FF2102B0BDE87040FFF7C2BA8268417CA4
:10BC600090F9100002F00102CDE90052FF22F8F72E
:10BC70007BFBDFE7002A43D0F0B5044683B00E46D5
:10BC80008F18051D20689622FF21FDF757FC90B9FB
:10BC9000002003B0F0BD8268417C90F9100002F0F2
:10BCA0000102CDE90052FF22F8F75EFB0028EFD039
:10BCB0002379DB0710D520680379012BEBD0022B09
:10BCC000E6D18368DB072A464FF0FF015CBF2A46B6
:10BCD000FF21FFF733FAE9E7E12220681146FDF77B
:10BCE0002DFC0028D4D020683246FF21FFF778FAD7
:10BCF0000028CDD00136B742C4D1012003B0F0BD39
:10BD00000120704770B505460B460446164655F8A7
:10BD1000040B82B087211A46FDF710FC20680379D6
:10BD2000012B1AD0022B02D0002002B070BD836814
:10BD3000DB072A464FF0FF015CBF2A46FF21FFF7D1
:10BD4000FDF90028F0D02379DA07E7D4002EECD0F3
:10BD5000C3F34013337002B070BD8268417C90F928
:10BD6000100002F00102CDE90052FF22F8F7FCFAC0
:10BD7000E7E700BF70B5782182B004461646006838
:10BD80000022FDF7DBFB10B9002002B070BD251DBD
:10BD900020680379012B14D0022BF5D18368DB07CF
:10BDA0002A464FF0FF015CBF2A46FF21FFF7C6F984
:10BDB0000028E9D02379DA07EAD45B09337002B0AE
:10BDC00070BD8268417C90F9100002F00102CDE95B
:10BDD0000052FF22F8F7C8FAEAE700BF30B5CC22DC
:10BDE00083B00446A5210068FDF7A8FB10B9002028
:10BDF00003B030BD20680379012B04F1040514D091
:10BE0000022BF4D18368DB072A464FF0FF015CBFA9
:10BE10002A46FF21FFF792F90028E8D02379DB07B3
:10BE2000E6D520680379012BEAD18268417C90F93C
:10BE3000100002F00102CDE90052FF22F8F794FA57
:10BE4000EAE700BF30B5B42283B00446FF210068A2
:10BE5000FDF774FB10B9002003B030BD251D20682C
:10BE60000379012B22D0022BF5D18368DB072A4608
:10BE70004FF0FF015CBF2A46FF21FFF75FF9002862
:10BE8000E9D02379DA07EAD4CC212046FFF71AFE5D
:10BE90000028E0D002E02379DB07DDD520682A46C0
:10BEA000FF21FFF79DF90028F5D1D4E78268417C96
:10BEB00090F9100002F00102CDE90052FF22F8F7DC
:10BEC00053FADCE72DE9F04F8BB0CDE907230446A8
:10BED000002004908A460390251D049B079A204663
:10BEE000DE0002EBC30BFFF7B9FD20B935E0237983
:10BEF00013F0010207D020682A46FF21FFF770F9EE
:10BF00000028F4D129E005929A07099040F1D880E1
:10BF1000F0212046FFF7D6FDF8B1079BDDF814802D
:10BF2000083E3344012606933746BAF1000F54D039
:10BF3000082F52D807F1FF394AFA09F909F0010927
:10BF400020684FEAC9127821FDF7F8FA28B1206875
:10BF50000379012B50D0022B06D00020089B049AB5
:10BF60001A700BB0BDE8F08F8368DB072A464FF0EC
:10BF7000FF015CBF2A46FF21FFF7E0F80028ECD064
:10BF8000237913F00102E2D1C3F3801CD9099B0687
:10BF900046D5BCF1000F60D1BAF1000F5AD0082F7E
:10BFA00058D8894540F08880B9F1000F48D01BF877
:10BFB000083033430BF808307600013716F0FF06DF
:10BFC000FFB2B2D108F101085FFA88F8B8F1080FA2
:10BFD00043D00126BAF1000FAAD1049BC3B1039B41
:10BFE000BB4215D9069B13F808301E4214BF4FF010
:10BFF00001094FF00009A3E78268417C90F9100025
:10C0000002F00102CDE90052FF22F8F7ADF9B5E7E1
:10C01000039BA3EB0709B9FA89F94FEA59198FE78E
:10C02000BAF1000F13D0082F11D8894596D1B9F174
:10C03000000FBCD1059BBCF1000F08BF3B46059328
:10C040001BF8083023EA06030BF80830B4E7002990
:10C05000ADD1EFE70029AAD1F2E7402F06D8089B1F
:10C06000049A1B7893423FF638AF77E79BF8077046
:10C070000BF1FF360BF1060B16F801CF082182EA0F
:10C080000C0343F30003013923F0730383EA5202E4
:10C0900011F0FF01D2B24FEA5C0CF0D1B345EBD105
:10C0A0009742DCD1049B0133DBB20493059B002B48
:10C0B0003FF454AF0393D2E7DDF8248040464DE7C8
:10C0C000804640464AE700BF10B5044686B0006887
:10C0D00000238DF80F300379012B31D0022B02D0D1
:10C0E000002006B010BD8368D9070DF10F024CBFC8
:10C0F0002721A721FFF722F80028F1D09DF80F3063
:10C100001B07EDD52068062304AA2821FEF768F94D
:10C1100028B3BDF91030BDF91220002BB8BF03338E
:10C120009B10E386BDF91430002AB8BF0332002B00
:10C13000B8BF033392109B102287638706B010BDEF
:10C14000826890F910C0417C02F0010201920DF169
:10C150000F02009260462722F8F706F9CCE7C4F8F0
:10C16000360060870020BCE730B504464FF0000C75
:10C170000068C4F836C0A4F83AC00379012B87B030
:10C180002AD0022B02D0002007B030BD8368D90727
:10C190000DF10F024CBF61468021FEF7CFFF002852
:10C1A000F1D09DF80F301B07EDD52068062304AAB7
:10C1B0000121FEF715F90028E5D0BDF81430BDF8CF
:10C1C0001010BDF812205BBA49BA52BA5B42E18640
:10C1D0002287638707B030BD8568417C90F91000E5
:10C1E00005F0010501950DF10F0562460095F8F780
:10C1F000BBF8D4E710B5044600230068C4F8363015
:10C2000063870379012B86B023D0022B02D0002054
:10C2100006B010BD8368D9070DF10F024CBF06218F
:10C220008621FEF78BFF0028F1D09DF80F30DB0749
:10C23000EDD52068062304AA0021FEF7D1F80028D6
:10C24000E5D0049ABDF81430C4F83620638706B0F0
:10C2500010BD826890F910C0417C02F00102019289
:10C260000DF10F02009260460622F8F77DF8DAE73A
:10C2700010B50368DA6B82B0044612B1904740B142
:10C2800023685B6B1BB1214601A8984718B9FF23AF
:10C29000E38202B010BDBDF80630013B9BB2F7E768
:10C2A000F0B5044683B018460D4616461F4672F098
:10C2B0001FFD2844D4F800C0A073E6732046002474
:10C2C0000094DCF814403B4632462946A04703B0B0
:10C2D000F0BD00BF38B58B68016004460D46984735
:10C2E00000230B4A226123752B6B13B1204698471C
:10C2F0002075084B93F8CC3F1BB1237D23F001033D
:10C3000023750023E3822046BDE83840B0E700BF34
:10C310000001FF00005F002010B5154BD3F8D04F8F
:10C3200084B084B12379012B10D0022B0BD1A168EA
:10C3300011F00101024618BF8021204604B0BDE87B
:10C340001040FBF707B9002004B010BDA268617C63
:10C350008DF80F0002F0010294F910000DF10F04A6
:10C36000CDE900428022F8F733F804B010BD00BFD9
:10C37000005F0020F0B5294BD3F8D05F85B09DB1A8
:10C38000B02280212846FDF7D9F840228021284696
:10C39000FDF7D4F8002280212846FDF7CFF81022BF
:10C3A00080212846FDF7CAF84FF480642DB9013C7E
:10C3B000A4B2002CFBD105B0F0BD00270DF10F0693
:10C3C0002B79012B08D0022B04F1FF3217D094B245
:10C3D000002CF0D0012BF6D1AA6895F91000697CE9
:10C3E0008DF80F7002F00102013CCDE90062A4B2A9
:10C3F0004022F7F7EDFF002CE2D105B0F0BDAA68AE
:10C40000013C12F0010218BF002240212846A4B2CC
:10C41000FBF7A0F8002CD3D105B0F0BD005F0020E1
:10C420000B4B10B5D3F8D04F8CB15038C2B280212D
:10C430002046FDF783F8002280212046FDF77EF894
:10C4400020461022BDE810408021FDF777B810BDCE
:10C45000005F0020F0B5264B264CD3F8D05F203883
:10C4600000EB8000661D85B00444064425B9013404
:10C47000A642FCD105B0F0BD0DF10F072B79227853
:10C48000012B1BD0022B0AD00134A642F7D1002287
:10C490004021284605B0BDE8F040FDF74FB8AB6835
:10C4A000DB074FF04001284619D50134FBF752F85D
:10C4B000A642E3D1002DEAD105B0F0BD8DF80F20E2
:10C4C000AA6895F91000697C02F00102CDE90072BA
:10C4D00001344022F7F77CFFB442CFD1D7E70134D3
:10C4E000FBF738F8B442C9D1002DE5D0CFE700BF43
:10C4F000005F0020546F0808F0B5754BD3F8D05F8B
:10C5000085B0002D00F09680D42280212846FDF7CA
:10C5100015F8802211462846FDF710F8A822802140
:10C520002846FDF70BF83F2280212846FDF706F844
:10C53000D32280212846FDF701F8002280212846D9
:10C54000FCF7FCFF402280212846FCF7F7FF8D22F4
:10C5500080212846FCF7F2FF142280212846FCF7B0
:10C56000EDFFA12280212846FCF7E8FFC8228021A8
:10C570002846FCF7E3FFDA2280212846FCF7DEFF9D
:10C58000122280212846FCF7D9FF812280212846EB
:10C59000FCF7D4FFCF2280212846FCF7CFFFD92219
:10C5A00080212846FCF7CAFFF12280212846FCF7AB
:10C5B000C5FFDB2280212846FCF7C0FF40228021F6
:10C5C0002846FCF7BBFFA42280212846FCF7B6FFD3
:10C5D000A62280212846FCF7B1FFAF228021284601
:10C5E000FCF7ACFFA62280212846FCF7A7FFAE226D
:10C5F00080212846FCF7A2FF202280212846FCF754
:10C600009DFF002280212846FCF798FFB022802160
:10C610002846FCF793FF402280212846FCF78EFF36
:10C62000002280212846FCF789FF1022802128461D
:10C63000FCF784FF4FF4806435B9013CA4B2002CB0
:10C64000FBD1012005B0F0BD00270DF10F062B79BD
:10C65000012B2AD0022B04F1FF3214D094B2002C0B
:10C66000F6D1812280212846FCF768FFC82280216C
:10C670002846FCF763FFAF2280212846FCF75EFFC7
:10C68000012005B0F0BDAA68013C12F0010218BFFC
:10C69000002240212846A4B2FAF75CFF002CD6D134
:10C6A000002DDED1012005B0F0BDAA6895F910007B
:10C6B000697C8DF80F7002F00102013CCDE9006247
:10C6C000A4B24022F7F784FE002CC0D1C9E700BF16
:10C6D000005F0020FBF7D0B9FBF7CEB9FBF7CCB970
:10C6E000FBF7CAB9FBF7C8B9FBF7C6B90120704719
:10C6F000034620B1026812B1D26902B1104793ED2E
:10C70000017A084BB8EEC77AD3ED016AF6EE007AEB
:10C71000E7EE267AFDEEE77A17EE900A00F30B00BB
:10C72000704700BFD46E0020034620B1026812B1EA
:10C73000126A02B1104793ED027A084BB8EEC77A3D
:10C74000D3ED026AF6EE007AE7EE267AFDEEE77A9E
:10C7500017EE900A00F30B00704700BFD46E002064
:10C76000034628B102681AB1516A09B193691847A2
:10C7700093ED037A074BB8EEC77AD3ED036AF6EE72
:10C78000007AE7EE267AFDEEE77A17EE900A00F3DC
:10C790000B007047D46E002010B5044630B103681A
:10C7A00023B1DB6813B1BDE81040184703F0ECFF7C
:10C7B000D4E904239042994134BF0120002010BDE8
:10C7C000F8B170B506680F4B06F13F4202F57E02E4
:10C7D00003EB92230C4682B0054693F838056AF0C5
:10C7E0002BFFC4F34112C4F30013A9883046CDE9EE
:10C7F0000032C4F3810304F0030272F0D3F802B0F4
:10C8000070BD7047C06C0808B0B3F0B507681B4B2B
:10C81000144607F13F4202F57E0203EB92230546E0
:10C8200083B093F838050E466AF006FFA988B1FA7E
:10C8300081F3C3F11F03C3F3CC0207EB820203F0C1
:10C840000703156A4FF00F0C9B009C400CFA03F392
:10C8500025EA03031362136A1C431462C6F3001330
:10C860007209CDE900323846C6F3810306F00302AF
:10C8700072F098F803B0F0BD704700BFC06C0808B4
:10C8800010B50409013C032C19D80F4A00F00F031E
:10C8900032F8140040FA03F212F0010211D0012222
:10C8A00002FA03F3013B18407AF01CF8074B084AE0
:10C8B0001B5D184400EB400002EB800010BD00201F
:10C8C00010BD104610BD00BFB86C0808B46C080855
:10C8D000F03300202DE9F04F542204460021C348D4
:10C8E00091B079F043F8C24A611EE01C144611F879
:10C8F000013F5D1E052D88BF0023814244F8043BA3
:10C90000F5D102F11003114651F8040B012800F093
:10C9100058819942F8D1114651F8040B022800F0D1
:10C9200046819942F8D1114651F8040B032800F0D2
:10C9300052819942F8D152F8041B042900F02D814C
:10C940009A42F8D10520FAF75FF90620DFF89C92A9
:10C95000DFF8BC82FAF758F94C464FF01A0A002665
:10C9600008F5A86B277B57B3384694F90D50FFF7AD
:10C9700087FF28B105238371002380F807A0037285
:10C980001321FFF71DFF00231BF83310B9422FD0EE
:10C990000133102BF8D10021964B216105EB4505A1
:10C9A00003EBC5050122D5F8F43923751344C5F806
:10C9B000F4390723A375627585F8F02916440AF146
:10C9C000010A5FFA8AFABAF1200F04F10C04C9D106
:10C9D0005EB1894D894F00262B7C73B90136032E39
:10C9E00005F1180507F58C77F6D111B0BDE8F08F89
:10C9F00008EBC303D3F84415CEE768796AF01CFE50
:10CA000028796AF019FED5F808A05046F6F73EFEE0
:10CA1000D5F814802C680397142303FB08F30593BF
:10CA20000023CDE90C33CDE90E3304930693EB6874
:10CA3000019304F14C034FF4806202934FF40063BE
:10CA4000CDE907234FF400514FF48073CDE909136A
:10CA500050464FF4003301A90B936AF0C1FDDAF898
:10CA600000206749674B42F00102CAF800204A687B
:10CA7000134043F440334B606368B8F1010F23F077
:10CA80004073D4BF0022012223F4807343EA0223BF
:10CA90006360A2685C4B134043F00203A360E36A47
:10CAA00008F1FF385FFA88F823F4700343EA08536B
:10CAB000E36209F148014B4601204FFA86FC02E08F
:10CAC0000C338B4231D05A7D002AF9D093F90D20D6
:10CAD0006245F5D11A7C93F816A0092A36D802EBE4
:10CAE000420BD4F810800AFA0BFE4FF0070A0AFA3C
:10CAF0000BFA28EA0A084EEA080EC4F810E00628E5
:10CB000037D800F1FF3ED4F834800EEB8E0E4FF094
:10CB10001F0A02FA0EF20AFA0EFE28EA0E0E42EA86
:10CB20000E0262630130C0B2CAE7A36843F4007327
:10CB3000A360A36843F48073A360A36843F0010378
:10CB4000A360A36843F08043A36047E7A2F10A0E05
:10CB5000D4F80C800EEB4E0E4FF0070B0AFA0EFACB
:10CB60000BFA0EFE28EA0E0E4AEA0E0EC4F80CE08E
:10CB7000C5E70C284ED8A0F1070ED4F830800EEB94
:10CB80008E0E4FF01F0A02FA0EF20AFA0EFE28EA83
:10CB90000E0E42EA0E022263C4E71C4B93F8542C9B
:10CBA0003021013283F8301C83F8542CCAE617492F
:10CBB00091F8540C3524013081F8184C81F8540C4C
:10CBC000B1E6124991F8540C3424013081F80C4C30
:10CBD00081F8540C9FE60D4991F8540C2024013043
:10CBE00081F8244C81F8540CA5E600BF006B0020AE
:10CBF000045F0020300C002010160020586B00202D
:10CC000000230140E030FCFFFDF7FFC0005F002083
:10CC1000C06C0808A0F10D0ED4F82C800EEB8E0E1F
:10CC20004FF01F0A02FA0EF20AFA0EFE28EA0E0E62
:10CC300042EA0E02E26275E710B503681A79022A29
:10CC4000044603D000232371236010BD987AFFF7B8
:10CC500017FE0028F6D040F61A610022C180027249
:10CC60002021FFF7ADFD00232371236010BD00BF1D
:10CC70002DE9F04FB24EB34CA64285B057D21D46B7
:10CC800002E00C36A64252D273798B42F9D1337945
:10CC9000834201D00028F4D1F3799342F1D1346872
:10CCA000002C44D000236360A360E36023616361D0
:10CCB000A361E36126603379237196F806B0C4F866
:10CCC00008B0317AE160012B33D0022B2FD1F07AFA
:10CCD000FFF7D6FD96F90970A061B07A2774FFF7C7
:10CCE000CFFD06466061F8B1DFF8788207EB870177
:10CCF00008EB8101BB00D1F820900193B9F1000F3E
:10CD000012D091F83200E8B10E220023F271337292
:10CD1000B57109213046FFF753FD3368B2881A8395
:10CD2000204605B0BDE8F08F2046FFF785FF0024C0
:10CD3000F6E7F07AFFF7A4FD727AB37A6374A06124
:10CD40002274EDE791F828A050466AF075FC4FEA8E
:10CD50005A1001210AF01F0A023801FA0AF10328C9
:10CD600008D8DFE800F0ADA1A702774B586920EAA8
:10CD700001015961BB00D91908EB810107F1010AD2
:10CD800091F82500FFF77CFD5FFA8AFA014620B191
:10CD900080F808A040F60A30C880BB00D81908EB1C
:10CDA0008000029190F82700FFF76AFD0299019038
:10CDB000034620B180F808A040F60A50D880BB0096
:10CDC000D81908EB8000029190F82600FFF758FD73
:10CDD0000299034620B180F808A040F60A40D880A6
:10CDE000BA00D01908EB80001BF0040290F829A0CB
:10CDF000CDE902230846524668D04A21FFF704FDD8
:10CE0000019852462A21FFF7FFFC039B5246184621
:10CE10000A21FFF7F9FCBB00DA1908EB820292F84D
:10CE200024B0BBF1000F61D1484A914571D0484A06
:10CE3000914563D0474A914500F0A180464A91450B
:10CE400000F09280454A91456ED0454A914500F0E8
:10CE5000A180029BB9F80010002B01F441510CBFD6
:10CE6000032200220A4342F44572A9F80020B9F8CF
:10CE70001C2022F400621204120CA9F81C200722C4
:10CE8000A9F81020B9F8002092B242F04002A9F8A7
:10CE90000020BBF1000F20D1BB003B4408EB83080E
:10CEA000012388F832302FE7274B186A20EA010166
:10CEB00019625FE7244B186920EA0101196159E7FB
:10CEC000214B586A20EA0101596253E70A21FFF712
:10CED0009BFC019852460A2195E75846FFF7D0FC83
:10CEE0000028D9D0026883881383D5E75846FFF716
:10CEF000C7FC52460921FFF787FC95E702F500328F
:10CF0000116A41F480411162116A21F48041116279
:10CF10009FE702F58432516A41F480515162516AAF
:10CF200021F48051516294E702F56842516A41F45C
:10CF300080115162516A21F48011516289E700BF6A
:10CF4000E4A00908A0A2090800380240003001400E
:10CF500000380040003C00400034014000500140D7
:10CF600000540140300C002002F58232516A41F435
:10CF700000515162516A21F40051516269E702F592
:10CF8000FE32116A41F400411162116A21F400413C
:10CF900011625EE702F56442516A41F40011516288
:10CFA000516A21F40011516253E700BF2DE9F04F9F
:10CFB000614BD3F8E49F91B0B9F1000F04D05F4A00
:10CFC00003214846F5F77AFE00214846F5F7EEFEC4
:10CFD000D9F804305A4DD3F800801F690022560159
:10CFE00005EB4210A959794011F47C5402F1010279
:10CFF00008D0102AF3D10023C9F80C30002011B05A
:10D00000BDE8F08F027FC9F80C00002AF6D1B8F80D
:10D010004420DFF844A16FEA42426FEA524292B2E2
:10D02000A8F84420B8F8002092B242F08002A8F894
:10D03000002093F805B09B790AEB0B025B0792F88E
:10D04000C015B8F820204CBF042301238B409BB2AD
:10D0500092B222EA0302A8F82020B8F82020394929
:10D0600092B21343A8F82030B8F8003042689BB25F
:10D0700043F00103A8F80030334B9A42334A136B54
:10D080000CBF43F4001343F48003136306F118024A
:10D090004FF0070C354421F802C04B462C490322BF
:10D0A000F6F7E8F8AD682846F6F7F0FA2B6823F0B3
:10D0B00001032B602846F6F7E9FA0023CDE90C338B
:10D0C000CDE90E3306930A93BBF1030F05D8DFE8D1
:10D0D0000BF0302D022A08F13C04FFB20AEB870A5C
:10D0E00040F62B4205921B48DAF8C43501934FF401
:10D0F00080614FF48042079109924FF480514022A1
:10D10000CDE9030208914FF40033284601A90B939F
:10D1100002946AF065FA2B68012043F010032B603B
:10D1200011B0BDE8F08F08F14004D6E708F13804EB
:10D13000D3E708F13404D0E7005F0020009F24000B
:10D14000E8090020EC09002000600240003802409D
:10D15000A102000834750020C06C080838B5104DD5
:10D16000D5F8E44F24B10F4A64212046F5F7A6FD17
:10D1700000212046F5F71AFE6368012285F8E82FA2
:10D180001A68B2F844306FEA43436FEA53439BB2E4
:10D19000A2F8443013889BB243F00103138038BDDA
:10D1A000005F0020009F24001E4AF8B5D2F8E43F3B
:10D1B00073B15D6892F8E82F6C7906464AB1032C8A
:10D1C0002CD8DFE804F0222528022B6840331E60AB
:10D1D000F8BDDF681449D7F808C031F814E0DCF86E
:10D1E0000010286821F00101CCF80010818989B273
:10D1F00021EA0E0181811A7403889BB243F0010376
:10D2000003803A77FFF7AAFFD9E72B683433DEE7CC
:10D210002B683833DBE72B683C33D8E700231B60EF
:10D22000FFDE00BF005F0020C86B080810B5224C6D
:10D23000D4F8E43F83B194F8E82F6AB194F8EC2F66
:10D24000032A0AD0022A10D0002384F8E83FFFF70F
:10D25000ADFE08B984F8ED0F10BD5A685379032B61
:10D2600027D8DFE803F023201D185A685379032BD1
:10D270001FD8DFE803F00D0A0702136840330022CD
:10D280001A6010BD13683C33F9E713683833F6E7CA
:10D2900013683433F3E71368403364221A6010BD17
:10D2A00013683C33F9E713683833F6E7136834330F
:10D2B000F3E700231B60FFDE005F00202DE9F04F45
:10D2C000C44BC54993F8F07F93F8F18F93F8F2EFD0
:10D2D00083B003F6F4704FF0000C00F5007ACDF83F
:10D2E00004C001228378C578C3F1FF039BB22C46AA
:10D2F000002B00F03B81B0F80090B84EC3F1FF0363
:10D30000A6FB09B605FB03F376091B12052E00F2F6
:10D310006E81DFE816F01701FB00E300C600AB00EA
:10D320000600AE4EA6FB09E46409C4EB0414A9EBA5
:10D330008404A4B2EF1AC4F13C0407FB04F4A6FB76
:10D3400004645FFA83F808EB54145FFA84FE2F46F6
:10D350001C462B460125764601951D0245EA0445EB
:10D360001724354383460CEB0406331B02FA04F9F9
:10D370009BB219EA050F03F12A030CBF012002201A
:10D38000013C41F82300631CEFD1584604300CF1F6
:10D39000180C50451FFA8CFCA4D1914B4FF44062FD
:10D3A000A3F8FC208022A3F8FE20019B33B1894B17
:10D3B00083F8F2EF83F8F18F83F8F07F854A92F8D3
:10D3C000ED3F002B4FD0D2F8E43F002B4BD0EFF3D2
:10D3D0001181102282F31288D8685D6884682268FF
:10D3E00022F0010222602C687E4A6D7932F81550D5
:10D3F000A28992B222EA0502A281026944681F2A28
:10D4000040F2BC80203A202000FA02F2E260CAB268
:10D4100082F31188DA686F489268D0F8E40F40F61A
:10D420002B41516011680124214311601C74036871
:10D430001A7DA24204BF02221A7593F82C100CBF69
:10D440004FF400720022012900F0B18093F84410DB
:10D45000012900F0988093F85C10012900F0B48055
:10D46000002A40F0C18003B0BDE8F08FDFF86CE126
:10D47000EF1A2E46AEFB09546409C4EB0414A9EB61
:10D480008404A4B204FB07F7AEFB07E75FFA83F856
:10D4900008EB5717FFB201251C46B6463B460195DF
:10D4A0005BE74E4FA5EB030E2E46A7FB095464091C
:10D4B000C4EB0414A9EB84081FFA88F8C8F13C08EF
:10D4C0000EFB08F8A7FB0878DFB207EB58185FFAE5
:10D4D00088F801254446B64601953EE73F4FEE1ACF
:10D4E000A846A7FB09E56D09C5EB0515A9EB850560
:10D4F000ADB205FB06FEA7FB0E7EDFB207EB5E1E9C
:10D500005FFA8EFE01257646019526E7334EA5EBA0
:10D51000030EA846A6FB09756D09C5EB0515A9EB19
:10D520008507BFB2C7F13C070EFB07F7A6FB0767ED
:10D530005FFA83FE0EEB5717FFB21E4601230193DD
:10D540003B460AE7A5EB0308244C09FB08F8A4FBBB
:10D5500008485FFA83FE0EEB58185FFA88F81E46FB
:10D560002F462B46012544460195F6E6AE462E464B
:10D570002B46A8462F4601250195EEE6202000FA0D
:10D5800002F2A26043E7022183F8441093F85C1092
:10D59000012942F4006217D043681B6800215962D8
:10D5A000998989B20A439A8103B0BDE8F08F0221BC
:10D5B00083F82C1093F84410012942F48062E2D0E1
:10D5C00093F85C100129E7D1022183F85C1042F442
:10D5D0008052E1E7005F0020347500208988888848
:10D5E000F86F0020C86B08084FF40072D4E7444677
:10D5F0003B467646B1E600BF2DE9F04FA14FA7B0FC
:10D6000000210A260C4607F580754FF0050B0196A0
:10D610008BE0BAF1000F19D143F04003BEF18C0F3B
:10D6200087F8043500F2E48004F1010C98340DEB26
:10D63000040A0CF198040DEB040C74464FF0040E30
:10D640000AF88CEC0CF88C3C04F1020EBEF18C0F45
:10D6500042F0020C00F2CC8004F198036B4403F812
:10D660008BCC04F1040CBCF18C0F03F88CBC00F2E1
:10D67000BF800EF198060DEB060E4FF0060A0EF86D
:10D680008CAC04EB0A0E4FEA8909BEF18C0F5FFAED
:10D6900089F603F8890C00F2AB8004F19C0CEC4491
:10D6A0004FF007090CF88C9C04F1080CBCF18C0FAE
:10D6B00003F8876C00F29C800EF198060DEB060EC5
:10D6C0000EF88CBC03F8852C04F10A028C2A00F2B7
:10D6D0008F8004F1A0060DEB060C0CF88CAC03F85F
:10D6E000830C04F10C008C2800F2828004F1A20269
:10D6F00004F1A3036A446B4402F88C9C044603F8CB
:10D700008C8C480901F01F0C55F82030012202FAD8
:10D710000CF223EA020345F82030019B013B019300
:10D720006ED00131B1F5F07F6AD23C222846FAF77B
:10D73000D5F9011E5FDB07EB410297F80435B2F81B
:10D740003CC11CF0040FC1F30722C8B25FFA8CF988
:10D750004FEA1C2803F0400A04F1020E7FF459AF8F
:10D76000BAF1000F03D103F0380CCC4519D003F007
:10D77000870343EA0903BEF18C0F87F8043537D8D5
:10D7800004F1010C0CF1980698346C440DEB060C76
:10D790004FF0040904F88C9C74460CF88C3C0EF194
:10D7A000020EBEF18C0F23D804F198030DEB030C8D
:10D7B000231D8C2B0CF88B2C0CF88CBC18D80EF17C
:10D7C00098020DEB020E06220EF88C2C0CF8890C38
:10D7D000A0188C280CD804F19C0304F19D026B4422
:10D7E0006A44072403F88C4C044602F88C8C88E7C2
:10D7F0006FF0004485E7204614B927B0BDE8F08FEC
:10D80000D7F8FC54204A95F91030A96803EB83033C
:10D8100002EB83038A07186A20D5234603AA002156
:10D8200071F01AF9AB689B0701D50120E5E7174BAA
:10D8300017491A68174B4FF4FA7000FB02F2A3FB6A
:10D840000232486892094B681B1A9A42FBD26B69F4
:10D85000002BEAD01A689B881383E6E76B6913B143
:10D860001A689B885383094B09491A68094B4E680B
:10D87000D200A3FB023292094B689B1B9A42FBD257
:10D88000CBE700BFF86F0020300C0020A43600204A
:10D89000001000E0D34D6210F0B5284CD4F8FC0421
:10D8A00083B010B194F802350BB103B0F0BD012381
:10D8B0000DF10702842184F80235FDF791FC94F8FC
:10D8C0000425D4F8FC0404210A43FBF737FED4F8FE
:10D8D000FC040DF107028421FDF782FC9DF807305E
:10D8E00013F00406F3D1164D84F804353C2231467A
:10D8F000284678F03BF83246124E05F13A0005F220
:10D90000FA374FF0010E30F8023F334002F01F01AA
:10D910009BB24FEA521C0EFA01F1013223B155F8C5
:10D920002C300B4345F82C30B842ECD1FFF764FEA5
:10D930000028FBD184F8020503B0F0BDF86F002089
:10D94000F870002004DFFFFF70B5414DD5F8FC44AE
:10D9500082B094B395F80035012B42D0022B2ED122
:10D96000082194F910303B4A85F8031503EB830333
:10D9700002EB8303A2688DF80510002040F20441F9
:10D9800092078DF80400ADF80610186A42D50423FA
:10D990000DEB0302002171F05FF8A3689B0722D50D
:10D9A0002D483C22FF2177F0E1FF95F8013523B99E
:10D9B000FFF772FF012385F8013502B070BD0DF14C
:10D9C0000302A0212046FDF70BFC9DF8033003F075
:10D9D0000503012B37D0002B2FD1D5F8FC440821AB
:10D9E000BFE74821BDE71D4B1D491A681D4B48681C
:10D9F0004FF4FA7606FB02F2A3FB023292094B685F
:10DA00001B1A9A42FBD26369002BC9D01A689B8803
:10DA10001383C5E7636913B11A689B8853830F4B5F
:10DA20000F491A680F4B4E68D200A3FB02329209CD
:10DA30004B689B1B9A42FBD2A9E70B4A126840F243
:10DA4000DC539A42B9D9D5F8FC44482189E700BF94
:10DA5000F86F0020300C0020F8700020A436002061
:10DA6000001000E0D34D6210242A00202DE9F0417F
:10DA7000334D95F8023582B003B1FEE7012285F8F7
:10DA8000022595F80325044602F0F702D5F8FC04B8
:10DA900085F803250E461946FBF750FDE2B207460E
:10DAA0000921D5F8FC04FBF749FDB4F5807F3FD090
:10DAB000D5F8FC04DFF88C8050220821FBF73EFDEE
:10DAC000D5F8FC040DF10702A021FDF789FB48B948
:10DAD000D8F8D830B8F8DC2059690A4214BF5A8304
:10DAE0001A83EDE79DF8074014F02004F0D1E2B26C
:10DAF0000A21D5F8FC04FBF721FD3219D5F8FC0406
:10DB0000C0210134FDF76CFB362CF0D157B995F8E4
:10DB10000325D5F8FC0402F0F702394685F8032501
:10DB2000FBF70CFD002385F8023502B0BDE8F0815B
:10DB3000D5F8FC0440220A21FBF700FDB8E700BF3E
:10DB4000F86F0020F03300202DE9F04F5F4D95F87D
:10DB50000275C3B007B1FEE795F80325044602F04D
:10DB6000F7020123D5F8FC0485F803250E46394653
:10DB700085F80235FBF7E2FCFF2C4FF009038DF826
:10DB8000054088BFA40801AA8CBF04F0C008B846AD
:10DB900002204FF0000C4FF00A0B0DF1050A4FF078
:10DBA0000B09137014E0B1F5827F02F800B00AF897
:10DBB000003016F80C3017D80CF1010CBCF1360F00
:10DBC00002F8079004F1060402F80E30084614D05B
:10DBD000871C48EA0C03B7F5827F00F10401044674
:10DBE000DBB200F1030EDED90CF1010C6FF0004145
:10DBF000BCF1360F364C0846EAD1B4F5827F62D8C4
:10DC0000082353540DF10503A0211954831CD5F8A2
:10DC1000FC44304E94F9101001EB810106EB8101B8
:10DC2000086AA168890722D5002170F015FFA36852
:10DC30009B0731D5284CD5F8FC040DF10302A02137
:10DC4000FDF7CEFA48B9D4F8D830B4F8DC205969D9
:10DC50000A4214BF5A831A83EDE79DF8033013F08C
:10DC60002003F0D185F8023543B0BDE8F08F61693B
:10DC700011B10E68898871831849194F0E681949C6
:10DC8000D7F804C0F600A1FB0616B6097968A1EB27
:10DC90000C018E42FAD2C7E7104B11491A68114B9A
:10DCA00048684FF4FA7606FB02F2A3FB02329209AF
:10DCB0004B681B1A9A42FBD26369002BBAD01A68D0
:10DCC0009B881383B6E76FF00043A0E7F86F00204E
:10DCD00001000080300C0020F0330020A43600202A
:10DCE000001000E0D34D6210014B1B685B681847C1
:10DCF000E0A50020024B1B6808309B68184700BF56
:10DD0000E0A50020012070470120704701207047E6
:10DD1000012070470120704731B10C4BD3ED017ADF
:10DD2000F8EEE77AC1ED007A72B1084BDFED086AD0
:10DD30009B68A3F5D543333B07EE903AF8EEE77ABC
:10DD400087EEA67A82ED007A704700BFE0A500203A
:10DD50000000C842012070470120704710B4414CB8
:10DD60000023224692F90410012902F10C022DD061
:10DD70000133052BF6D12246002392F90410032922
:10DD800002F10C0234D00133052BF6D1002394F9B3
:10DD90000420052A04F10C043FD00133052BF6D1F1
:10DDA000314B1B68D9034ED5304B016803F1F004A9
:10DDB00002E01433A34246D01A689142F9D1DA68DE
:10DDC000D201F6D501205DF8044B7047284A03EBD9
:10DDD000430302EB8303DB68EBB1264A037992F835
:10DDE0003DC09C45EED092F83C209A42C3D1E9E771
:10DDF0001F4A03EB430302EB8303DB68002BC6D00F
:10DE00001D4A037992F83D109942DBD092F83C20EC
:10DE10009A42BBD1D6E72246AFE7154A03EB43034C
:10DE200002EB8303DB68002BBAD0144A037992F823
:10DE30003D109942C6D092F83C209A42C2D00A4B7B
:10DE40001B68D903B0D40379203BDBB2152B06D86D
:10DE50000B495DF8044BD94001F0010070470020E8
:10DE6000B1E700BFECA50020B40000105816002058
:10DE7000E0A50020000300204C05002098070020AA
:10DE8000010031000C4B10B5844603F1F00E002068
:10DE900002E014339E450ED01A686245F9D1DA6863
:10DEA0008A4218BFD96000F1010403F1140318BFBE
:10DEB000E0B29E45F0D110BD58160020704700BF5B
:10DEC000044B40F2FF7203EBC0039142A8BF11461E
:10DED0009980704774600020112806D8044B03EB2A
:10DEE00080039B6C0BB19B6819602AF0FDBF00BFDB
:10DEF000E0A50020112806D8034B03EB80039B6CA0
:10DF00000BB19B6819607047E0A500200D4A92F89C
:10DF1000F03083B10C4B93F8901061B193F89110ED
:10DF200061B1D2F8F4000022FA2883F89120A8BF4A
:10DF30004FF0FF3070476FF0010070476FF0020044
:10DF4000704700BF58160020E0A500202DE9F041E1
:10DF5000104C04F1940884F895101746002502230C
:10DF60004246FF21064684F89450FCF7BFF968B199
:10DF7000424630460223FF21FCF732FA30B1B4F8B2
:10DF800094305BBA28463B80BDE8F0816FF00C000E
:10DF9000FAE700BFE0A500200C4B93F894218AB16A
:10DFA00093F895215AB10A49D1F8F8000022B0F54A
:10DFB000967F83F89521A8BF4FF0FF3070476FF030
:10DFC000020070476FF00100704700BFE0A500201D
:10DFD00058160020024BD3F898315B68184700BFF1
:10DFE000E0A50020024BD3F898319B68184700BF8A
:10DFF000E0A50020024BD3F89831DB68184700BF3A
:10E00000E0A50020014BD3F8FC0070475816002013
:10E01000054B93F89C311BB1044BD3F800017047BA
:10E020006FF00100704700BFE0A5002058160020E7
:10E0300070B5324C05460323006804F5D072002108
:10E04000FCF7CEF958B96FF00103C4F8A4312C4A9B
:10E05000D4F8A831116832338B4245D370BDB4F87F
:10E06000A03194F8A2015BBA9BB207EE903AF8EEA9
:10E07000E77AF2EE046A87EEA67A94F8A0310821D6
:10E08000BDEEC77A84ED697A4FFA83FCBCF1000FCC
:10E090004FEA4C02A8BF5B0082F00702B4BFD3B2C4
:10E0A000DBB20139F0D194F8A121082153405AB2D2
:10E0B000002AB8BF52004FEA4303B6BF82F00702FE
:10E0C000DBB2D3B20139F2D19842C0D1D4F8A43135
:10E0D0002BB1D4F8A4214FF6FF739A42B7D14FF079
:10E0E000FF33C4F8A431B2E7C4F8A8112868054A80
:10E0F000BDE8704001233121FCF7F8B8E0A500200D
:10E10000242A00208CA70020014BD3F8A4017047DB
:10E11000E0A50020437A5A1C0344D2B2427299729D
:10E12000037A934200D97047002AFCD010B5044608
:10E1300004F10A01D0E9003098470023637210BD52
:10E14000324ED6F8AC51D6F8B80180B52EF018FD95
:10E1500028462EF015FDD6F8B87179798B074BD586
:10E1600000210846F9F7A8FC00210120F9F7A4FCDA
:10E17000274C3B6838465B68984760B92B6828464F
:10E180005B68984708BBD6F8B8713B6838465B684F
:10E1900098470028F2D0D6F8B801D4F8D820036800
:10E1A000B4F8DC10DB68518398472B6801461B6884
:10E1B00028469847D4F8D830B4F8DC201A832B6866
:10E1C00028465B6898470028DDD0D4F89C202B684F
:10E1D000B4F8A010DB685183284698470146D6F86A
:10E1E000B80103681B689847D4F89C30B4F8A020A5
:10E1F000D6F8B8711A83BCE73B6838469B6941F092
:10E2000002019847D6F8B871AAE700BFE0A5002040
:10E21000F033002030B5032083B00D461446FBF7E1
:10E22000B5FA01909DB107EE900A9FED0B7AF8EEDA
:10E23000677AF0EE006A67EE877AB8EE047AA7EEA6
:10E24000A67ADFED067A67EE277AC5ED007A0CB183
:10E25000034B236003B030BD6740533A00007A445B
:10E260003313904300B500680379012B85B00DD0BE
:10E27000022B07D1012303AAFF21FCF759F805B0AF
:10E280005DF804FB002005B05DF804FB8268417C6A
:10E2900090F9100002F00102019203AA0092FF22FD
:10E2A000F6F762F805B05DF804FB00BF30B5044630
:10E2B00000680379012B85B02DD0022B0ED0224BA4
:10E2C0006FF00102C3F8FC202049214AD1F8E43163
:10E2D00015683233AB422CD305B030BD826812F0E2
:10E2E000010F18BF512103AA08BFD121FCF720F864
:10E2F0000028E4D0BDF80C30134A5BBA9BB2C2F8D8
:10E30000FC30D2F8FC30B3F5C87FDDDD4FF0FF33D1
:10E31000C2F8FC30D8E78368417C90F9100003F024
:10E320000103019303AB009351220223F6F71CF87B
:10E33000DEE701F5F472C1F8E451206800235121B1
:10E34000FBF7D4FF05B030BD58160020E0A5002033
:10E35000242A002000B500680379012B85B02DD058
:10E36000022B24D1826812F0010F18BF002103AAEA
:10E3700008BF8021FBF7DCFF1B4B83F89C0198B1A1
:10E38000BDF80C305BBA9BB2B3F5FA6F24D2174AD2
:10E390001749A2FB0323DB0807EE903AF8EEE77A71
:10E3A000FDEEE77AC1ED407A05B05DF804FB0E4B57
:10E3B000002283F89C2105B05DF804FB8368417C52
:10E3C00090F9100003AA03F00103CDE90023022312
:10E3D0000022F5F7C9FFCFE7054B4FF0FF32C3F836
:10E3E000002105B05DF804FBE0A50020CDCCCCCC2D
:10E3F0005816002010B500680379012B84B00C4634
:10E400001FD0022B02D0002004B010BD826812F091
:10E41000010F18BF002103AA08BF8021FBF788FF66
:10E420000028F0D05CB19DF80D309DF90C20DB097F
:10E4300003EB830302EB820203EB4203238004B06D
:10E4400010BD8368417C90F9100003F00103019333
:10E4500003AB009300220223F5F786FFE0E700BF3D
:10E4600070B50668F56982B00446002D59D00023C6
:10E470002B7004230DEB03023046FF21FBF7B0FFA6
:10E4800010B9002002B070BD206804236A46FF2145
:10E49000FBF7A6FF0028F4D09DF804309B09023B4F
:10E4A000012BEED9BDF80430BDF80620BDF80010F0
:10E4B000BDF802605BBA43F6FF74C3F30D03A342D9
:10E4C000DFD0002BDDD052BAC2F34A1240F2FF7CFB
:10E4D0006245D6D0002AD4D049BAC1F30D01A14279
:10E4E000CFD00029CDD076BAC6F34A166645C8D03B
:10E4F000002EC6D05C1A002CB8BF6442FF2CC0DCD2
:10E50000941B002CB8BF6442FF2CBADC0B445B1098
:10E5100032445210C5F805300123C5F801202B7094
:10E52000B0E709211420FAF781F8F0610546266862
:10E530009DE700BF70B50668F0690D461446A0B3AC
:10E54000D0F80130CDB1D0F805209FED1B7ADFED7A
:10E550001B5ADFED1B6A07EE902AF8EE677AB7EEDA
:10E56000006A77EEC77A77EEA77A87EEA57A77EE1C
:10E57000467A67EEE67AC5ED007AACB107EE903ADE
:10E580009FED107ADFED106A9FED106AF8EEE77AE2
:10E5900067EE877A87EEA67ADFED0D6A77EE467A28
:10E5A00077EEA67AC4ED007A70BD09211420FAF73F
:10E5B0003DF8F061C4E700BF9AC9CC449AC94C4603
:10E5C0000E76D7450000484300E0FF440000484273
:10E5D0003393884370B50668F46982B0F4B10023C0
:10E5E000237004230DEB0302FF213046FBF7F8FEF6
:10E5F00010B39DF804309B0919D1BDF80420BDF873
:10E60000063052BA5BBA92B2C3F34A1301212170A9
:10E61000C4F80520C4F8013002B070BD05460921D8
:10E620001420FAF703F8F06104462E68D7E7044A8D
:10E6300004210320F9F774FF002002B070BD00BF71
:10E640006C18090870B50668F06982B00D4614466A
:10E65000002848D0D0F80530DFED266A9FED267AF5
:10E6600007EE903AF8EE677AD0F8013077EEE67A66
:10E67000F3EE096A67EE877AB2EE047A67EEA67A5D
:10E68000F4EEC77AF1EE10FA20DCBAEE047AF4EE7A
:10E69000C77AF1EE10FA19D42DB19FED187A67EE12
:10E6A000877AC5ED007A7CB107EE903A9FED146A47
:10E6B000DFED146AB8EE677ADFED137AE7EE067ADB
:10E6C00077EEA67AC4ED007A02B070BD17EE900A1C
:10E6D00070F07AFC0D4ACDE9000104210320F9F71E
:10E6E0001FFF02B070BD09211420F9F79FFFF061F0
:10E6F000B0E700BF00000046000080380AD778432A
:10E700000319C83D33938843000048C29018090894
:10E71000F0B52DED028B4E4E16F8143C022B83B053
:10E720000D46144619D0DFED4B7A7DB19FED4A7A44
:10E730009FED4A6ADFED4A6A67EEA77A67EE877A4D
:10E7400087EE867A77EE267AC5ED007A0CB1454BD6
:10E75000236003B0BDEC028BF0BD434B96F848102C
:10E760005B6803F0020239BB5B0525D42AB3B6F916
:10E770006E3007EE903AB6F96C30F8EEE77A06EEB6
:10E78000903A27EEA77AF8EEE66AB6F97030A6EE70
:10E79000A67A07EE903AF8EEE77AA7EEA77AB5EEFA
:10E7A000C07AF1EE10FABEDBF1EEC77AF4EE677ACA
:10E7B000F1EE10FAB9D7B6E722B9D6F88830D3ED22
:10E7C000337AB2E7294F0DF1060029F04FFEBDF86C
:10E7D0000630D7F8D4259FED266ADFED266A9FED37
:10E7E000267A9B1A07EE903AF8EEE77AB0EE408A66
:10E7F00067EE867AA7EEA67AFDEEC77AB0EE470AF4
:10E8000017EE903A2033402B1FD8F9F7D1FC1B4B61
:10E8100097F8FA11D6ED157AA3F12C021846443B6D
:10E82000002918BF134693ED057AD0ED006A77EE04
:10E83000877AE8EE406A27EEA77AA6EEA67AB5EECA
:10E84000C07AF1EE10FAAFDA6DE79FED020ADEE76B
:10E85000D8B6002000000000CDCC9C3F00409C4674
:10E8600082E6C54733139043B4000010E0A50020B2
:10E870000AD7233C35FA8E3CDB0FC93FC8AB0020DA
:10E8800010B50B4B82B053F8304001916CB107EEDC
:10E89000901A94ED047A94ED030AF8EEE77AA7EE65
:10E8A000870A71F0C5FFA368186002B010BD00BFF1
:10E8B000746000202DE9F0414D4F97F8903082B000
:10E8C00043B14C4E96F88C50012D04463BD0022D9E
:10E8D0005AD015B102B0BDE8F08101228021006854
:10E8E000FAF72CFE20680122FF21FAF727FE2A46BC
:10E8F00029462068FAF722FE96F88D20206891219B
:10E90000FAF71CFE294620680122FAF717FE2A466C
:10E910002068FF21FAF712FE2A4620688021FAF7C4
:10E920000DFE294620680122FAF708FE324B3349D2
:10E930001A6881F8F0000123C6F8902086F88C3020
:10E9400002B0BDE8F08101AA0068DFF8B0800021C4
:10E95000FCF746FC9DF8043088F8F000DA073ED555
:10E96000D6F89430002BB5D0234AD6F89010126810
:10E9700092B2521A9342ADD24FF0FF320023C8F840
:10E98000F42086F88C30A5E70068DFF8708001AAD3
:10E990001321FCF725FC9DF8043088F8F0005B0794
:10E9A000DED020682B4601AA1E21FBF719FDBDF819
:10E9B0000430206801220B215CBAFAF7BFFD104B2E
:10E9C00088F8F000A4B2A3FB0434E4080122002379
:10E9D000C8F8F44087F8912086F88C307AE7064A28
:10E9E00002231268C6F8902086F88C3072E700BFC8
:10E9F000E0A50020D8B60020242A002058160020C8
:10EA0000CDCCCCCC2DE9F041DFF8BC802C4E2D4D87
:10EA100041F0010284B000210446FAF78FFDD8F8D6
:10EA20000070C6F8907019E0022B3FD1A368DB0795
:10EA30000DF10F024FF0130120465EBF0DF10F02E2
:10EA400093212046FCF77AFB9DF80F3085F8F00003
:10EA500013F0070319D1D6F894204ABB2379012B70
:10EA6000E2D1A268617C94F9100002F001020192E7
:10EA70000DF10F0200921322F5F776FC9DF80F308E
:10EA800085F8F00013F00703E5D001220B212046A2
:10EA9000FAF754FD002211462046FAF74FFD0123F4
:10EAA00085F8F000184604B0BDE8F0810020CBE7FF
:10EAB000D8F8001089B2C91B8A42CFD2F2E700BF52
:10EAC000D8B6002058160020242A002010B5164C75
:10EAD00084F89510017984F8962001294FF00002FE
:10EAE00082B084F8942010D0022903D06FF00C007B
:10EAF00002B010BD032304F19402FF21FBF79EFB3B
:10EB00000028F3D0002002B010BD8268417C90F94B
:10EB10001000943402F00102CDE900420323FF22E9
:10EB2000F5F756FCECE700BFE0A50020006803798C
:10EB3000012B0BD0022B00D0704783680E4A13F0D4
:10EB4000010315D000235121FBF778BB00B5836882
:10EB5000094A417C90F9100083B003F00103CDE92C
:10EB6000002300235122F5F733FC03B05DF804FBCA
:10EB7000D121FBF763BB00BFC8A700200068037961
:10EB8000012B0CD0022B00D0704783680E4A13F083
:10EB9000010F4FF0010313D00021FBF74FBB00B56D
:10EBA0008268417C90F9100083B002F0010201926A
:10EBB000054A00920022F5F70BFC03B05DF804FB58
:10EBC0008021FBF73BBB00BF8CA7002030B5194D5F
:10EBD00095F8943183B00BB903B030BD04460DF104
:10EBE000050100686EF04AFF9DF805307BB920688A
:10EBF000114A01214FF4064485F896100323FF21A2
:10EC0000A5F8944003B0BDE83040FBF76FBB0DF1B1
:10EC1000060296212068FFF799F9084ABDF80630E8
:10EC20000749A2FB0323DB080122C1F8F83085F86D
:10EC30009521DCE7E0A5002074A60020CDCCCCCC4B
:10EC400058160020F8B504460F4616460025204603
:10EC5000202177F052FD0446C8B10378202B03D160
:10EC600014F8013F202BFBD02046FAF7D1F9B0F57C
:10EC7000617F10DB40F63403984211DD30231A46E1
:10EC8000C5B17B703378013333702046F8BD002D59
:10EC9000FBD10125DBE700231A46002DF1D109E065
:10ECA000074AA0F56173A2FB0323DA08C3F3C70385
:10ECB000002DE6D13A70337801333370E9E700BFB5
:10ECC0001F85EB51002ABCBF80185242002B30B583
:10ECD00003EB010503DA0C465B4229462546002872
:10ECE000B7BF121A841814460020A4F11D0C002985
:10ECF000BCBF2B460021BCF1000FC4BFA2EB0C022D
:10ED00001418A5F10F02002AC4BF9B1A5D18844293
:10ED10001EDBC1F1010C0F4AC1EB0113AC4400EB47
:10ED20004303CCEB0C1C01344FEA4C0C02EB4302C6
:10ED30004FF0200E8D42A8BF002304DB22F813E021
:10ED40001E339C45FAD10130A04202F10202F1D1FA
:10ED500030BD00BF347100201B4B1C48196C1C4A8D
:10ED600010B441F080510124196404625321FF243E
:10ED7000CA205462506251625B6FDB0085B013D4CD
:10ED80000023144902930291029A1348043202921A
:10ED9000029A136003930391039B0393039B1860F0
:10EDA00005B05DF8044B70470A4B002201920193B5
:10EDB000019B0193019A084B12689A42E0D105B079
:10EDC0005DF8044B704700BF0038024000000E425F
:10EDD000002800405028004076614E6970B5054615
:10EDE000BDF8106001600C4619B119462046F3F7D2
:10EDF00065FF31462046F3F7D9FF61680B68B3F829
:10EE000044206FEA42426FEA524292B2A3F8442091
:10EE10001A8892B242F001021A804A79032A17D85E
:10EE2000DFE802F0110C070240330022AB601A60E9
:10EE300070BD3C330022AB601A6070BD38330022D5
:10EE4000AB601A6070BD34330022AB601A6070BDD5
:10EE50000023AB601B60FFDE2DE9F04F85B0064656
:10EE6000BDF838B09DF83CA0894617469846F3F7A0
:10EE7000D5FE002856D02C4C94F898300A2B4CD84C
:10EE800003EB430204EB421202900020C2F89C0004
:10EE900082F8A0005A1CD2B284F8982003EB4303F6
:10EEA000307903929C3404EB4314FDF7E9FC02999A
:10EEB000054618B3039A027280F806900220E871A2
:10EEC00043463A46CDF800B02046FFF787FFBAF137
:10EED000000F0AD111212846FDF772FC2B68AA8881
:10EEE0005A83204605B0BDE8F08F2846327A0221C9
:10EEF000FDF78AFC204605B0BDE8F08FCDF800B0E4
:10EF000043463A462046FFF769FFBAF1000FECD1BD
:10EF100011215046FDF754FCE3E7044A0021042088
:10EF2000F9F7FEFA0024DCE7D8B60020B418090887
:10EF300030B50368284D294C2DED028BAB42246877
:10EF400083B0F0EE408AB0EE608A10D005F580659F
:10EF5000AB420CD005F57055AB4208D005F5806585
:10EF6000AB4204D005F58065AB4218BF6408B4FB22
:10EF7000F1F303F57F43FF331B0CB4FBF3F40023E1
:10EF8000B4FBF1F5019200932246ABB20221FFF7E8
:10EF900063FFE0B1B5EE408A07EE904AF1EE10FA59
:10EFA000F8EE677A0ABF07EE105A28EE278AB8EE05
:10EFB000478A9FED0B7AC8EE076A0123037127EE9B
:10EFC000667AC0ED046AA8EEA77A80ED037A03B0F2
:10EFD000BDEC028B30BD00BF00000140E409002001
:10EFE00000007A442DE9F04F2DED028BAA4BAB4E79
:10EFF0001B78AB4DDFF8CC92B5B000270293B0463A
:10F00000B246BB46DAF80040002355F8332094425C
:10F0100003D001330E2BF8D1FF234B4493F8BC34BB
:10F02000022B00F0BB80032B00F0AF80012B09D135
:10F03000DAF80C3023F0807323F0080343F0040364
:10F04000CAF80C305046FEF789FE48B90BEB8B032B
:10F0500008EB8303D96801F00C03042B00F0A980AE
:10F060000BF1010BBBF10C0F0AF1140ACAD18D4D43
:10F07000DDF80880A5F1F00408E02068E260FEF702
:10F0800001FF5044C7B21434A5421FD02046FEF7FA
:10F0900065FE0028F7D1E368590703F00C02F2D5AA
:10F0A000042AF0D023F0080242F00402781C4745FD
:10F0B00011465FFA80FA23F00403DED32068E36090
:10F0C00019461434FEF7DEFEA542DFD10025764F47
:10F0D000DFF8F4A12C46A846AB463046FEF73EFECC
:10F0E000002840F0A880F06842076AD5029B57F8D4
:10F0F0000C2C434500F2A680030764D4002D57F87A
:10F100000C3C40F3BD8028A900229C4602E0AA42A4
:10F1100000F0B58051F8043F1B689C4502F10102E4
:10F12000F5D1C20164D40BF1010BBBF10C0F06F158
:10F13000140607F11407D0D1574B93F800E0BEF145
:10F140000C0F00F30E82594B594A1B791370032B95
:10F1500040F2BC801A1F022A00F27582052B00F0D3
:10F160006382062B0CBF4FF47A564FF47A665149EE
:10F17000514800224A600027504AB2FBF6F20026AE
:10F180000A60C0E900674E4AA1E0DAF80C3023F0CB
:10F190000C0343F08073CAF80C3053E7DAF80C30F4
:10F1A00023F0807323F0040343F00803CAF80C3003
:10F1B00048E72046FEF766FE0137FFB20744FFB27C
:10F1C0004EE70207ADD5002C57F80C3C4BDD1DA9CE
:10F1D00000229C4601E0A24244D051F8043F1B6843
:10F1E0009C4502F10102F6D1410787D4C2019AD5AC
:10F1F000002C57F80C3C0ADD1DA9002251F8040F21
:10F200000068834202F101028DD0A242F6D1002DA6
:10F210000ADD28A9002251F8040F0068834202F198
:10F22000010280D0AA42F6D14FF080711846F160F9
:10F23000FEF728FE77E75B46524601210420F9F7E6
:10F240006FF970E720F00801F1601046FEF71AFE32
:10F25000F06808F1010803075FFA88F8B3D44107A2
:10F26000C4D54BE76346184634AB03EB850208214F
:10F27000F16042F82C6C0135FEF704FE53E763465B
:10F28000184634AB03EB84020421F16042F8586C59
:10F290000134FEF7F7FD46E7AC00001058160020D9
:10F2A000246C0808481700206416002038620020EB
:10F2B00028600020306000203860002040420F00AD
:10F2C000C1DE0008D8B60020F0180908B74AC9F80E
:10F2D000CC24B74A12F81330002B00F0AE81A645BB
:10F2E00000F3B381BEF1000F00F0A6809FEDB18A5C
:10F2F000DFF818B3DFF80C8304951DAC4FF0000A5B
:10F300007746AD4BDBF800201B7854F8046FC2F34E
:10F310000072062B00F23A81DFE803F0B4AAA0796C
:10F3200004040400052B00F07381A449A448062BB3
:10F3300018BF01460025019200950A4614230221B8
:10F340003046FFF789FD0290002800F01F819D4B99
:10F3500031681A78002A00F01081CDF80C8003E0A3
:10F360000135954200F00B812B0158F8033099428A
:10F37000F6D1EAB2082A00F009810298924B01689E
:10F3800005910D684E6807954FF4907101FB0231AD
:10F39000039BC16503EB02130691996013016A6E2A
:10F3A00008933568002A00F05481B5F844306FEABC
:10F3B00043436FEA53439BB2A5F844302B889BB27A
:10F3C00043F080032B8073790A9319467F4B585C76
:10F3D000B379298C5B074CBF0423012383409BB284
:10F3E00089B221EA03012984298C89B20B432B8439
:10F3F0002B889BB243F001032B80002A00F0578139
:10F40000029A01231371724B43F83A200EE0DFEDAC
:10F41000710A714BB0EE600A59883046FFF788FDDB
:10F420006B4B43F83A00002800F09D810AF1010A75
:10F4300057457FF466AF049D99F8D03D63BB674A9A
:10F4400002210420F9F76CF899F8CA04B0FA80F0A8
:10F45000400935B0BDEC028BBDE8F08FDFED600AEE
:10F460009FED600A30464FF4FA61FFF761FDD7E780
:10F47000DFED5D0A3046B0EE600A4FF47A71FFF7B7
:10F4800057FDCDE79FED4B0AF0EE480A30464FF4AA
:10F49000C871FFF74DFDC3E799F8D18D99F8D23DBA
:10F4A00008F10108A8EB0308B8F1120F0BDD1223D5
:10F4B000022100934D4A89F8CA14434600210420D2
:10F4C000F9F72EF8C0E799F8DC3D012B00F0B18088
:10F4D000022B40F09F8069F0C7FD454A99F8DC3D5A
:10F4E000C9F8E02D002B00F0A280022B40F096809E
:10F4F000122D2B46B8BF12239BB24345C0F2CD80DC
:10F50000A845A8BFA846B8F1000F9DDD394EDFF829
:10F51000FCB0394F28AD002404E00134444546F8DE
:10F52000040B91D0DBF80030B9F8D41DC3F300729E
:10F53000B9F8D63D01920091B7FBF3F32E4A55F886
:10F54000040F9BB20321FFF787FC0028E5D10525B6
:10F5500001462A4A89F8CA5423460420F8F7E0FFF6
:10F5600072E7274ACDF800B0012189F8CA14734622
:10F5700000210420F8F7D4FF5EE7224B0393130128
:10F580000398C1500F49531C0B70F3E6104A049DB9
:10F59000002342F83A30052189F8CA141A4A534622
:10F5A00000210420F8F7BCFF46E700BF81E800080F
:10F5B000CC6C08086F12833A28600020001BB7004B
:10F5C000C0C62D0070600020A8BB00208072080813
:10F5D000746000200000000038620020B81909089B
:10F5E000ACC5A737ACC5A7366F120339D4190908C3
:10F5F000D9DE000828A6002040420F00741A09082E
:10F6000008190908D460002090190908B4000010F6
:10F6100056498FE6564AC9F8E02D43B1554A0221B2
:10F620000420F8F77DFF0FE74FF4FA569FE52B46CD
:10F6300062E769F019FD504A50E7504A0221042060
:10F64000F8F76EFFF8E64E4A41E64E4A0094032171
:10F650008BE7D6F810C04C49099213464FEA431E77
:10F6600001EB431051F80E208CEA020E1EF47C5F71
:10F6700003F1010309D0102BF0D1059A0023D360C8
:10F68000424B029A43F83A20D0E6059B099AD8608B
:10F69000037F002B3FF489AEF2E7042000953C4A3B
:10F6A00089F8CA0443460021F8F73AFFCCE6059BE7
:10F6B0003849DB6809931A46374B526809989A42D1
:10F6C000364A136B0CBF43F4001343F480031363F7
:10F6D000072383830322059BF3F7CCFD09988068F9
:10F6E0000B90F3F7D3FF0B98069A03680F9223F061
:10F6F0000103327C03602A4B069053F822300D93AD
:10F700000023CDE91833CDE91A331293169312234F
:10F7100011934FF4806313934FF480464FF480535A
:10F72000CDE9143640234C3510930DA94FF4003326
:10F730000E95179367F054FF0698089D039A036887
:10F7400009992A44079D43F0100303606966154B2D
:10F750000A9933F81130A5F8683093815060059A02
:10F76000012313744CE6049D15E700BF808D5B00F8
:10F77000F5DE0008001A0908E98E030834190908A3
:10F78000BDDE000854190908E80900207460002053
:10F790003C1A0908A102000800600240003802403B
:10F7A00084720808C86B080810B5104CD4E904230B
:10F7B000A16882B002FB03F38B428DF8070012D0E0
:10F7C0006368E0680DF10701184474F0ADFF6368E9
:10F7D0002269A16813446269B3FBF1F0013201FBB5
:10F7E00010336360626102B010BD00BF486000204A
:10F7F00010B50379012B84B00C4627D0022B23D1FE
:10F800008368DB070DF10F024CBF01218121FBF75B
:10F8100095FC9DF80F300022C3F3001161F307023D
:10F82000C3F3800161F30F220F49C3F3C00C6CF3E3
:10F83000174281F8F000C3F3801161F31F62DB0906
:10F840002260237104B010BD0020E2E782680DF150
:10F850000F0102F00102CDE900121A46417C90F935
:10F860001000F4F781FDD4E7581600202DE9F0418F
:10F8700082B014460E4601AA50210546FBF7B0FCA3
:10F880009DF80430DFF8F080394F01335B00DBB2C4
:10F890004621238001AA2846FBF7A2FC23789DF885
:10F8A000042008FB03F303F5FA73A7FB03130132EB
:10F8B0009909DB0902FB0133A280A7FB03239B0903
:10F8C00001AAE360512102232846FAF789FD237833
:10F8D000BDF8040008FB03F340BA03F5FA73A7FB75
:10F8E0000323C2B2C0F307208240013292B29809CA
:10F8F000DB0902FB0033A7FB03739B097021E28045
:10F90000238201AA2846FBF76BFC9DF804300133E3
:10F910005B00DBB201AA6380712102232846FAF75B
:10F920005FFDBDF80430134AF17882F8F0005BBA4D
:10F93000DAB2C3F307239A40013292B2228119B19D
:10F94000E388D21A92B222810B48A378084900FBBF
:10F9500003F303F5FA73A1FB03039809DB0902FB28
:10F960000033A1FB03139B09638202B0BDE8F08161
:10F97000D34D621058160020002F3A002DE9F04FA9
:10F98000DFF89C82DFF89C92DFF89CA2A34F8DB039
:10F99000054600264FF4FA7307AA89210068C8F8C3
:10F9A000943089F89060FBF71BFC9DF81C202868B8
:10F9B000892142F00102F9F7C1FD32468821286809
:10F9C000F9F7BCFD012280212868F9F7B7FD012273
:10F9D000FF212868F9F7B2FD324631462868F9F769
:10F9E000ADFD07AA91212868FBF7FAFB9DF81C30B2
:10F9F000286888F88D3031460122F9F79FFD32469C
:10FA0000FF212868F9F79AFD324680212868F9F726
:10FA100095FD07AA60212868FBF7E2FB9DF81C20F2
:10FA20002868602142F01202F9F788FD4FF4005374
:10FA3000ADF81C3007AA022344212868FAF756FCC7
:10FA4000FF2201212868F9F779FD2C680122802125
:10FA50002046F9F773FD0122FF212046F9F76EFDDC
:10FA6000324631462046F9F769FD0622FF2120463D
:10FA7000F9F764FD07AA83212046FBF7B1FB9DF847
:10FA80001C20832142F004022046F9F757FD07228B
:10FA9000FF212046F9F752FD012281212046F9F786
:10FAA0004DFD012280212046F9F748FD6B2294216B
:10FAB0002046F9F743FD324683212046F9F73EFD03
:10FAC000DAF80060C8F890602379012B00F0988084
:10FAD000022B0FD000209DF81C3087F8F000DBB916
:10FAE000DAF800309BB29B1BB3F5FA7FECD90DB06E
:10FAF000BDE8F08FA368DB0707AA4FF0830120461B
:10FB00005EBF07AA83212046FBF718FB9DF81C3037
:10FB100087F8F000002BE3D0012283212046F9F77B
:10FB20000DFD07AA92212046FBF75AFB00228121F6
:10FB300020469DF81CB0F9F701FD0622FF21204662
:10FB4000F9F7FCFC07AA83212046FBF749FB9DF847
:10FB50001C20832102F0FB022046F9F7EFFC012272
:10FB6000FF212046F9F7EAFC012200212046F9F79F
:10FB7000E5FC0022FF212046F9F7E0FC20460022A8
:10FB80008021F9F7DBFC0623B02105AA2868FAF7E3
:10FB900027FC0122FF212868F9F7D0FC00224F2121
:10FBA0002868F9F7CBFC2C224E212868F9F7C6FC0F
:10FBB0000022FF212868F9F7C1FC4FEADB1628680C
:10FBC000B422B621F9F7BAFC0024002E18BF0C2687
:10FBD0000BF07F0BA2464FF0010EC4F3C403303389
:10FBE0006B44E2B213F81C0C04F0070C0EFA0CF193
:10FBF000964220EA010119D903F81C1C0134ECE7F4
:10FC0000A268617C94F9100002F00102019207AA37
:10FC100000928322F4F7A8FB5DE700BF581600208E
:10FC2000D8B60020E0A50020242A0020DA4540FABA
:10FC30000CF200F01183D30744BF0AF1010A5FFA06
:10FC40008AFA0134302CC8D1062305AAB0212868CD
:10FC5000FAF74CFB0122FF212868F9F76FFC00221C
:10FC600011462868F9F76AFC0022FF212868F9F795
:10FC700065FC002209212868F9F760FC00221021A8
:10FC80002868F9F75BFC002211212868F9F756FC77
:10FC9000012224212868F9F751FCFF222521286838
:10FCA000F9F74CFC002275212868F9F747FC01227E
:10FCB000FF212868F9F742FC2C224E212868F9F729
:10FCC0003DFC002248212868F9F738FC2146202213
:10FCD0002868F9F733FC0022FF212868F9F72EFC89
:10FCE000214609222868F9F729FC002254212868B6
:10FCF000F9F724FC042231212868F9F71FFC0322BC
:10FD000032212868F9F71AFC832240212868F9F784
:10FD100015FC252246212868F9F710FC00226021F5
:10FD20002868F9F70BFC002227212868F9F706FC60
:10FD3000062250212868F9F701FC00225121286889
:10FD4000F9F7FCFB962252212868F9F7F7FB082205
:10FD500056212868F9F7F2FB224657212868F9F75F
:10FD6000EDFB002261212868F9F7E8FB00226221FF
:10FD70002868F9F7E3FB002264212868F9F7DEFB25
:10FD8000002265212868F9F7D9FBA022662128689E
:10FD9000F9F7D4FB0122FF212868F9F7CFFB3222C3
:10FDA00022212868F9F7CAFB142247212868F9F7AD
:10FDB000C5FBFF2249212868F9F7C0FB00224A2130
:10FDC0002868F9F7BBFB0022FF212868F9F7B6FB8A
:10FDD0000A227A212868F9F7B1FB00227B212868E2
:10FDE000F9F7ACFB212278212868F9F7A7FB01225B
:10FDF000FF212868F9F7A2FB342223212868F9F7AC
:10FE00009DFB002242212868F9F798FBFF2244213C
:10FE10002868F9F793FB262245212868F9F78EFB1D
:10FE2000052246212868F9F789FB402211462868F7
:10FE3000F9F784FB06220E212868F9F77FFB1A22C6
:10FE400020212868F9F77AFB402243212868F9F736
:10FE500075FB0022FF212868F9F770FB032234218B
:10FE60002868F9F76BFB442235212868F9F766FB0F
:10FE70000122FF212868F9F761FB0422312128685B
:10FE8000F9F75CFB09224B212868F9F757FB05229B
:10FE90004C212868F9F752FB04224D212868F9F714
:10FEA0004DFB0022FF212868F9F748FB002244217E
:10FEB0002868F9F743FB202245212868F9F73EFB23
:10FEC000082247212868F9F739FB282248212868A9
:10FED000F9F734FB002267212868F9F72FFB042289
:10FEE00070212868F9F72AFB012271212868F9F7A7
:10FEF00025FBFE2272212868F9F720FB00227621DB
:10FF00002868F9F71BFB002277212868F9F716FB10
:10FF10000122FF212868F9F711FB01220D21286831
:10FF2000F9F70CFB0022FF212868F9F707FB0122F3
:10FF300080212868F9F702FBF82201212868F9F7E7
:10FF4000FDFA0122FF212868F9F7F8FA01228E2133
:10FF50002868F9F7F3FA012200212868F9F7EEFA88
:10FF60000022FF212868F9F7E9FA00228021286899
:10FF7000F9F7E4FA04220A212868F9F7DFFA2C6875
:10FF8000842107AA2046FBF72BF99DF81C20204668
:10FF900002F0EF028421F9F7D1FA01220B2128683F
:10FFA000F9F7CCFA2C6803A92046FFF721FC07AA31
:10FFB00003A92046FFF75AFC9DF80C30002B00F0F7
:10FFC0005C810A9C04F684549DF80E30002B00F0EE
:10FFD0004A810A9B03F2B22304EB43049DF80F30DD
:10FFE00023B1BDF82C3003F525731C449DF8103067
:10FFF00023B1BDF82E3003F226231C44E822012150
:020000040801F1
:100000002868C8F8E44DF9F799FA286821466DF098
:100010006BFD012211462868F9F790FA402187F814
:10002000F0002868FEF7EEFC00283FF460AD0121E7
:1000300028680222F9F782FA002187F8F000286880
:10004000FEF7E0FC00283FF452ADE82201212868C9
:10005000F9F774FA4FF4005307AAADF81C304421A5
:1000600002232868FAF742F92C6803A92046FFF713
:10007000BFFB07AA03A92046FFF7F8FB5022572130
:100080002046F9F75BFA082256212046F9F756FA7E
:10009000082250212046F9F751FABDF82C204FF4E0
:1000A0007A7148F20E6301FB0233794A934240F2BF
:1000B000EB80784AA2FB0332120C013AFF2A4FF080
:1000C000000306DD52080133FF2A9BB2FAD81B0257
:1000D0009BB21343C3F30722DBB28DF808208DF8DF
:1000E000093002AA022351212046FAF7FFF80A9AA2
:1000F0004FF47A7148F20E6301FB0233664A934271
:1001000000F2C080634AA2FB0332120C013AD2B261
:1001100046212046F9F712FA2046D8F8E41D6DF082
:10012000E3FC02AA01212046FBF75AF802229DF8BF
:10013000086001212046F9F701FA00212046FEF768
:1001400061FC324620460121F9F7F8F92C6803A931
:100150002046FFF74DFB07AA03A92046FFF786FBC1
:10016000482211462046F9F7E9F90822472120469E
:10017000F9F7E4F9032232212046F9F7DFF90722E3
:1001800030212046F9F7DAF90122FF212046F9F75C
:10019000D5F9202230212046F9F7D0F90022FF219D
:1001A0002046F9F7CBF9062270212046F9F7C6F967
:1001B000BDF82E10394A4FF47A7046F6440300FB1E
:1001C0000133A2FB03239DF80F201B0B1AB1BDF8CE
:1001D000222013449BB2002B52D05A1EFF2A4FF00C
:1001E000000306DD52080133FF2A9BB2FAD81B0236
:1001F0009BB21343C3F30722DBB28DF808208DF8BE
:10020000093002AA022371212046FAF76FF8D8F8C4
:10021000E41D20466DF068FC02AA01212046FAF791
:10022000DFFF9DF80850022201212046F9F786F9E8
:1002300000212046FEF7E6FB2A4620460121F9F779
:100240007DF96422012387F8F000C8F8942089F82A
:1002500090300DB0BDE8F08F0EFA0CFC20EA0C00D7
:1002600003F81C0CEDE49DF80D30002B3FF4B6AE06
:100270000A9B03F525731C44B0E640F63634A3E62A
:100280001A46BAE7FF2243E700231A4625E700BFD4
:100290001B0C0100950370F41B280D014963A41386
:1002A00010B5164C84F89510017952BAA4F896202E
:1002B00001294FF0000282B084F8942010D0022966
:1002C00003D06FF00C0002B010BD042304F19402BF
:1002D000FF21F9F7B3FF0028F3D0002002B010BDD2
:1002E0008268417C90F91000943402F00102CDE95B
:1002F00000420423FF22F4F76BF8ECE7E0A50020AE
:100300002DE9F04F9D4F9E4D06683C464FF000088A
:1003100085B0834685F894815B37C4F12D0905F1DA
:10032000940A13E0022B0FD1B26812F0010F4FF0C4
:10033000030352464FF0FF01304601BF03235246EC
:10034000FF213046F9F77AFFA7421AD0337985F8B2
:10035000948009EB0401012B14F8012F85F8951006
:1003600085F89620DED1B368717C96F9100003F011
:100370000103CDE900A3FF220323F4F729F8A742E4
:10038000E4D14FF40743A5F89430402385F8963024
:1003900052460323FF213046F9F7A8FF00238DF8CA
:1003A0000E300DF10E0130466DF068FB9DF80E30F9
:1003B000002BF6D04FF40643A5F894300123714A80
:1003C00085F89630FF2103233046F9F78FFF4FF46D
:1003D00007436C4AA5F8943000240323FF213046DC
:1003E00085F89640F9F782FF4FF40063A5F8943042
:1003F0000923644A85F89630FF2103233046F9F734
:1004000075FF4FF43063A5F894305E4A85F8964046
:1004100030460323FF21F9F769FF002800F0AC8084
:10042000DBF800400DF10E025E212046FDF78EFD47
:10043000BDF80E30B3F5D77F00F08C806AD8512B11
:1004400000F0848078D81D2B7ED10F2608BB0A22AD
:100450004B212046FEF73AFB0F2260212046FEF793
:1004600035FB0D2263212046FEF730FBB8226921BF
:100470002046FEF72BFB40F60D7278212046FFF751
:100480000FFF40F60E627A212046FFF709FF002891
:100490006DD0DBF8000021216DF046FADBF800405A
:1004A0000DF10E02DE212046FDF750FDBDF80E30A5
:1004B0009FED357AC3F3090303EB8303DB0007EEFB
:1004C000903AF8EEE77A4FF4D84267EE877AA5F8CB
:1004D0009420FCEEE77A524617EE903A1BBAC5F824
:1004E0009630FF2106232046F9F700FF4FF407411D
:1004F0004023DBF80000A5F8941085F896305246AA
:100500000323FF21F9F7F2FEB0B385F8940105B09B
:10051000BDE8F08F40F2E132934219D01CD840F28E
:10052000D922934214D040F2E122934202D0B3F593
:10053000E67FAED1642689E7AD2B0BD0D62B01D058
:10054000602BA6D1212681E71E2BA2D114267DE7A0
:10055000C8267BE7322679E740F28F42934203D0E8
:1005600040F29152934294D14FF4FA766EE73146BD
:1005700020466DF0D9F98CE70020C6E7BB72080869
:10058000E0A5002074A600209A99893F03682DE910
:10059000F0411F6A1FB13B46BDE8F0411847002AF1
:1005A000164611DD04460D460E4400E023689B68A4
:1005B000204698470028F9D0236815F8011B1B68CE
:1005C00020469847B542F1D1BDE8F081DEE700BF93
:1005D000204A214B116893F8F22DC90603D5B3F8D0
:1005E000F41D490715D4F2B993F8102ED3F80C3E38
:1005F00052B143B120B11A689B88138370473BB353
:100600001A689B885383704780F00100002BF1D15A
:10061000F9E7B2B993F8102ED3F80C3E002AEED1C8
:10062000002BE8D17047D3F8042E002AEBD058B144
:100630009268B3F8081E094BB3FBF1F35B1013602B
:100640007047D3F8042E22B1936800221A607047D5
:1006500070477047B0000010D8B6002040420F002D
:10066000BFF34F8F0549064BCA6802F4E06213439B
:10067000CB60BFF34F8F00BFFDE700BF00ED00E090
:100680000400FA0508B572B600224FF0FF3193005E
:1006900003F1604303F561430132082AC3F8801077
:1006A000C3F88011F3D1FFF7DBFF00BF00B583B0C3
:1006B0000D49002200920091009B04330093009B9F
:1006C0001B68012B02D003B05DF804FB019201917D
:1006D000019B064904330193019B1A600B6883F365
:1006E00008884B689847FEE7502800400000FF1F2D
:1006F00010B4EFF31183102282F31288094C0A48D8
:1007000022684FF0E021013222608A69C0F8142E7D
:100710000022C0F8182E0A69DBB283F311885DF855
:10072000044B7047242A0020D8B6002030B4EFF3E1
:100730001182102383F312884FF0E023D2B299691B
:10074000186910F4803F0D481EBF0121C0F8181E23
:1007500099690B4B1D68D0F8183E82F3118809483F
:1007600004684FF47A7202FB04F02B44401A002113
:10077000B0FBF4F030BCE3FB02017047D8B60020B8
:10078000242A0020A4360020124B5B68C3F3080320
:10079000FBB9EFF31183E3B930B40F4A0F4C4FF0BC
:1007A000E02C1368DCF8180011688B42F9D1D4F8FA
:1007B000141E8842F5D80A4A15684FF47A7404FB6F
:1007C00005F20021101AB0FBF5F0E3FB040130BC88
:1007D0007047ABE700ED00E0242A0020D8B60020E7
:1007E000A436002090B170B5461EFFF7CDFF044639
:1007F0000D46FFF7C9FF001B61EB0501B0F57A7FDD
:1008000071F10001F5D3013EEFD270BD704700BF1A
:1008100070B5006801220921F8F790FE6426FFF701
:10082000B3FF04460D46FFF7AFFF001B61EB050168
:10083000B0F57A7F71F10001F5D3013EEFD170BDC3
:100840002DE9804883B0431C0193DFF844810A23DB
:100850000093D8F89C10D8F8D830B8F8A000B8F8B1
:10086000DC20DDF804B048834FF0320A1A834FF0E1
:100870000509D8F89C30B8F8A02059690A4214BF7D
:100880005A831A83D8F8D830B8F8DC2059690A425C
:1008900014BF5A831A830120FFF79AFE5646574623
:1008A000FFF772FF04460D46FFF76EFF001B61EB7A
:1008B0000501B0F57A7F71F10001F5D3013FEFD169
:1008C000D8F89C30B8F8A02059690A4214BF5A835E
:1008D0001A83D8F8D830B8F8DC2059690A4214BF16
:1008E0005A831A830020FFF773FEFFF74DFF04467B
:1008F0000D46FFF749FF001B61EB0501B0F57A7F5C
:1009000071F10001F5D3013EEFD1B9F1000F1CD018
:10091000B9F10109ADD14FF4FA76FFF735FF04467E
:100920000D46FFF731FF001B61EB0501B0F57A7F43
:1009300071F10001F5D3013EEFD14FF0FA0ABBF19E
:10094000000F07D04FF0000993E70BF1FF3BBBF11D
:10095000000FF7D14FF47A76FFF716FF04460D46E5
:10096000FFF712FF001B61EB0501B0F57A7F71F113
:100970000001F5D3013EEFD1009B013B00937FF4D2
:1009800068AF01210846F3F7B1FEFFF77BFE00BF19
:10099000F033002018B103685B6903B11847704752
:1009A00018B103681B6A03B118470020704700BFE5
:1009B00038B50B4D0C4620B10368DB6A0BB1984784
:1009C00060B90020C4E90000C4E90200C4E906558A
:1009D0002D2230232061227584F8203038BD00BFDD
:1009E0006C7809080178F9B1F8B5104F0546002672
:1009F00002E015F8011FB1B1D7F81C4E637A5A1CFA
:100A00002344D2B262729972237A9342F1D804F1EC
:100A10000A01002AEDD0D4E900309847667215F833
:100A2000011F0029E8D1F8BD704700BFD8B60020EB
:100A300070B5124C05460E461148FFF7D3FF2A4603
:100A40001049D4F81C0E334668F05AFDD4F81C5EE9
:100A50006A7A32B12B68686805F10A019847002369
:100A60006B7294F8203E3BB194F8223E012213446D
:100A700084F8212E84F8223E70BD00BFD8B6002035
:100A80009C1A090815E1000880B51A48FFF7AAFF6B
:100A90001948FFF7A7FF194BD3F81C4E627A32B101
:100AA0002146606851F80A3B984700236372144B53
:100AB000D3F8AC713B6838465B699847B0B90A26F1
:100AC000FFF762FE04460D46FFF75EFE001B61EB7A
:100AD0000503B0F57A7F73F10003F5D3013EEFD142
:100AE0003B6838465B6998470028E8D001200EF043
:100AF00007FD00BFA81A0908C41A0908D8B60020C3
:100B0000E0A50020154B93F8242E012A00D0704751
:100B100010B593F8292E062A84B00DD00A2A06D1E2
:100B200033F062F90E4804B0BDE810405AE70D48B2
:100B300004B0BDE8104055E7D3F8484E4CB10A4A1E
:100B400007CA01AB03C301A91A7020460922FFF7A7
:100B50001DFD064804B0BDE8104043E7D8B60020AC
:100B6000E01A0908D01A0908181B0908FC1A090814
:100B700080B52F482F4FFFF735FF2F48FFF732FF83
:100B8000B7F84C6E002E44D1D7F81C4E627A32B1C1
:100B90002146606851F80A3B984700236372274B4F
:100BA00000251D7087F8505EC7F8905E23F032F87C
:100BB0002348FFF717FFD7F81C4E627A2AB1214667
:100BC000606851F80A3B984765721E4BD3F8AC71C8
:100BD0003B6838465B699847B0B90A26FFF7D4FDF1
:100BE00004460D46FFF7D0FD001B61EB0503B0F591
:100BF0007A7F73F10003F5D3013EEFD13B683846AD
:100C00005B6998470028E8D000200EF079FC013E8F
:100C1000BAD0FFF7B9FD04460D46FFF7B5FD001B3E
:100C200061EB0501B0F57A7F71F10001F5D3EEE7D4
:100C3000241B0908D8B60020F81E0908BC5F002054
:100C4000C41A0908E0A5002070B50C48FFF7CAFED9
:100C50000B4BB3F84C6E16B970BD013EFCD0FFF7DC
:100C600093FD04460D46FFF78FFD001B61EB050168
:100C7000B0F57A7F71F10001F5D3EEE7F81E0908AF
:100C8000D8B6002070B504460F48FFF7ABFE2046EB
:100C9000FFF7A8FE0D48FFF7A5FE0D4BB3F84C6E0D
:100CA00016B970BD013EFCD0FFF76EFD04460D463F
:100CB000FFF76AFD001B61EB0501B0F57A7F71F16A
:100CC0000001F5D3EEE700BF501B0908F81E090824
:100CD000D8B60020800601D5002933D10CB470B5F8
:100CE000194C1A49D4F81C0E82B007AB069A01932E
:100CF00068F006FCD4F81C5E6A7A32B12B6868682A
:100D000005F10A01984700236B721148FFF76AFE4C
:100D1000B4F84C6E3EB9012002B0BDE8704002B09C
:100D20007047013EF7D0FFF72FFD04460D46FFF751
:100D30002BFD001B61EB0501B0F57A7F71F100011D
:100D4000F5D3EEE700207047D8B6002015E1000883
:100D5000F81E090810F0400031D00CB470B50C46F4
:100D600082B029B1002002B0BDE8704002B07047E7
:100D7000194ED6F81C5E6B7A5A1C2B44D2B2232132
:100D80006A7299722B7A93421AD9069A134907AB61
:100D90002846019368F0B4FBD6F81C4E627A32B153
:100DA000D4E9003004F10A01984700236372FFF789
:100DB0004BFF012002B0BDE8704002B070477047A1
:100DC000002AE2D0D5E9003005F10A0198476C729B
:100DD000D6F81C5ED9E700BFD8B6002015E10008A0
:100DE0000FB410B582B004AB0C4C53F8042BD4F8FC
:100DF0001C0E0B49019368F083FBD4F81C4E627AF9
:100E000032B1D4E9003004F10A019847002363723B
:100E100002B0BDE8104004B0704700BFD8B6002053
:100E200015E100082DE9F0413C4884B0FFF7DAFDF8
:100E30003B4B1B6D5BB119689A880B691A4206D14E
:100E40003848FFF7CFFD04B0BDE8F041FCE6364C72
:100E50002368002B4AD09B699847002846D0236816
:100E6000002B59D0DB69DFF8E88098470646407CC4
:100E70003268337DB1790290307C0190708A0090A5
:100E800052082A48B51DFFF7ABFF00270B3601E0DB
:100E9000B54216D0D8F81C4E15F8011F637A5A1CBB
:100EA0002344D2B262729972237A9342F0D8002A14
:100EB000EED0D4E9003004F10A019847B5426772D8
:100EC000E8D11B4C1B48FFF78DFD6378022B18D02F
:100ED0000ED804F580541848FFF784FD94F8B43117
:100EE000022B15D0032BAED11448AAE71448A8E76B
:100EF000032BA8D11348FFF775FD04B0BDE8F041FE
:100F0000A2E61148FFF76EFD04B0BDE8F0419BE694
:100F10000E48FFF767FD96E79B79FFDE581B09082F
:100F2000CC290020641B09089C3C0020841B090874
:100F3000D84C0020B41B0908DC1B0908001C090858
:100F4000741B0908C41B0908CC1B0908E41B090809
:100F5000D8B600200FB470B582B006AB174C53F86A
:100F6000042B1749D4F81C0E019368F0C9FAD4F881
:100F70001C5E6A7A32B12B68686805F10A019847ED
:100F800000236B720F48FFF72DFDB4F84C6E36B995
:100F900002B0BDE8704004B07047013EF8D0FFF7E2
:100FA000F3FB04460D46FFF7EFFB001B61EB050169
:100FB000B0F57A7F71F10001F5D3EEE7D8B60020E5
:100FC00015E10008F81E09082DE9F041C37913F076
:100FD000C00224D0402A20D1047A1F484D2C35D895
:100FE000FFF700FD1D4B03EBC40393F814528DB1C2
:100FF000D3F810721A4EDFF87480002402E04046E5
:10100000FFF7F0FC57F8241030460134FFF7E8FEF4
:10101000A542F4D1BDE8F04116E6BDE8F0810F4CE1
:10102000427A03F0070304EB8202062BD26D08D04C
:10103000037A0C4804EB8304B4F95C10BDE8F0417A
:1010400088E7BDE8F0410848114683E7FFF7CAFC8E
:1010500000231B79FFDE00BF3C1C0908BC72080896
:101060007C3E0908241C0908141C09084C1C0908AA
:1010700070B508B10378EBB9FCF7D8F81348FFF75F
:10108000B1FC1348FFF7AEFC124BB3F84C6E16B927
:1010900070BD013EFCD0FFF777FB04460D46FFF71D
:1010A00073FB001B61EB0501B0F57A7F71F1000164
:1010B000F5D3EEE7F7F7ACFF044680B2FCF774F81F
:1010C00021460548BDE8704044E700BF641C09089C
:1010D000F81E0908D8B60020501C09082DE9F84F61
:1010E00006466DF005FEDFF83C910446D9F8947E83
:1010F000F8B94148414DDFF82481FFF773FC012620
:101100003F49542304E055F8041F013471B10B78B2
:1011100006FA04F2002BF6D03A42F4D04046FFF72C
:101120005FFE55F8041F01340029F0D1BDE8F84FE7
:101130008AE5024633493046F7F724FC002842D0BE
:101140003378DFF8B8A02E4D2D2B03BF013604F104
:10115000FF344FF0010B4FF0000B4FF0000804E09C
:101160005AF8045F08F10108C5B122462946304605
:10117000F7F708FC0028F3D1012303FA08F3BBF1C9
:10118000000F32D027EA03031F48C9F8943EFFF747
:1011900029FC29461D48BDE8F84FDBE61C48FFF74F
:1011A00021FC1C48FFF71EFCFFF74EFD99F8203E7E
:1011B0003BB199F8223E0122134489F8212E89F887
:1011C000223EBDE8F88F14480C4C144DFFF70AFC82
:1011D0000B49542300E00B7828460BB1FFF700FEC3
:1011E00054F8041F0029F6D1A0E73B430C48C9F886
:1011F000943EFFF7F7FBCCE7801C09083C77080812
:10120000701C0908901C0908B41C09087C3E0908D8
:101210009C1A0908A41C0908981C09088C1C0908B8
:10122000C01C0908D8B600202DE9F84F07466DF01C
:101230005FFDDFF830910446D9F8A06EC8B93D488B
:101240003D4F3E4DFFF7CEFB4FF001083C49234692
:1012500007E00134E4B207EB84022346D2F8041518
:10126000D1B108FA03F33342F3D02846FFF7B8FDB3
:10127000EFE7024633493846F7F784FB78B932483E
:10128000324C2E4DFFF7AEFB2D492846FFF7A8FD47
:1012900054F8041F0029F8D1BDE8F84FD4E43B7896
:1012A000DFF8A8A0264D2D2B03BF013704F1FF3432
:1012B0004FF0010B4FF0000B4FF0000804E05AF81C
:1012C000045F08F10108C5B1224629463846F7F700
:1012D00059FB0028F3D1012303FA08F3BBF1000FF7
:1012E00020D026EA03031A48C9F8A03EFFF77AFB8C
:1012F00029461848BDE8F84F2CE61748FFF772FB5F
:101300001648FFF76FFBFFF79FFC99F8203E3BB1B3
:1013100099F8223E0122134489F8212E89F8223EB1
:10132000BDE8F88F1E430E48C9F8A06EFFF75AFBC0
:10133000DEE700BF801C0908BC7208088C1C090885
:10134000C81C0908901C0908981C0908C0770808DF
:10135000B41C09087C3E09089C1A0908A41C090849
:10136000C01C0908D8B600202DE9F84F80466DF062
:10137000BFFCDFF8ACA1DAF8E86DD0B95C485D4C91
:10138000DFF89481FFF72CFD04F590770125237891
:10139000013B05FA03F33342404602D0A168FFF750
:1013A0001FFD0C34BC42F2D1002E58D0BDE8F84FDE
:1013B0004AE40746024650494046F7F7E3FA002858
:1013C00054D098F800304B4D2D2B03BF08F1010885
:1013D00007F1FF374FF0010B4FF0000B002404E042
:1013E00001341A2C05F10C0524D0D5F808903A46A2
:1013F00049464046F7F7C6FA0028F1D1BBF1000F85
:1014000043D0182C65D0192C55D03C4A3C4804EBED
:10141000440402EB8402012392F84025013A9340F0
:101420003343CAF8E83DFFF7DDFA49463548BDE8E1
:10143000F84F8FE53448FFF7D5FA3448FFF7D2FA72
:10144000FFF702FC9AF8203E3BB19AF8223E0122B7
:1014500013448AF8212E8AF8223EBDE8F88F2C48E2
:10146000FFF7C0FABDE8F84FFFF7EEBB2948214C63
:10147000294EFFF7B7FA04F59C75A16830460C3485
:10148000FFF7AEFCAC42F8D190E7182C29D0192C0C
:1014900019D01A4A214804EB440402EB84020123C8
:1014A00092F84025013A934026EA0306CAF8E86D0F
:1014B000FFF798FAB9E7DAF8EC3D1148CAF8E83DC9
:1014C000FFF790FAB1E71548CAF8EC6DFFF78AFA12
:1014D000ABE76FF07F430A48CAF8E83DFFF782FAAE
:1014E000A3E70E48CAF8E8BDFFF77CFA9DE700BF06
:1014F000D01C0908FC770808901C0908BC72080871
:10150000B41C09087C3E09089C1A0908A41C090897
:10151000DC1C0908EC1C0908E41C0908C01C0908AB
:10152000D8B600202DE9F843A0B1037893B1F7F7BE
:101530006FFD1928044667D8374D00EB400305EBD3
:1015400083034FEA4008D3F84895B9F1000F5BD008
:10155000324A11E0314AD2F804410134192C2CD816
:101560002D4D04EB440305EB83034FEA4408D3F805
:101570004895B9F1000F20D0294EC2F80441A0448B
:101580000027002005EB8805FFF722F886F8A87EE3
:101590002BF0C2FD234886F8A97E4A462146C6F8AC
:1015A000AC7EA6F8B07EC6F8B47EFFF7D3FC95F803
:1015B0004005BDE8F8432BF0DFBD17482346013353
:1015C000192B05DD0024DFF86890134DA046D3E702
:1015D000192B04D99C4210D00133192BFAD803EBF4
:1015E000430100EB81010546D1F848954FEA4308D5
:1015F000B9F1000F0DD19C42E1D10B48FFF7F2F990
:10160000BDE8F843FFF720BB21460848BDE8F84392
:10161000A0E41C46B0E700BFBC72080858160020C2
:10162000D8B60020381D09080C1D0908201D09081E
:10163000F81C090808B548B103783BB1F7F7E8FC96
:10164000013802280AD8C0B207F0ECF8044B05486C
:1016500093F8B81EBDE8084001317BE408BD00BF27
:10166000D8B60020501D090808B548B103783BB131
:10167000F7F7CEFC013802280AD8C0B207F01AF9F1
:10168000044B054893F8B91EBDE80840013161E4F8
:1016900008BD00BFD8B60020641D090808B548B1D0
:1016A00003783BB1F7F7B4FC013801280AD8C0B27F
:1016B00007F06EF9044B054893F8BA1EBDE80840E0
:1016C000013147E408BD00BFD8B60020781D0908E5
:1016D0000FB470B582B006A951F8040B0191FFF761
:1016E000A7F90E48FFF77EF90D4BB3F84C6E36B9EB
:1016F00002B0BDE8704004B07047013EF8D0FFF77B
:1017000043F804460D46FFF73FF8001B61EB050167
:10171000B0F57A7F71F10001F5D3EEE7F81E090804
:10172000D8B6002070B5C379044603F007008CB02A
:101730001546062800F29E80DFE800F00A263537BD
:101740003A42040050480CB0BDE87040FFF748BB77
:101750000E7813F0C0031CD0402B22D13146237ADF
:101760004D2B60D8494A02EBC30393F814229142EF
:1017700059D2D3F8103253F82100002853D00CB0BE
:10178000BDE87040FFF72CBB13F0C00391F9006077
:10179000E2D13F483146FFF723FB15B1E3793F2BF8
:1017A0004FD90CB070BD0E88D3E7B1F90060D0E717
:1017B000096813F0C0030E463FD0402BCFD0F0E7AE
:1017C00091ED000A6846F7F7FFFA01462E48FFF749
:1017D00007FB002DE5D0E3793F2BE2D8237A2B4D90
:1017E00005EB83036846B3F95C3000EE103AB8EEBF
:1017F000C00AF7F7E9FA01462648FFF7F1FAE3795C
:1018000003F0C003402B2CD0637A05EB830595EDE4
:10181000170AB8EE400A6846F7F7D6FA01461D489F
:10182000FFF7DEFABDE7694620461FF0EBFD1A48D8
:101830006A463146FFF74CFFB3E71848FFF7D0FA86
:10184000ABE7217A114B627A154803EB820203EB76
:101850008103D26DB3F95C100CB0BDE87040FFF7A6
:10186000BFBA237A05EBC30595F81432013B00EEAD
:10187000103ACEE713F0C00304D0402B91D10021E1
:101880000E466CE71E4684E794310908BC720808CE
:10189000283609087C3E0908941D0908381C0908E7
:1018A0008C1D09082DE9F04F0378202B8FB00546D9
:1018B00003D115F8013F202BFBD000242B464E4EC0
:1018C000DFF85081DFF850B1DFF850A125461C4603
:1018D00002E00C3646452FD002A930461FF092FD9B
:1018E000214602A874F059FF0028F2D0434802A90B
:1018F000FFF776FA029B5B45304622D01FF052FE7E
:10190000DFF80C91014600223046FFF70BFF5046EE
:10191000FFF768F8B9F84C7E67BB3046FFF754FB19
:101920005046FFF75FF8B9F84C3E002B37D10C3624
:10193000464505F10105CFD1002D45D00FB0BDE8DA
:10194000F08F9DF80C30002BD8D11FF02BFE2C4AC5
:101950002C4BDFF8BC9001460078202814BF1046BD
:101960001846FFF73DFA5046FFF73CF8B9F84C7EB1
:10197000002FD2D0CDE90065FEF706FF05460E46E2
:10198000FEF702FF401B61EB0601B0F57A7F71F1B3
:101990000001F5D3013FEFD1DDE90065BDE79946D0
:1019A0000096FEF7F1FE06460F46FEF7EDFE801BA1
:1019B00061EB0701B0F57A7F71F10001F5D3B9F160
:1019C0000109EED1009EB2E70F48FFF70BF80F4870
:1019D000FFF708F8FFF738F90D4B93F8202E002A8F
:1019E000ACD093F8222E01210A4483F8211E83F8FB
:1019F000222E0FB0BDE8F08FA88208082821090820
:101A000094310908B41D09089C1A0908A41C090886
:101A1000D8B6002010A208086E616D65F81E09088E
:101A20002DE9F04F0478202C8FB0074603D117F82A
:101A3000014F202CFBD038466DF05AF98246002821
:101A400000F0A780012800F0A1803D21384674F005
:101A500054FE0546002800F0358110F8013C202B8B
:101A600040F09581431E1A4613F8011D2029FAD033
:101A70006B78202BA2EB070205F1010503D115F8C5
:101A8000013F202BFBD0DFF878B3D3B201935E4641
:101A90004FF000090DF1080840F29E2406E009F11C
:101AA0000109A14506F10C0600F04481414630468B
:101AB0001FF0A8FC40466DF01BF9414682460246E5
:101AC0003846F6F75FFF0028E9D1019B9A45E6D139
:101AD00009EB49030BEB83034FEA490493F807A092
:101AE0000AF00707062F00F0AD801AF0C00A00F0D8
:101AF0008880BAF1400F40F092801A7A4D2A00F2A5
:101B0000F781BC4B03EBC20393F81492B9F1000FB9
:101B100000F08580D3F810320446A3F1040E6FF074
:101B2000004A5EF8041F284601EB0A0C05E020334A
:101B3000934240F0D5808C4512D011F8012BA2F1D0
:101B40004103192B10F8013BA3F1410B98BF203240
:101B5000BBF1190FEBD9934240F0C280002AEAD1C1
:101B6000A54940466DF06AF8002800F0B281304681
:101B70001FF018FD0346052F00F21981DFE817F06A
:101B8000A701A701A501A501A30116012A2C7FF435
:101B90005CAF9A489A4FDFF894B2DFF87C92FEF778
:101BA00021FF0DF10808FFF74FF802E00C37BB45A5
:101BB00045D0414638461FF025FC41469148FFF785
:101BC0000FF938461FF0EEFC524601463846FFF743
:101BD000A9FD8D48FEF706FFB9F84C6E002EE5D042
:101BE000FEF7D2FD04460D46FEF7CEFD001B61EB6D
:101BF0000501B0F57A7F71F10001F5D3013EEFD117
:101C0000D4E72A78019352B18049284674F0B5FD93
